:10000000FEEFFFF0FF00FF00FF00FF00FF00FF001A
:10001000FF00FF00FF00FF00FF00FF00FF00FF00E8
:10002000FF00FF00FF00FF00FF00FF00FF00FF00D8
:10003000FF00FF00FF00FF00FF00FF00FF00FF00C8
:10004000FF00FF00FF00FF00FF00FF00FF00FF00B8
:10FCF000FF00FF00FF00FF00FF00FF00FF0000EE1D
:10FD000060F0300EEE6AE806FDE1000177EF7FF06B
:10FD1000000E7E6E7E987E867E847E927E903F016F
:10FD20005E933F015E81000E7F6E7E8E1200000E9C
:10FD3000AC6EAC508F0B3009AC6EF00EAC16B40E3E
:10FD4000AB6E000EAA6E010EAE6E040EAF6E3901E0
:10FD500094953901A495AC8E1200000E0001986FA5
:10FD6000000E996F000E9A6F000E9B6F90A1BBEF73
:10FD70007EF0BDEF7EF0C5EF7EF09451982795514F
:10FD8000992396519A2397519B23D890943795376E
:10FD900096379737D890933392339133903390516D
:10FDA000911192119311D8A4D8EF7EF0DAEF7EF082
:10FDB000B6EF7EF098C090F099C091F09AC092F0A2
:10FDC0009BC093F012009CC09EF09DC09FF000016C
:10FDD000A06BA16B9EC090F09FC091F0A0C092F06C
:10FDE000A1C093F0400E0001946F060E956F000EB7
:10FDF000966F000E976FADEC7EF090C09EF091C0B4
:10FE00009FF092C0A0F093C0A1F000019E07000EE9
:10FE10009F5BA05BA15B9E290AE19F2908E1A029C5
:10FE200006E1A129D8A417EF7FF019EF7FF005EFC5
:10FE30007FF01200000EBA6E430EC26E000E3A0141
:10FE4000406F000E3A01416F000E3A01426F3A01D5
:10FE500043693A014469BA96000EBB6ECF0EC36E79
:10FE6000000E3A01506F000E3A01086F000E3A0181
:10FE7000096F000E3A010A6F000E3A010B6F080E6F
:10FE80003A01C06F030E3A01516F000E3A01526FF2
:10FE90003A0153693A015469000EBC6E890EC46E72
:10FEA000000E3A01606F000E3A01106F090E3A0120
:10FEB000116F000E3A01126F000E3A01136F000E1F
:10FEC0003A01146F000E3A01156F130E3A01166FC6
:10FED000170E3A01E56FBC8A000E3A01626F0F0EF1
:10FEE0003A01636F3A0164693A0161691200600E78
:10FEF0003901D96F000E3901DB6F000E3901DD6F5A
:10FF0000080E3901DF6F000E3901DE6F010E0001AE
:10FF10009D6FF40E9C6FE3EC7EF0900E3C01E56F5C
:10FF2000030E3C01E66F1AEC7FF0000E3E01BC6F41
:10FF3000000E3E01BD6F000E0001856F800E846FC4
:10FF4000600013F27CFF00018551030B7D6EAC9EB7
:10FF5000000E0001706FFA0E716F000E726F000ECE
:10FF6000736F600E00016C6F050E6D6F000E6E6F8B
:10FF7000000E6F6FD29CD29E97EC7EF088EC7EF0E4
:10FF8000AC8E7E8E000E0001746F000E756F000E39
:10FF9000766F000E776FEBEF7FF0000E7D6E9C0E9C
:10FFA00000017425F66E000E7521F76EF86A010ED9
:10FFB000F82208006F00D7FF7CFFCB0E00D000D0E6
:10FFC000E82EFCD700D000F0010E00017427000ECF
:10FFD000752376237723000170510001745D0001C1
:10FFE00071510001755900017251000176590001EB
:10FFF000735100017759D8A000EF80F002EF80F034
:020000040001F9
:10000000CDEF7FF0000E0001746F000E756F000ED3
:10001000766F000E776F2BEF80F0000E7D6E9C0EDA
:1000200000017425F66EFA0E7521F76EF86A010E5E
:10003000F82208006F00D7FF7CFFCB0E00D000D065
:10004000E82EFCD700D000F0010E00017427000E4E
:1000500075237623772300016C510001745D000144
:100060006D510001755900016E5100017659000172
:100070006F5100017759D8A040EF80F042EF80F037
:100080000DEF80F07E9EAC9E070E00019D6FD00E9E
:100090009C6FE3EC7EF0FF00FEEFFFF07678756B6F
:1000A0006A6D6B666869696C72737072757372766B
:1000B00078747178756B6C73736C6C726E686A713E
:1000C000747171716F7176767778747173716F7402
:1000D0007673707276777475757376797A73737DCB
:1000E000807C7E807C83898B8A8E8D8D8E8B888AA6
:1000F00089868589918F878791938B8C9699959323
:1001000095928B8A8D8B87888C8D8780828585815F
:100110007E7C7E8177767F837F7F807F89848181EB
:100120007F8082838A93938B837E7F848586868A71
:100130008E8483898984838384827D8388817D8280
:10014000837A777C7F7F888C858184858381868C88
:100150008E88808286858589898383888589928F28
:10016000898A8A868992938D89908D87868A8A87E3
:1001700084817B7574756E6E7471666971736C6F52
:1001800076726D73746E6D6F6C696B6E73777C7E57
:1001900077737A7F7A787F7E7D868C8784817A7B7D
:1001A000868B878383827D7A797976757675787B7D
:1001B0007A74737578787878797C7F7C7B86877F92
:1001C0007F7F8082827C7C7F82827D78787D79755A
:1001D0007D8281848A8C8B8A8C92938B88908D838C
:1001E000848A8A888A8985848588898983818486A6
:1001F000837F7E7C7B78787C7D75747D7B77787A55
:100200007873737A7E7C7C7D7B8082807D7F7B7A35
:100210007E7E787C848984818183848682838584C0
:100220008485888D8C898E8F8680838688898C8C46
:100230008A8F938D898A888484858A8F8E8C8D8C11
:100240008887898D8B8787858183827F7F7E808861
:10025000847F7E7D787679797A8489807B828880B4
:100260007C7D7D7E7F7D7A797F81797173757372F4
:10027000716F6B6C6E70716F70737876737A7A765B
:1002800076716F7678757675777A7876797C787707
:100290007E7F808180868985858A85818B8C8A8A0C
:1002A0008B85858A87848A8A888D8C8888868888C9
:1002B000868C90898C94908D8E8A878A8886848695
:1002C00089857F84878380838382817E81827B7E10
:1002D000898980828B8B82858E8C868A8A878B8F98
:1002E0008B8683868B86828585868D8E898887829C
:1002F000838A8C8A87878B8D8B8E918E8C8E8F8C48
:100300008A898A88828185827F8083817F838785AD
:1003100081808586878D908E8C8A8A8D8D8788884E
:10032000827E8185858786828284858080838180A4
:100330007D7D7F7D7B7D7C7C7E7E787B7D7B787305
:10034000727274757777757576757371707074766F
:1003500075757471727A7B75737577787A7D787537
:10036000767779746F737A7977797F7C797A7A7D09
:1003700081817D7C7B7979797B7D7F838683808099
:100380008687817C7E817E7B82878888857F7D7E53
:100390007E80818081868382828687858788868425
:1003A00084868A8E89837F8185847F7D7D7D7A7A2C
:1003B0008086878484878A8B8882818687848082EE
:1003C00086868283838381818283827F7C7E7F8213
:1003D00083807F81827F8284807E838483848686FB
:1003E000858788868588857F7E7F808386888D91B6
:1003F000938E8B8E8E8A888989898B8D8D8C8D8C3E
:10040000888586847C7D82827F7F837F7F848482CF
:10041000817D7879767375767271707177787A7A72
:100420007C7C79767777787A7E7B7876737374774D
:100430007B7C7A7877787C7A797C7D7C7977777B1E
:100440007D7C7D7F817D797A7E7D7C797B82827CDB
:10045000797C7C7B7B7B7C7C8284807F807D7A79CD
:100460007C818182817C7E82817F80807F868B8C73
:100470008E8B8A8986818386888A8C8B8B8B8A87F0
:100480008584828082848786847F7B7B7D7E838552
:1004900085878B8A8A8C8D8B8A8785878B8D8B8AC3
:1004A00087888D8F8F8C8B898888878889898B8DA9
:1004B000908D8C8D8B8C8F8F8B888A8C8782817F9F
:1004C0008286837D7D7B7A7B797B7D7E7B7D7C7D57
:1004D0007D7C7D7D7A7A7B7A7D7D79797B7A78786F
:1004E000787D818182817C7C7E7C797976706E7169
:1004F0007B7F7D7F807E807E7B7A7B78797A777642
:10050000767A7F7D7A7A7B78797A7A7A7474797957
:10051000777B7C7A7A7C7A787A7F807E7C7B7B7C26
:100520007F7E7C7F7F7F8182828586848586847FB3
:100530007E808180807C7A7B81848181868C8882A8
:10054000807D7A7A797A7B7A7A7B7D8285838180D5
:1005500082817F7D7F80807F7C7C81817E808181A4
:1005600082838585838486868686858285898C8D2F
:10057000898888868382817F807E80838385858346
:10058000828181858682808388858081858683803B
:10059000818383858A8C8A87848585858382878801
:1005A00085868687837E82898A8B8C89868A908FCE
:1005B0008E8F92918D8B8A8B8B89898B898887838B
:1005C00084858484868583807E7D7C808283817F10
:1005D0007B787A797A7C7C7A797D7F7C7C7D7B7B69
:1005E0007979767374777572757677797C7B7C7C94
:1005F0007A7976767572757A807E7E807D77777966
:100600007D7D7E807F7C797A787877777B7F7E7F2F
:100610007E7D7A79787875787D7D7A78787B7C7A3A
:100620007C7E7D7F80807D7C7E7B787B80838384E5
:100630008787878686898C90908D8D8E8A86888A1A
:100640008A8C8A898887888B8B898B8A878889841A
:10065000878A8987817E878C84818583838485844A
:1006600084838384848484858889888985827F7C47
:100670007C7D7C7D7C7D7E7B7977777778767676DE
:100680007274797C7B787B807E7C807E848D8B8588
:10069000888D8D8E8E8A88898986838583838583DC
:1006A0008182817E7E8084827E7C77767977757484
:1006B000716F74767674716E6A6E7679767573730F
:1006C00073757677797878767578787575777B7FB6
:1006D00082817F7B7D80827D7A7B7F81807E7D7C35
:1006E0007E7D7A7B7D7E7E7F7F80818384817F7F1C
:1006F0007F82848282807F838585848281848583D2
:1007000083868B8D8E8C8B8A87888A87858A8D8A53
:100710008989888D9192908D87898B8B8B8785862F
:100720008687898784848584848483848684888A70
:10073000898889847D7F808283848584838283867F
:100740008684838786848183858485858181888763
:10075000838585817F80848482838787858584855E
:10076000888C8C8B8C8E90929392928E888A8C8BB4
:10077000878787888785838282838384848484872C
:1007800089868281838382827F79757979797A7C7F
:100790007C7A7B797D808080828384848988837F52
:1007A0007D807F7A76767676736F71737171706EF5
:1007B0006F6E6D6F6F6C6B6C6C6C6A6A6C6C6C6A74
:1007C0006C70706F727371717274757676797A79F4
:1007D00078787676747272757B80818485878A8C4E
:1007E0008E8E8C8A8783868A8C8A89898887888579
:1007F0007E7F8587878786837F8083807C7C7E7FE2
:1008000084848280848688868584888C8B89848091
:100810007F8181858785858483848582858683849D
:10082000858687868385878585868684827E818482
:1008300083807E82888B8A88888888898986858655
:100840008382868686868183898B8B8B8A8C8D8E2C
:100850008E8D8783878A87868580808080807F7E53
:100860007E8080807C7B7B7D7F7E7E7E7F7F7E7FA7
:100870007A78797D7E7C777577797C7E7D7C7D7BCF
:10088000787A7F82828281838282807F7F7B7C7C78
:100890007977747576757675767877757A7D7E7FDB
:1008A0008281817F7D7C7A797C7A75787D7B7B7C87
:1008B0007A7C7B7A7B8081858480828382817C784C
:1008C0007F817F7F7C7C808284898D8C8E8E8987DE
:1008D000888A8F8E8B8A898D91909091938D8A8D45
:1008E0008D8D8B8889898785878A8B8C8E908E8A5F
:1008F0008A8E8E89888785828188888485888D8F75
:100900008E8E92918E8D8A898D8B87858281828150
:10091000818383848586878986858282847D7D82A2
:10092000888B8C898586898C8B878485898A898642
:100930008483858680808487868586878685848370
:1009400082807B7A7B7878787777797B7C7F7F7CF5
:100950007C78767A7A78787674727374716F72753F
:1009600074777D7F7B76757575757571727274732A
:1009700073736E6A6B6E717274777A7C7E7F81801E
:100980007E7F7F7E7B7B7B7C7A7A78797B7F82809F
:100990007C797B7F7F79777678787A7A7A7D7F80A9
:1009A0007F8285817F807F7E7E7E7D838D8F8D8A15
:1009B00087868888898884848A8A88878586898AC0
:1009C0008A888A8A8A8D8F908F8E8D8E8C8B8C8B65
:1009D0008A88858583828586898B87848B908B8A9C
:1009E0008C8B8C89848586847F7C7C7F7F818381CE
:1009F0008285868582818085868688888887898C9D
:100A00008F8F919391908E8D8A8889898687898628
:100A1000868989837E828A8B8986868780807E7E8E
:100A20007D7D7C7C7E7D7B7A7B7D7A7A7C808180FB
:100A30007E8081807C7D80848687847F7A777574D0
:100A4000757A7D787A7D7B79787978737172747331
:100A50006F6C6C6B6C6C6967696D6C6A66686E6EE6
:100A60006A6A6D70727271787A7575787776767455
:100A7000737472757B7D7D8186878B8C8887898472
:100A800084818080848684817F7F8084848485853E
:100A90008282817D7C7C7A7D808181807B7C7C7D73
:100AA0007F7F81827D7C7F7D7E8183808184888D34
:100AB0008D8988898D92908E908F91979A99949133
:100AC00090918F8F8D89888A8A8887888686868587
:100AD00085878788898684868584898B8B8D8C8A97
:100AE00088898988878B8C8B87878886858686848A
:100AF0008283868583817E7B7B7B7A77777A81810F
:100B000081817F7D7E7C7B7C7B797B7E807F808208
:100B100084858486848588898784827D76747978C3
:100B200073726E70767A746B635E60656866666316
:100B300061606165686B6E6D6D71737372757677E8
:100B40007778797B79737173727577787A7B7A7F2E
:100B5000838787868382828584848888898B8C8C2E
:100B60008986828081838585868788898582848439
:100B7000848B8D8F8E8C919897979D9D9691919057
:100B8000908F8C86848891999A94919495908E8A6E
:100B90008884868A8A87919CA3A9A9A4958A817E44
:100BA0007B78797E87909193959493897C736F6B12
:100BB0006B70747A7D7D7E7E8086858487847F7E5F
:100BC0007C7A7B7A78777877777B848E9397958F0A
:100BD0008F9492919596938F9099A7AAA8A8A2987E
:100BE0008F8B8B959C9D9B9B9CA3AFAFA697887D7D
:100BF0007C7B71645C5A5F666E767A756654515B75
:100C00005F584E47413E3F47505557565E646970A6
:100C1000746F6A6A665E5B60676D707682808085DD
:100C2000888985878F908F8F8B8685838692979210
:100C300091959391959B98929197A0A39F9EA2A323
:100C4000998D8D9497938A89929D9E9D9DA09D9646
:100C5000909297988C8386877B675C5F6E7E827F9D
:100C60007C746F717273716C635A51493E3F4B5380
:100C700051505158677681898D8B837A6F655F619A
:100C80006B7D91A0A6A4A1A09E9B9B9EA0A39F95D7
:100C90008E9092919090908D8A8A8C8EA0A2A2A222
:100CA0009F9D9A97969B9D9C9CA09B908E909196C1
:100CB000A1A5A29C9796979CA29F988E8A877E73E7
:100CC0006D69696C7176736B655B575F635A4D43F1
:100CD0004350657374727065564A4339313131330C
:100CE000384252656D6D6E716C645A5353575C6433
:100CF00074838F9899918F8E8E939B9C9B9F9C90D1
:100D0000847F82868887888A8A8C9094979B998F23
:100D10008A898A8B8D909AA1A49E9187848A8E92CB
:100D200095938E87898E8E8E9399A3AAA290837FA6
:100D30007A77797B807E71655E5E62696B696F78B8
:100D4000796A554C4D525D666E7676706C6D6D6A43
:100D5000686560605D5A6171828B90918D88847D39
:100D6000797A7D8081858F95999EA1A7ADAAA7A448
:100D7000A4A4A49E958F8E8E8A89898B9196969530
:100D8000929092989A96928F8E9597918A89868260
:100D90008187909898959293918A868B928D86817F
:100DA0007D746E6C6A6A6C6B655D5A5C5C5B5958ED
:100DB0005957534D4D535455606B6A6B706F69634F
:100DC0005F605E5246485354565C656E75797F8607
:100DD0008C8F8E8B8B898B8F8E8E959C9FA5A9B0C7
:100DE000B3AEA7A29F9D96908B8D91919090908786
:100DF0007F7C7E8384817E838583848987888986BE
:100E000082817A777B7F828687888A8A8E908E928B
:100E10009B9A948E8B8B8A8075757772605F6468FD
:100E20006A635E61686B6C6B6B686461646567754F
:100E3000828A91908F90887971706B636162636C24
:100E400079828A96A2A6A5A3A2A3A8A29EA2AAADD1
:100E5000AAA9AFB5B4B0B0B1B4B2A5A0A5A59E92F1
:100E60008E8E8B86858585827E7F7F7C7E868C8E2E
:100E70008D8C90928E86868885807D7A7671778635
:100E80008E8F8B8F95958F8D8C8677696565656361
:100E9000626060615E57514D4B4C53576162625FB7
:100EA00060686C635F6E82858383817C766E615B34
:100EB00058534E4E55626F81939C9F9F99959B9E70
:100EC000A1A7ABADAFAEAEAFB3B4BBC2C1C0BEB8ED
:100ED000AFA196908C8A85817B736D6A6866697014
:100EE00072706F71767E838990918B827B787B8024
:100EF0008585878B8B8D939FA6AFB7B7AFA99E894A
:100F00007D7A7D817B6E6A6F7171706F7676727596
:100F10007C7E7977797462545969717A97948D855A
:100F2000766B67543E34312824314A63788A969828
:100F300098928A8A9096999FA5A9ACADB0B5BAC08F
:100F4000C1C0BDB6B0A99B8F8A837B79766C64667D
:100F50006A696868686E71696A7984837F80868847
:100F60008686878C8B84869294949BA3A8A7A8B32B
:100F7000B4AAA59C8A77675A55544F505051575F71
:100F80005C55565D696F7168554A4E504E566F8B71
:100F90009386776F7683795D442E201D3753676E75
:100FA0006E72849BA6A49D91898A8D93A2AFB2AEE6
:100FB000A4A2B1C2C5C2BBAFA49C948C88837A6A38
:100FC000626A717473736F6D6E74808A8E8D939D77
:100FD0009F9D98959394999DA09B949197ABB7B141
:100FE000B6C9D5D1C0B5BCC2AD9080786F66605F20
:100FF000696F69564A5C7A8A86735B556468595191
:1010000063787C6C5C647D8F7E522D242F39363260
:10101000323B4555678195958779788AAAA197953E
:10102000A0AEB5B9C1C6C2BEB9B7B6AF9C8D8888EF
:1010300084766D727776716C6E757B7D8287898B15
:101040008E9AA9B0A9A29D9CA5B0AD9F97959AA391
:10105000A8A6A3ABB2ADA0A1B4C0B3906E62686401
:101060005341302B36474C4B4F5555535C70807075
:101070004D4158747A64525D74735D453531343432
:101080002A283343494B5973817D747482979F9703
:10109000979F9D97999FAAB7BAAEA4A7AAA79F9119
:1010A00088847E797F7E7470777C838980777C8E5C
:1010B0009C9E9C9EA0A2A8ACB4B6AFA4A3ADB7B2B0
:1010C000A29EA7ACB3BBBDB3AAA5B4C7BE99838D7E
:1010D0009D9073636664513C3C596F5A32325D7E19
:1010E00077625E6E878C76687980674A3F3A3832DD
:1010F00024212F3A3736475B626A706F7D8E837E7C
:1011000093A2A8A39EABA38188AAA5A4AEA49991FB
:1011100083838B837A746B6F797E7E7E7579868C00
:10112000898F979CA3AAA6A3A7A59EA0A7A89F96D0
:10113000929EB0AC91899FAEA5928E9DACA4877A09
:10114000848876645D5F5F544444535542394B5FF5
:101150006965515175948A7678838377675B5044CB
:101160003D393C3D3024304D5E605D606D7D83894E
:10117000979A98A2B0B3B3B2ABADB9BAB7B3AC9EBD
:1011800092877F7E7D786E707D7F7A7A7B7C838587
:101190008997A6A79F9BA3B0B8B6AAABC3BAAFB1B5
:1011A000B7B6B4B3B9BBB0A6B0BAB6AEB3BBAE9D1A
:1011B0009DA0978B7A6F727167605D5B5B5650572D
:1011C0005A524E5D6B655B5F71878A72687B84796A
:1011D0006F63544A473F3B3F3D404F5B5E646667E9
:1011E000707A7A84999F9C999BA0A2A0A3A7A6A29B
:1011F0009A8E8B8C85858273696D70737A776F6830
:101200006C747B7F8384848B9393969B9CA2A49D18
:101210008E8B9191908E8A89939791909DA0978DB6
:10122000909893857D7A797369605E5A5658544CCC
:10123000494C4F5357565C636B7071747F88898239
:101240007D7C7C7973675C554E4B4A494B4F4F50C0
:101250005E6A6F747C8491989594999FA7A9A8A8B9
:10126000AAA9A6A19FA19E938F979A9999969395C3
:10127000999E9E9E9E9E9C9C9E9FA2A1A09F9F9D8C
:101280009B9794908A86888B8A857E7D82868788C4
:101290008785878C8D8E8F8A86817E78717072703B
:1012A0006F6D69696D6F6F6F71747B818285888ED8
:1012B000909093938E8989857B75716E6C6863615C
:1012C0006262605F60625F5F6973797E7E7E858A3D
:1012D0008E929593908F91938E85818284827B7973
:1012E0007D8185838080858C8D8B8B8988858386A5
:1012F000878480807E7D828273686A6A6C706F7377
:1013000078716F7574727879787F837F7F858B8F22
:101310008C89898B8B86818282818380888A848272
:10132000817D7C7D7B7D7E7C7771706F6E6B66606E
:1013300062625D5F6766666C6E707476797D7F86CB
:101340008A8E96979499979596979B9E999699963B
:1013500095A2A7A29D99969592939895908A84813B
:101360008588878785848994938E908E8B8B8A89D4
:10137000837E858680868A898C8F8A8B88808892F6
:10138000918F908F908D8A8F908E8C8A8C8F918F79
:1013900090918D8C8F908E8E8A858586888D847DA8
:1013A0007C7B7A756A666B6D70706C6B69686B6953
:1013B0006E797B777C7E77767A7A78727072767BBC
:1013C000797A80817C797671747A777175777A7C95
:1013D000797676736F7070737A78767E7D7B827F94
:1013E0007E87847D898B898F8F8A8F918F8E91954F
:1013F000969295969494918F938F8C919089847EF8
:101400007D7D75717778726D6B6F736B64686D74C9
:101410007F8279737A7E75675D56534D5256524C72
:101420004C525B63666770777779808588827A7DB6
:10143000827F828381858D8782837F7D80787179A9
:101440007E7A7B8183878B8A8784868787898A8D4A
:101450008B8A8F929394918A8A8B898B8C8A8A8DBE
:101460008F90959B9C998F889097918F8C868C9369
:101470008D8B8F8B86858A9294898287929BA19D82
:101480008D828997A5BBBE9E86899394805D443DDD
:10149000363C494B4445495B7A89898B8E9EA59F92
:1014A0009E93868B918B847A6A676D6F7370666486
:1014B0006A72767369656C74797F7F7C7F868C92A3
:1014C0008F888790969A988F909FA6A9B0ADA7AC69
:1014D000B1B0B3AB9896A5B5B9B3A1908E9BA89CBB
:1014E0008274747A7E7567594E4C546A77685B5C77
:1014F0006B84969182818992A3C4D0A1747B8680EB
:101500008A80491D172027344043485A749ABBBE2D
:10151000ADAFBCC2C5BFB5A99D9898957F737882C1
:101520007E75797B7A7B81817D78737883867D78FF
:1015300074757D7F7B7471717B89929594969EA45E
:10154000A0948C8C919092928D8E97A0A3AFB7AB04
:101550009491A5AE9975615E5A51463E3325222A73
:101560003B4C4B393960898D6F5B6C7F7076A5A0E1
:1015700061363240523B120608020B1921313E4AB5
:101580006A9BB5B2A8A6ABB3B7B2A79584807F7F9C
:101590008077737B7F808892918F909396908C91C7
:1015A0009899959392969A9A97949291949EA8A6B8
:1015B0009C99A3AEACA197969FA5A6A4A3A9B9B9DF
:1015C000AFBBD2C1A2A2B4B0977661626456453E69
:1015D0003E3D3D41516367616B819BA49584858548
:1015E0007A8095936C40313D46381D0D0F161D29AC
:1015F0003F55636F83A0BCC9C8C5CBD1D1C7BDBAA5
:10160000B8AFA7A3A9ADA8A1A2A2A29D9798978EB3
:10161000868B9092928D8E92979A98958E8F8F88C6
:101620007D818F959498A2A4A0A1A7AAAEAEA8A4EC
:10163000A6ABACAAB0C1CEC4ADA7B0AA9177656085
:101640005A49404043413C3C53676A62626A7A7F30
:101650007B766E625C5E594C3D34384545311F22C5
:101660002D3331292F3C3E445C76817F7C869AA8BD
:10167000A99D928E90939AA2A6A1958B8EA1B0AAB5
:101680009D9599A2ACB1AFA6968F99A096898483B7
:101690008080868479716F70747678787B83858892
:1016A00091948D91A0A6A09B9CA0A2998F90948AC2
:1016B00073666C75684C404C5E616062686B6E7CF2
:1016C0008A8C877D73747E7C746C666563606567E5
:1016D000615C554E55677674686671839196928603
:1016E0007979879495938B868B90999F9FA0A09DE5
:1016F000A4ACAEA9A0989D9D9B9F958693A29C9C0F
:10170000A1A4A7A7A09997949087807D756C6A6D16
:101710006E6F6A6362697476777E86899B9F9F9FEE
:10172000A5A8A49E948C878686807B7370737A7F2D
:10173000837E7880888E908C827B7B736B66645FFF
:101740004E42404852534A403D41505A5955534FDA
:10175000566569645A545E738378686D7F878583A4
:10176000828281808697A5A7A0999B9D9FA19E9626
:101770008E8A878D9A9F948E939DA8ABA8A6A59ECE
:10178000989CA29E91817B7D847D6D626465656578
:10179000686D6A666D798285868A91969598999426
:1017A0008F8B8D8C8E949B9C9A9AA9BAB1A1A2AC76
:1017B000AB9F8F868482776D6A6C6C636064696AA4
:1017C0006A6B70757A7E82827D747281867A6F6BA5
:1017D0006E767566667E8E847B8AA0AAA0928E8CB9
:1017E000857C797F8475686E7F847C7276878D8C2A
:1017F000959F9F999DA9B1ABA5A7B1B9B9AEA7A473
:1018000099908C8A85736058575554535053555648
:101810005C5C58616F7979706C788A918C939CA02C
:101820009B9B9D9894979DA19E968E8B909187717E
:101830005D63706F655B52565B555A6254444C5FF2
:101840006968554956656467736F605B6282ADAEC7
:101850007E5D6D97B19A6F594C4650575140272D78
:101860005E7E72605D6A879BA1A6A7A4ADC9E0D821
:10187000BFB9CBDBD7C5AEA3A29D968F7C60637644
:101880006B5757574E56615C5A65717788998E7EB3
:1018900098BEBBAAAEB4ACB3C5BDABB3BBCACFBFD9
:1018A000CFE9D5ADA2AFBEAF7C5F66727468564B10
:1018B0003B232F514624192037585E4D4F585E78F0
:1018C000908E9DB692698AB59962433F48472E151E
:1018D0001614183753483B4E7095B3AEA8C7EDF6B3
:1018E000F6FEFAEAE5E9E9E6CFA1949F8E7164502D
:1018F000404043433D32415B5A5E645D6B7E818D67
:10190000A4A5A7AAA3A9B5B6B7B5AEB4BEBAB9C9BE
:10191000D0C2B5C2DBE4E4DCC9BBC1CAB088656B28
:1019200084835D312B403C261E211C191A2644520B
:101930003B35658866497698764E49514D32120D91
:10194000140C0A161B1513213E575C576181A0B673
:10195000C9D6D5D5E6FAFFF6E8DDDDD5B293886CB9
:101960004F4A4A321A1927333A424C5B6E778097B6
:10197000A1A2B8C9C1C3D1D5D5D9CDC4D2D7C7C406
:10198000C9C4C9CDC0BDCED5C5BDCAD7C8ABA3AD2E
:10199000AC9D88756F67554D575238315757606900
:1019A00057496483816D574244544F3F322828364B
:1019B0003C2D2322212C424537405E717D93979226
:1019C000ABC7D1E0F0E5DCDFD8D0CAAA8580866E4F
:1019D0004F3A21101220272A1E17335C67636B7F52
:1019E00099B4C4CCCFD5E4F3FBF4E3DFE6E2E1E263
:1019F000CFBFC6CBBBA6A6B3A78991A79E8B837E7C
:101A00007D797978716558546C826E607B815F5DF9
:101A1000848B69565550483A25242B1A3A351A2199
:101A20003336383B3D4E58555F797C798AA3B0B246
:101A3000B2BECEC8B8B7B19B8A857B61484B5139DD
:101A4000202A3C403D3B4458616F8E9B97ACD5E6C5
:101A5000DDDEEEFAFDFEFCFAF3EFF3FAEBD1D3EDA7
:101A6000E6B8B2CEC0968E9F9B88726B736B555949
:101A70006B614B515D63635859788867536E877704
:101A8000606B806D49444E4835364542251A3140D9
:101A9000372D3139424C586871767D8EB0B6B7C15A
:101AA000CCC7B8B2AB97827D7454403F3626212A0A
:101AB000312C2939576C7D92A4ADB6CCDEDBD6DC57
:101AC000E6EFF0E0D4E2ECDED0D8D4C0C1C1998C0E
:101AD000B9BB87829EA29882666E7F6D61675B4507
:101AE0004553544737313D4F4C3A3D6980543F751B
:101AF0009F8364697A816B4E535C3D2130483A2064
:101B000028403B323E494C5966768C9899A6C0CF06
:101B1000D2D4D5D7D8D5C7B5A1938A7A65554A4BC3
:101B20004E4F555A63768996959AB9D4C5B5CAD29F
:101B3000CDE2EACFC1D0DEE7D4A1A2D6D5A39CC323
:101B4000C7A096BDB97C73A3A7887B747B886E4FB2
:101B50004F4D38333835271923434227294E6260C9
:101B60005D5B657F998E6E6E8C97826D5845475090
:101B700044261924383F3930314D6B6E6A789BBA50
:101B8000C0BDCEEAF3F2EFE5E7F2ECDAC5ABA7B5FC
:101B9000AC8A7A7B7A776C605A58657257556F8E2B
:101BA000886B6F94A7957E8BA7A298A8A78983A11D
:101BB000B9B0877099C7AC86A6BF958AAD9C7B8863
:101BC0008B7770654D464D46362E2F38463F26346E
:101BD00060614C5C6C626D908E6F738C8B807B61EE
:101BE0004751646452352B46645D453A4F687374BF
:101BF000656288ADA59CB2C7C7C2C5D6D9C7CAE4BD
:101C0000DCB4B1D2DCB68D96BDCBA78DA5C3B5A58E
:101C1000AAA99F9C958F96927C7681846571836F2B
:101C20005666868B7754527F8D676FA4996677B01E
:101C3000B3867084979286898257487F9E642B4131
:101C40007F8F5C304E80765D6E81654C70976D370E
:101C50005DA5A46A4A62949E6848646E595C6645B4
:101C600027417880523460A0AA8E8393B1C0AD948E
:101C700094A2A691869DA489859C9E8F817992B419
:101C8000996D89C7C5989AC7D0ADB1DBD7A49DCF50
:101C9000DBA27994BCA1625A89977560696B7471F3
:101CA0005A526377817552385B9C93563C548DB67B
:101CB0008E444586A083776D4747879058475B6978
:101CC0007E724F667F6A6D7F6B6674747873505155
:101CD00086A281484687B19470758B9B9D928B81BB
:101CE00069739D997172A0BAAB969AB3BDAE937C9D
:101CF00073737E846648587372737A6A6991B19B74
:101D00007B89BDE5D7ADABD9F5E0C2C7C6B1B5CAD1
:101D1000B37F6E86978360515A5F5E5F515B6B69DC
:101D20005D5F6565757E635070A5AC7D546593A558
:101D300096683F54808D887155698D7D70867F6669
:101D40007282715E687E7553475B6A635A60625146
:101D500053767A5D567092957367879E8C6B6A8F07
:101D6000AF956E79989787705D5148474A413545E0
:101D70006573707891A4A7ADBAC4CCD2D2DBEAE285
:101D8000C8C6DBE4D6C1B6B5AFA5987C5F5E62631A
:101D900067532F3D75876C5D6C7E8081837A79886F
:101DA0008E8684939485838F9B9A897E8894968A65
:101DB0007F899A886C687B8A744546798252394F4C
:101DC000665A4340506259445B857E687B9E9561AC
:101DD0004F94DBC4796DA0C3A670524334292113FC
:101DE0000E161F335163637099BCC0BFCBD9E2E8B4
:101DF000ECF0F0E3CDBBAFB7B4895E64848865478F
:101E000052717D8184818AA4B6BAAF9F98A5B5AF7F
:101E1000938394A6A59C95919BABA9A7B8AEB2C697
:101E2000CAAE96A6D4E3AC7282B6BB885A62848AE4
:101E30006F5248494C4B443E3B343A545C4D403E13
:101E40003F517B9C8D645B747F6B4F2E1108131880
:101E5000110C0E1E3954656D77889BA6B3BFBCADBF
:101E6000ACB9C2B39B93A1ABA498897E797E857EE1
:101E7000695E6B8089847B7B828D96978E84899C3A
:101E8000A9A79C9FAEB9B5AFB0B4B0A39BA0A49CCA
:101E90008F8C8C909AAFC6C4A298C0E1A0888F9D09
:101EA0009C84664E474D53534B4039476876655581
:101EB0005B68768D9D937156565D51331608070900
:101EC0001013171E2E4D6F81898E97A0A3A09F9C83
:101ED000958B827E858D8A868EA4B5BBB5ABA9A96C
:101EE000AAA79B8A7C797C7F7D746D6F798CA0A377
:101EF0009C99A4B8C4C4BCB3A9A0A1A299837275CB
:101F00008E9B897783A2B9BABCCFD6C3BCC8CEBDDD
:101F10009773666A65574839313747596360647407
:101F20008B8E7869655F6A868F704F4953533F2364
:101F3000120D0B15202A34455C7F9EA8A7A6A196FA
:101F400089878E856F686D7282949CA8BAC9D5D630
:101F5000CCBFB3A1938C7F6B534B5B6D6F6D768C55
:101F6000A4B2B7B6B1B2BBBDAF9B877E7F85827985
:101F7000767F92A5B6BBB4B9CAD8E2E1CFB2A9B216
:101F8000B59F79554852666453444A617C8B908A68
:101F9000808091A19F8E6D4F464E5A5A55625E5970
:101FA000615F5445311E1917191E2228436D8E9CFE
:101FB0009DA0ACB7B8AB9C91878189938F868A9797
:101FC000A8B2B3B2B2B1B2B1A89B9187807B77754A
:101FD000726D707C8586888A95A19F979596929060
:101FE000908D857872839BA39D9DABBFCBCECECBCE
:101FF000C9C9C1AF9E89706257483E3D414A4C46AF
:102000004E67879C998B8DA5AA92756768614A3A3D
:1020100040463D3F5366695D4D3F3D4422141612D4
:1020200018314C5E707A8DB9D5CBB7A99A979D9F20
:102030009D947F72798895948E939BA0A9B3AF9C51
:102040008B92A8A384757B7B7574777A746B7C9C68
:10205000AAA09BA5B8C2B49B939D9D928483919F97
:10206000A3A3ADBCBFBAB6BAB9A7978F82736557A1
:1020700050565C595B61646876858D8A7C737D8679
:10208000837867584D49555F5340392C1B285E8231
:102090006B48475C73806F504747465B8084898AF2
:1020A0009FBFC3B8B4AFABAFAFA9AAA7988D9198A3
:1020B000958C8B97A19C96999B9B988C8582766C2E
:1020C0006C6C675E595F6D7A81858992A0AEB2AC07
:1020D000A5A4A7A3A0A19D968F9397948E867877A9
:1020E00092AC9F7F799AB3A68C898077828E857512
:1020F000614C3C3E5461553E384B6B807F74675653
:102100004F585E54371D172332311E163668868AA3
:10211000827C8296A29B897460545A6D7E79717616
:102120008EABB9AFA3A0A4AFBCC5BEAAA2B2C7D1A3
:10213000CCBBACA7A7A39F927C6E727A7D7C787C87
:10214000888E898B959D9D9492A1AFABA5A4A8A9DB
:10215000A59A9194938B88827C7F8A8C84808EA7A9
:10216000A88F7F8E9C97866D5652574F4445453FAA
:102170003A455C6864595A6C7B7A736959545D645A
:10218000625B52494957666A6A6860606A717D900D
:10219000948E8B8C939B9A8C827D75707580878BC7
:1021A0008C919FAEB5B7B5B1B5BABBB8B3AAA4A46C
:1021B000A5A1A4A699857F858E908776717E8A8B4E
:1021C0008B91949594929594887D7C7C7D7A7271A4
:1021D0007D8E928C8586898F9086776C6A675F5733
:1021E00058635F4E434A63726A56526272756C63FB
:1021F0005D5F6973736E635A575F70746961636A78
:10220000778689837E7C848C867A787D7C75788ECF
:10221000A19E8E8998ABAB99867C7F898D8B8D91A1
:1022200099A4AEB8BCB4ABABADB1B3AFA296949524
:10223000989A9593949393948F89827D7E83827FDD
:102240007A74737C848B8C87858585878C8A837C64
:10225000797D7F7E7C7E7B7775797E7E79767471E1
:102260006D6C768280756B6D797E78706767717240
:10227000665F6063615D5B6367625D636D74777306
:102280006F70797C74696469768183848A8C8589AE
:1022900094948B8170646973766F63637F87888B96
:1022A000929697A4B3BCBFBBB3B1BAC4C4BDB4AE1D
:1022B000B0B7B7ACA19B99948B847B736C635F5C64
:1022C000565353575D676B6C7580888E91959995C1
:1022D0009092979A94837D888F8C837F7C787A857F
:1022E0008376767A7A78766C64686D6E67616162FF
:1022F00065646261656A6B706F6F7073777A7B7FFC
:102300007E7F828899A49C8682929F997F604D559A
:102310006669635C595E6C7880878F9599A5B2BCBD
:10232000C1BDBBC2CFD6D3CCC9CDD1CFC7BEB6AE4F
:10233000A8A0938576665A55524A43424A50505354
:1023400057616D767E82848A96A1A19F9E9FA1A2ED
:102350009C94959EA29B918D959D917E7777776EAB
:102360005A4C50585040313646484136323F4E4F15
:102370004C4D51525D6E7984908C79778A98917723
:10238000594A515C563F2A26374A524F4A505F6D90
:102390007886979EA5B2C6D9DEDBDADFEFE9DED418
:1023A000D0CEC6B9AAA0978D7F6D6563605B524E93
:1023B000505355575A6371797C84939FAAAFB0B735
:1023C000BEC2C4C8C9C3C0C9D4D6CFC9C4C0C1C1A4
:1023D000B8A0898386837C684F454E5246392E2E9D
:1023E00031313335394558696D677698A4927B72DF
:1023F00070746A4A2F32403D30262126363D3439EA
:1024000045535F6873808C9AACBFD4E4EDF0F7FE5F
:10241000FEF4E0D4CBBAA48B73635A503936373B01
:102420003E4046505F6E7A818B9DAEB2B1B7C2CC52
:10243000CFC9C1C4D0D0C9C3BFC1C5C0B7B4B4AD82
:10244000A095979C968774676B766C524545453F7F
:10245000342D39535C4C3D5584947B5C5867766DC4
:10246000492D334E56412D2527363F372C292E40F6
:102470004F4E4B5664768CA0AEB2BDD4E7EBE9E18B
:10248000DDDFDBC8B3A39887725E5147413D37302B
:102490002D333A474E525D7389989FA9D6EBF3EEE0
:1024A000ECF2FCFFF7EFEEF0E3D0D0DED2AB98A970
:1024B000B9B39879718090876B5254676C5A4439DC
:1024C0004D7C8D6C4D6297B099766B768A8B5E33BE
:1024D000314B5E512E1C2A474E2F1D282E446E6311
:1024E0003B3B484D64797E8794A6BECCD0D0CCD2FD
:1024F000DAD4C7B7A49B9B8F79665C5D5A4D403E8A
:10250000464D4D4B5162727B87949EAABDC8C9C986
:10251000CED7DAD1C9D0DBD6B8A4AFC6A28284A206
:10252000AE926E64798F8A6E5C64726F625A5A538F
:102530004E56686B5754697F83715F5E6B7260455E
:102540004458594A433E3E46483F353A434644483C
:102550004A4B5B7177778296A8B2B1B1B9C3C6C452
:10256000BBB3B4B3A99D92857E7C77706559575BE8
:10257000676E615B6D808A8B888FA6BBBDB0AABE7B
:10258000D5D3C5BDB8C4D8D3B29CAFC9C1977F90CD
:10259000AFB79D776E899B8B72696D72645F5F5A6E
:1025A0004B47566466635E5E6B7F82756C6F6E6CC4
:1025B00070695B5757565A5A4D434752574E4447D6
:1025C000556162616A7C8B94A1ACB6BFC1C8D0D0A2
:1025D000C8C1C5C9BEA69C9F9E96877A767B7B7034
:1025E00066636B7372737A7D80858A909290909AFD
:1025F000A0999095A09F9D98949AA29890999B9449
:10260000929091948B858F877879786E69635C5E00
:102610005E5855515654494F6562565F77786B6ADC
:1026200074777574696463605A554F4A494E544AC9
:10263000404D5F5E5D676E77889294A0B3BABDBE71
:10264000C2C8CECAC0B9BBC0B9ACA399959EA08A76
:102650007E888C817881867778847D81948B7F9445
:102660009C91959287939684858D8C929183829686
:102670009F8A7C89908182898080857477856D5D51
:10268000737A666267656C716C6B6F717C847F783E
:102690007F8B8D858186827C7D817A726C71685A90
:1026A0005C65615F696D656977797C8B9493A2B392
:1026B000A9A6B7BDBAB9B6B5B9B0A1A8B2A096A33C
:1026C0009C878993887E8383848B897F84857B83A1
:1026D00087726E807F6E6E7272777A736C747D769D
:1026E0006B6F7B7B6B68716F6B6B646374776F73FD
:1026F0006E66707369696867777461676F6C747F01
:102700007D8074627C9B8D797C8790887D746E6FF0
:102710007777757068767F6A6269676B6C737E7BAA
:102720007C8D958885989C91979B98A29C99ACA14B
:1027300095B1BBA89E9496A1989097908E95999EDE
:1027400093808C97918F8375858B7E818985786D39
:1027500072756E7981777370696D6E686C797B7054
:1027600068767F73738386807F83807F8B8885996B
:102770008F798D93787D857C8C908B93826F848EFE
:102780007D81857870797E71717D73707567666CF7
:102790006C808D808CA2928A9994858C8B888475AC
:1027A0008397796D887C6F8A8A757B75768D867341
:1027B0007E827980827E8A94979A8F8994928F996B
:1027C0009B969391948E82858A919687848F868238
:1027D00084746D6D6F848C7E7B777786838089822D
:1027E0007F7C737575758B8B768489727378747E34
:1027F00076686F67616D5D546D7765605D515258A5
:102800005C5F646B7680807B7B7E756D7983757889
:102810008D89818B867C828287948580876F797A87
:10282000768F978B938C7D919C929E9D8D9BA08B98
:1028300090A2A1A7AA9E999598A59D8D8D85899412
:102840008B7C7E8280879491807B8384858F866E4B
:1028500070786C727D73747E75757A747A7F7D7F03
:102860007E7A73616270696D797373746B74817B46
:102870007F806F6E746D738076717C747082837BE1
:102880008488838A88797F8682827E716D75808450
:102890007C7C8A847991947F919D898E8C9AA18E7B
:1028A000969A888D95929E9A909285767566667EA8
:1028B0007A7A8E8680857A78817B80827A7C797537
:1028C0007D7569716C667482827B7B8578677A829C
:1028D0006C70776B7E907D79817E8591847785851C
:1028E000777E89827C73707D7765788A7F8B978409
:1028F00083938B8489827E8483777575737C8782CA
:10290000818B8C868383888270777E7F91968B9073
:10291000958D8A858BA2947E8C938B95878E998CCE
:10292000879192877B777A81817C7E7B6D697C86BB
:10293000746E79767476747F857771766F7A8C820F
:102940007C878684959B8D8A8F8C8D8A7B7B7E6E1F
:102950006E7D7976797478786E717F7F7D7F8382E2
:102960007A7885908F7F6D747E79767E8A90878263
:10297000877A6C787C747C83797B8381817C6F74AB
:10298000807A788A8A757C8F8C818285888D8F8CFD
:1029900088828895988D7F7C87897B7B7577817904
:1029A0007076797B848788857A7A7F7A767C84854D
:1029B0007C7C84837A7E868480807F7A7D83898014
:1029C0006B6D7B7B7E868185918C8589867E808BF5
:1029D0008F88878C857981918C848E8E8288897589
:1029E000737A7C8989747476717470666D73747F80
:1029F0008277767A7C81818288887F7F84807D87D8
:102A000089878E90898E9591908D837B81897A6B51
:102A10007170707775727D767588908B91918C89C5
:102A20008B877C7B80838B8B8A918F8D918F878422
:102A30008B8D867E7F84878C8D857D818987848838
:102A40008A86807D7E7E7774756F6F8087828585AC
:102A5000858F8B7F8086858383807A7D84877D7A4E
:102A600083837F84817B7D7C7D827C7A8182817C73
:102A700078797970666765676D6A6769737D858740
:102A80008E97978F8D898584807D7B7673787C7B0C
:102A90008186817D858680807D79797A7C7A75785A
:102AA00076747A7A7B7E7D7C7E8186877F7E888540
:102AB00081837E7E84838487827C80807C81828502
:102AC0008C8C8C8D898A91918F8D898C918C82834D
:102AD00088837E7F808589868791908C8E8981808E
:102AE0007F818C9597908785837F807F7669595702
:102AF00064696E7774728191979B9B999690929D71
:102B0000A59D928A8484838485857F797A80848454
:102B1000868A857C78746C6C7070695C666C696898
:102B200068665F576495C1BEA39390918E87785B6A
:102B3000351B1B3658676F80909DB4D2EBEAC6A157
:102B400099A9B8BBAD9576646D8CA3A39A8F8D9728
:102B5000A0A4A69D8B8480786D64543D291B171F0B
:102B6000242428323C4D61737F76606A98C5CCB0CE
:102B700094949A8B756A50250F1F457B978796D141
:102B8000F7FBFBFBF6D59E858F8C6E5759696F63FB
:102B90006DA0CDE1EBF5FBEFD9CFCEBC765A3F2D42
:102BA000292F342E2D3B4A60778082807E88918049
:102BB000644A44688E8363585C636A6E6C55342F34
:102BC00056869994A2CFE6D1B8BBB89D785F57518D
:102BD0003F37557E888392B9E3F9FBFBF9E1BCAB43
:102BE000ACA28359433C39394C6875737386999DFF
:102BF00095856F635A4F4E482E192047788C807701
:102C00007C8A9A9D91734B394F6E74697092A49A25
:102C100093999989736361594D577896969DBADB5C
:102C2000EBE9E3D4B89A8E93896F5142474F5563CD
:102C30007681817F828177675C5B53494645454356
:102C4000445E8AA8A6968B8B90897D6A472723428B
:102C500069787386ADC3BDB0AAA18A6D5F5E584B1B
:102C60004A678FA1A3B1CCE7F4F0EADDBC9B8C8965
:102C7000856C534B4C53658099A3999092938775BB
:102C80006B5F4A3E475254505776A0B3AA9C9A971E
:102C9000887D72593E2E3154767E88ABC8BCACA27A
:102CA00099836D615F5D5D6F91ABB7C2D1E4F5F65D
:102CB000E9D3B3947F756E625852545C6A819EAAC0
:102CC000A0928E8B7C675A564E41414C63746F6262
:102CD000698CB5C5B6A39B8F7F74675039292F586F
:102CE00083909BB5C2B7A6969288735B4D4F5C6A82
:102CF000768DA8BDCBCFD3DDDAC1A18974645954D8
:102D0000575D5A575F73909F9A928E856F574C4FBD
:102D1000483B3A495855546992B7C0B3A99F8B7E36
:102D2000725E3D26326195A294A0BCBFAEA1988F81
:102D30007B605C747F747189B0C8C7BDBDC1BAA91E
:102D40009889755A4C5A6E736757556474838C8989
:102D50007D6C615A544A413F43484C54627EA5BD44
:102D6000BBB2AAA2907D796F4C3A445F8AA1959537
:102D7000B2C5BDAA9E9E94837F89938C7F8FB2BE7D
:102D8000B7B5B8BCBBB3ABA38E71626C77705C4E49
:102D9000494E57667682847E767167523E41464A36
:102DA0004F5A657390B3C1B9A89EA2A394816C5485
:102DB0004953708A8D8494B3C2B6A6A9ADA0918BF5
:102DC000857E74778FA6ACA7AAB7C6C7B6A28C704B
:102DD0005F5A54493A384658646F7A82827B746CE1
:102DE0005B453436434846464C5B6D788AA2ABA7B8
:102DF0009E969694877668595E737E7F848EA3BB79
:102E0000C2B8AFA59B928E8E897F7F8C9EB1BDC1CB
:102E1000C2BFB3A7957E6A5E5D5F60666D686562DE
:102E20006874766D666563564341494942455C76F0
:102E3000838C9199A2A6A09B958C86857F7B7D7BB8
:102E400081919BA3A9A6AAB2B3AFA89B999F98987A
:102E50009F9CA1B3BBB4A6989392877974706C6D54
:102E600070726C5F524E555F6C70665D5856564E70
:102E700042393D465469787C81898F8E8884898C5B
:102E800087817C7C838481858B909087899DAAA88B
:102E9000A6A8AAABAAACB0AA9F9B9BA09F99928818
:102EA000807A78767067687075726B6E706C6D7210
:102EB0006C5D514E565551534D485568797B75722E
:102EC0007A80858785827D7A858B87857F7B7F84E5
:102ED0008387959EA0A3A4A5AFB2A8A19F9A9A9A12
:102EE00096989993918E837C7A7A797063677071E2
:102EF000717677736B656A6B655E544E50525255AE
:102F000057595D6A7F888581858C92948E8C887FE5
:102F1000808E90888C939395999FACB2A1A7ABAC0F
:102F2000AAA4A09C928D929899908889857F7D7E95
:102F30007A7569646B70727272757C7B726B5F54A8
:102F40005A61606364616167707C807C7E878B8F6F
:102F50008C8A8D8B7F828D8F8A8284939C969297A8
:102F60009EA09F9C989B9F9E9B99989089898F90EB
:102F70008C817C81847F756B6973787675777473C7
:102F8000787B786C625B5A5B5E6667656D75757A97
:102F90007F7D8391948D8C8E8781818283888B90B5
:102FA0009293999D9895959295948C8C91959C9DD2
:102FB000948E8C8A8B877E7A7B75767C7E808078F7
:102FC000727880817D7D7F7B75726C605F636A6FD4
:102FD0006D676B72777E807C7672757C7F8384826E
:102FE000828485877F767A81838C999EA09E9B9E22
:102FF0009E9290948E8C8F929796908B8D87807BEB
:103000007A7B80828084868182857F7D7D7A7B79D0
:10301000787C7D746D70706D6E767E828482808126
:10302000838382797376797D80868784827D7E84AE
:103030008885828A959897928B8886838082827C05
:103040007C83898A827D7F81808586827C787C8072
:10305000817F80807D7B7C7D7F7C797A807F7A799F
:103060007B7E7D7C7D7E79788087827976737072B5
:10307000767A7C797C8387867E7B7E7C7A7A78768A
:10308000787676797D807F82858686817E7E7D805A
:1030900082807E81817F83878688888485827E7F07
:1030A0007E7E7F7F7E81817E828A8A8684838686F9
:1030B000807C7F80818484848279757B7F807C742E
:1030C0007275797C7E7E7B77797D808183807F823B
:1030D000828082848283848B908F8C929391909053
:1030E0008E8B898B8B878383868A8F8E8D8986854D
:1030F0008689888684868A8B8A8989848185868464
:10310000827B78797B7774736F6D7074777777755E
:10311000777B76757474767B7C7D7F7F84878889E6
:103120008584878B90908B8A8F8E8A898B86868800
:10313000878D8F8A85837E7E7F7D7C7E8184878458
:103140007F80827F7F7C797776787A77716E7071F5
:10315000737374727170716F6B696C6C6D6F6F6D7E
:103160006C6D72777978777B7D80828584838587A3
:10317000888C8C8886888D908F8C898789898889AE
:1031800087878A9191908F8C86878B8B87827E83AD
:10319000858182838381807D7F7C767777797C7956
:1031A000797D7E7C7B7F7E7C7B787B818381828046
:1031B00080868786878B898887868A8B8A8D8D8D86
:1031C0008E8D8A8D918E898A8B8D8F8F9094928F20
:1031D0009092918D868383848383817E7D81837F9A
:1031E0007D7B7B7877787974727274787775737277
:1031F0007071737476777777797F807C7A7B7F8143
:10320000807F7E7D7C818585858585898A8A8D8A7A
:10321000898E908F8C8C8E8D8D8B89878885848408
:1032200084848486898884838483817E7D7E7F7F75
:10323000807D787877757677787B79767879777806
:1032400079787978777A7B797B7A7B7978787A78EC
:103250007C7F7F7D7B7C7E7F7D808181817F83867B
:103260008382868584848182848586878685858518
:10327000868582817F7E8081807F7D7C7D7E7E7F52
:103280007F7B7D818280807D7A7A797B7C7B7C7C70
:103290008083828081827F7C80848484858685850A
:1032A0008B8D8C888B8E8B88888B8D8B8B8B8C8C6D
:1032B0008A8B8A8987888789898786878686868395
:1032C00083837F7D7F8080807F7F808284828281F4
:1032D0007F8081807E7F8181828485827F818283DD
:1032E0008383848589898886868686868585858385
:1032F00082828284848282807F7F838483808082B2
:103300008080807F808486817E7E7E7F7F808282B7
:1033100083858785838283817F81807F7E7B7C7BA1
:103320007879797A797A7A7B7C797C7E7C78797AFB
:103330007A7D7B777677767477777376787A7B7910
:1033400077767676797A7A7E7F7C7A797B7D8081D2
:1033500084838083838385858583807F8389888731
:1033600086858688898986888984848788878685F2
:103370008585838484818186868381808285868811
:103380008785888A888A8A878382807E7F7F8184F6
:1033900084828283828280807E7B7D7E7F7F807E2E
:1033A0007F8183818181808281817E7D7F7F80801A
:1033B000807F7F807E7E808183848383817D7D8109
:1033C0008282807F7F84858383838384827F8180E0
:1033D00080807F7E7C7C7C7C7D7D7E7E7D7E7E7E13
:1033E0007F7F8283807E81848483848684848584B5
:1033F000848484858482817D7B7C7D7D7B7B7B7BDB
:103400007B77777777737274777778797876787750
:103410007877777A7A797778787B7F7C7C7A7A7913
:10342000797D7F8080807F7C7F838583848381809A
:103430007F7E7D7E8082818387878485898886835D
:103440008385858685858585838280808082828646
:10345000868484858484858586878A89898886850B
:103460008483858383828080808082827F8083843E
:103470008588898A898A89888686868586888986D4
:1034800082828384848282838484858583817F7E13
:103490007F807F7F8180808182817E7E818281802A
:1034A00080808081838384858586868583828385E9
:1034B00085817F7D7E808384858586858586827FE4
:1034C000828684838280818180807E7E7E7F807EF2
:1034D0007D7B7A797A79797A7C7B7978797979794F
:1034E000797A7A7A79787A7C7B7C7C7B7E7E7D7F28
:1034F0007F7F81807E7E7F7E8080808383848584C1
:10350000848381848383838281807F7F82837F7EA3
:103510007F828181807E7E7D7E7E7F7F7E7E7F81B9
:10352000818285848181828488868686848285865C
:103530008787858282828486878787888B8A888826
:1035400087848888888A888687888583848483831B
:103550008483838281807E7E7F7F7F80807E7C7E6D
:103560007E7E7F81807F7F7C7D7C7C7C7E7D7F807A
:103570007F7F7F7E7E7D7F80828383828181838146
:10358000807E80817F7E8283828281808080808035
:1035900080838688858386868482828283868381EF
:1035A0008283838180808282818383838181818001
:1035B0007F7E7E7D7C7B7A78797A797C7D7D7B7C51
:1035C0007B7B7978777A7B7B7B7C7F817F7E7F8139
:1035D000828381818382828584817E7F7F818082D4
:1035E00083828282818083828282828181807F81C4
:1035F00081807E7E7D7F80807E7C7E7F83838181D3
:10360000828282828382817F807E8082807F7E80B0
:1036100082838385888A89888986837F838383835D
:103620008285868687878686878787868383838148
:1036300082838182838384827F807F7F8383818171
:10364000807F818183848380808082838483807E65
:103650007E7D7E807E7F808080808282848786845B
:1036600081817F7E7C7D7D7C7A7D7E7F7F7E7F7D7C
:103670007E7F7D7C7C7D7B7A7E7E7D7F7F7E7E7F74
:103680007E7F7F7C7C7E7E7D7D7E7D7F7F807E7D5C
:103690007E7E7B7B7C797B7A77797A797C7C7B7A7E
:1036A0007B7A7A7B7E7E7D7C797B7D7F7E7E7D7F53
:1036B0007E7F807F7F807F81817A7B84848283820A
:1036C0008386868786848486868687878482807FB1
:1036D0007F80808183817E807E80827E7D83817EEB
:1036E00081838186867F8088878586858486868695
:1036F0008786848587858688878687878789888562
:1037000084838084827F838481838581818180809A
:10371000807E7E7C7D807D7B7D7C7B7E807F7F80CC
:10372000807C7B7C7A7D7D7C7A7D7E7F7F7C7B7DCF
:103730008082808182828586868686878888888541
:10374000868785838483838687898885838889861D
:103750008787848383838384827F80827E7E817E49
:103760007F7D7A7A7E7D7B7D7C7C7D7A797C7B7D9A
:103770007C7C7B7C7C7E807E7D7D7E7B7B7A7B7D82
:103780007D7E80828283817D7D81817F7F81828039
:1037900080807F808181828282858583818282820E
:1037A000817D7D7F7E7B7C7D7D7E807F808282802F
:1037B0008282837E7B7E8080807E7C7C7D7D7D7F1F
:1037C0007F80807F818282818283838485858383D9
:1037D00085868686878787878A898A8C8B8A8D8B60
:1037E000878686878988878888888988858586826C
:1037F000808185848383858581817F8080808181AC
:10380000817F7E7D7F7E7B7F7F7E7E7E7D7F7F80D2
:103810008184838184848588868586868483838267
:103820008185878482828584817D797C7F7E7C7C92
:103830007D7E7F7C7B7E7E7F84848483827F7E7D91
:103840007D7E7C7A7C7C7A7A7B7977797B7B7B7CCA
:103850007E7D7A7B7A797676797A77777A7C7D7FC6
:103860007F7F807E7D7F7F80838486848281848841
:10387000888787868381808282828280808181811D
:10388000838384868582807F7F7E7E7E7F80808426
:10389000858180828181817D7E81817F8282838614
:1038A000858282828283817F7F7F818483838483F8
:1038B00085858488847B7D868481838484838382D8
:1038C0007F808483818384848484848383818080D3
:1038D0007F7E7C7D7B7D7F7E7E7D807F7E7E7F7F09
:1038E0007D7E7D7B7D7F80808281817F80828688D6
:1038F0008989898B8B88868585878684848384885B
:10390000878483828180807E7F8285848181828199
:1039100083817D7D7B7A7B79797B7A7B7A7E7E7FE2
:103920007F83838181807E7E7C7C7C7B7E7E7C7BB2
:10393000787878787A7D7F7E7F80807D7E7E8082B9
:103940008281807F7F81808081807D80818383826E
:1039500082868789868381828180807F7C7E7F804A
:10396000807F7F83837F7D7E7F7F7E82817F7E805D
:1039700082807E8184828484848485848484838319
:1039800085888784848587878989898887888888C6
:1039900088888B8D8C8B88878A8A8888888686849D
:1039A00084838383838280807F7E80808282807E06
:1039B0007E80807F80807F7E7F7F7D7A7A797A7932
:1039C0007A7B7C7D7D7A7B7A7A7C7E7F7C7D7F7D35
:1039D0007B7A7C7E7F808081818383818081807EF1
:1039E0007F7F7D7E7E7F7E7C7C7F818383828180E2
:1039F00080807F818081817F7E7F807E7F7F8082CB
:103A000082817E7B7B7B7E807F7D7B7C7C7D7D7AE3
:103A10007A7C7D7D7E7E7C7A78797D7E7E7F7D7DE1
:103A20007D7F7E7F807F7F81858784828586858676
:103A3000868688888482828283838280807E7E7F5D
:103A400081828483807F7F8084868483838384864D
:103A5000888988868582818283827F7F8080818237
:103A600081808183838383838789888786888A8905
:103A70008B8B8888898987848587898988868686CB
:103A800086888A8987878585878786827F7E7E80EC
:103A90008280808382818381807F7F808282817D1A
:103AA0008081807F807F7E7F7D80828387858589FE
:103AB000847C8189878688878486878685838383BB
:103AC00083828080807F80828283828183838383DC
:103AD000828284858684807F7D7E7E7F8283807FD4
:103AE000808082807F80807F7E7F7B7B7B797979FD
:103AF0007A797975777A7C7F7C7C7C7A7A7E7F7E16
:103B00007E7D7F7F7E7D7C7B7C7C7C80817E7F82D6
:103B100080808383828281807F7E7C7D7E7B7C7EB1
:103B20007D7D7D7E7E807D7B7E807E7B7D7E7F7FBA
:103B30008083828282828281808385828283828264
:103B4000818183848686878785858485898A89861D
:103B50008282838282848484858686868383858725
:103B60008787878788888888868182848080817F0C
:103B70007D7D7D7F807F7F807E7E7D7A7B7F807E66
:103B80007E7D7F7E7F7E7C7D7F7E8083858689882B
:103B900085848482838686868582828181818381F1
:103BA000818486878685818183838585817F7E7CEC
:103BB0007C7D7B7B7C7E7F7F7E7E7E7D7F807F7F2A
:103BC00080807F7E7E7B7D7D77757A7A7A7B7C7C38
:103BD0007D7D7B797A7A797877777777767477785D
:103BE00076767779797B7E7E7F7E7B7B7D7F7F811A
:103BF0008080838181808080807E828483848586AA
:103C000086868687898A8685868685858586868650
:103C1000848586827F808082838584848788888863
:103C20008785858887868787878585878A8B8B8C1C
:103C30008C8B888888888888878686878A8C8A89FA
:103C4000898889898786868684838181828180812B
:103C500082807E7F7C7D7B78797A78797A7B7B7CA9
:103C60007A7879787779797C7B7D7D7E7E7D7E7FA1
:103C7000807E7C7E7E7C7C80818384807F81838447
:103C8000878481817D787B7E7F7F7E7D7E7E7D7E49
:103C90007E7D80837F7E7E7D7B7A7B7C7A7C7D7F50
:103CA0007F7E7F807F7E7D7B7B7C7A797A787A7D50
:103CB0007A797D7F7E7A797C7D7E7E7D7E7E7D7F3A
:103CC0007F7F8080838384818283817F81818285DD
:103CD00085838381818282817E80858482838583BE
:103CE000828080818484817C7B7F817F7F7D7C7CDE
:103CF0007E80807F7E828384868485888B89868689
:103D0000888887878988868586898A8B8B88878536
:103D1000828484838184868483838383868789885D
:103D2000838282828585878583808183848483835F
:103D3000858482818182807F7F8387868583838358
:103D40008487888785828282848686868484858625
:103D50008482868787868788898687888885817F09
:103D60007E7F7F7E7F8082827D7B7C7D7E7E7C7D70
:103D70007A787A7A7B7B7E7C797D7C7B7B797A7B97
:103D80007C7B7A78787675747678797D7D7B7877A8
:103D9000787778797676787B7A7B7B7C797C7C7D8A
:103DA0007F7F8083858282838386878787868483DB
:103DB00085838484838384858787898B8A8A88879F
:103DC0008687868686848488868584858384888998
:103DD0008787878787878988868688898B8A86866A
:103DE0008786848688888887898C8988898A888755
:103DF0008684848687888784848381858785828377
:103E00008283858483838383817E7E7D7E7E7B7DAA
:103E10007C7C7C7E7E7D7D7B7D7E7D7E7B7F8182CA
:103E2000838384858585848385858381818282825D
:103E30008383848788878786838181827F7F7F8051
:103E4000808082817E7D7E7D797A7B7A7C7D7D7E9D
:103E500081807D7E7D7D7B7B7B7A7C7C7B7C7C7A9C
:103E600078757573717476747577777677787875F9
:103E700074767474747774737272747778797878EE
:103E800077787A7E7C787A7C7D7F7E7E7F7B787780
:103E900078797A7B7A7C7D7F81807F7F7E7F7F7D52
:103EA0007C7C7D7F7C7C7D7F7C7C7F808080828130
:103EB00083848383858686888988868688898C8B97
:103EC0008988898B88868582817F7E7D80828384B4
:103ED00086878784868887878787898A898887866F
:103EE00086837F7F818283838483838381818182B0
:103EF000817F7F7E7D7B7C7D7E7F80807F808082D6
:103F0000828283858585898988888989898A898744
:103F10008788898784848280808181828481817F6F
:103F20007E7E7E7D7E7E7C7C7A7C7D7979797778D9
:103F3000797A7B7B77797D7C7C7C7A7876767776EC
:103F4000737474757676787878777576787778770D
:103F5000797B7E7F7D7F818284858788888887873B
:103F6000878786868685848483817E7B7D7E7D7F30
:103F70007E7E7C7A7C7B7C7F817F7F828180828257
:103F800083848485848484868988858688888A8CCD
:103F90008D8E8E8E8C8B8B8B8A8A898A8A8986837A
:103FA0008383838683818181807F7F80807F7E7D04
:103FB0007D7A7D81808080828383817F80858787F1
:103FC0008381807F7E7D7F7E7F80817E7B7E7F7F01
:103FD00081848584838383838282828083848482B4
:103FE0008280808282868887878686868887868484
:103FF0008587848687858486868181828588868375
:104000008281807F81807B7A7D7E8080807F7F7EC1
:104010007D7D7B7A7D7F7F80807F7E807C7C7B7BCB
:104020007A797B7D7D7E7B78787878797C7D7D7FE1
:104030007E7D8081808080807E7F7E808486838379
:10404000838282838384858586878889837F7D7E3A
:104050007E7D807F81848180808283838281838151
:10406000807E7F8083838485848487888787858218
:1040700082848788878483838383848686848281FD
:1040800083838484838283878A88858585848484E6
:1040900082848482868788878888868486868687C5
:1040A00086828283827E8083848687848182827FE7
:1040B0007F838585848484828283848487898684BF
:1040C00083848585848281838686858584838484B0
:1040D000838282818182828181807F7F7E7F7E7CDC
:1040E0007D7E7F7D7E7E7D7C7A7C7B7C7D7D7C7D04
:1040F0007F7F817F7F7E7E7D7C7A7A787679767508
:10410000777874747777787778767577767274774E
:1041100078797D7E7D7E7E817F807F7D78797A7ED5
:104120007F7E8283807F7E7E7C7E7E7D7B7B7C7CAF
:104130007B7C7C7B7D7D7E7D808181838583817F8F
:104140007F7E7C7C7F808285868686838385888946
:104150008887888986828384858686868786838405
:104160008685818283848485888685868886858500
:104170008584848486878787898A8A8887858685D7
:1041800082808082817F7F7F7E7F7F8283807F7F2E
:104190007E807F7E7C7D7F7F807E7D7C7F80808136
:1041A000868785888A898686858383868888888AA3
:1041B0008A87868685818083807F7E807E7C7D7AEB
:1041C000787774717071737577777B7D7B7878778A
:1041D000787778777B7C7B7A797D7F7E818282801D
:1041E0007F7D7E7E7F7D7D7E7F80808181828584D4
:1041F0008282848385878786878887868581828275
:1042000084848282817F8082818384818286868683
:10421000888786878887848083848484818080825D
:1042200082817E7E7D7F7E7C7D7D7E808483838394
:10423000838183807E7E7F8183838281838588885A
:104240008888868584838283848485858584828228
:1042500085878584838585838483807E7E80818035
:10426000807F7F7E7B7B7A797B7C7A7879797C7E94
:104270007F818182817F8082817F7F7E7E7F7F8040
:1042800082838484868788898884848687878785D3
:104290008586838386828385837F7E7C7A7B7B7C15
:1042A000797A7A7D80807C7A797C7F7C7D7D7C7B4D
:1042B0007D7E7C7C7F7E7D7D7E807F7C7D7D7E7F24
:1042C0007D7C7D7E7D7E7D7B7C7A7C7C7D7D7C7E25
:1042D0008080808183817E7E7F7E7E7F807F7F81E4
:1042E000807F7E7D7D7F808081807E8080808183D5
:1042F0008282838789898889888583848384858469
:10430000858687868685817E7F8384838184868473
:104310008482818383878788888688878787898C3A
:104320008C8C8C8B8C8F8D8D8D89868587878687ED
:104330008686888785858584838184858380807E41
:104340007E7F81807E7F7F7E808080807E7F7F7E7B
:104350007E7D8081807F8080807F7F80838585884F
:104360008A8987888C8C8A878380808080808085FA
:10437000817F7F7E7E7F7E8080807F7D7D7D7C7D56
:104380007C77757577787A7F8181807E7E7E7F7E6F
:1043900081807F7E7D7E7F7D7B7C7D7C7A7C7C7B4B
:1043A0007C7C7A7C7E7C7C7B7D80807E7A7C7F803E
:1043B0007E7C797978797C7F7F807E7C7A7A7A7C42
:1043C0007C7A797C7D7C7D7D7C7E7D7B7977797A3A
:1043D0007B7B7A7C7E7C7C7C7A7B7B797B7D7E8020
:1043E000818384848182848484848484858586878F
:1043F0008685858785868686868787868383858961
:104400008B8B8889888A8B8B8A8C8B8A89898A8B0B
:104410008B8A8D8E8C8A8583838585838484878728
:10442000858383838280807D7C7B7B7B79787676B5
:10443000787B7D7B7D7B797A7C7E7D7E7E7D7F81B6
:10444000818183838385878988868888888A868313
:10445000848789898685848383838383828181801D
:10446000807F7E7F7F7F7E7E7D7D7D7F807F7E7D66
:10447000797B7C7A797979797A7B777576777574B7
:10448000767877787A7D7F807E7F7F7E7E7B7C7E6C
:104490007D7E81828182838381818384837E808605
:1044A000888482807E7B7B7E7E7D7D7F8181808013
:1044B0008081807E7F7F7E7B7C7C7D7E7F81848807
:1044C000868587888786848483838282858585859F
:1044D000878782818382827F8082828484838687A9
:1044E000888A8B89888A8C8C8C8985838486868649
:1044F000868482848584828484828380808283838C
:10450000838383858382807F7E7D7E7E7D80807FA6
:104510007F818382838283838385838382817F8279
:10452000838485848484838181808083838482835F
:1045300085807D7F7F7B7777787576747377797BDD
:104540007B7A7A7B7F7C7B7D7A7B7D7D7D7F7D7DA9
:104550007C7B7B7A777578797A7D7E7B7B7B7C7BB5
:1045600079787A7A7878797B7C7E807F7F81848283
:10457000818280807F8082838481808283807F7D2E
:104580007E7E7D7D818280807F7F80848685848021
:104590007F7F7E7D7A7B7F7F7E7F81838384868819
:1045A000898686898D8C8B8B8C909392918E8C8E44
:1045B0008E8B8A8B8D8F8D8A8D8D8B8C8C8C8E8E35
:1045C0008B878484848383848281818283817F7FBB
:1045D0007D7D7F7F7F7F7C7C7C7D7F7D7A79777519
:1045E000767A7C7E7F7F7B797B7C7E7E80828383F4
:1045F0008183848381838381818181848687888884
:1046000088888586888785828283848481807F826A
:1046100081807F7F7E7D7B7B7D7F7E7F7B7B7D80BE
:1046200081807F7E7F7D7D7C7F81807D7A7A7B7CAF
:104630007A787978797D7D7E7C7C7B797A79797DD1
:104640007F7D7B7A7D7E7E7D7C8183807F7E7D7D8C
:104650007E7E7F7E81838483838382817F80807F4F
:104660007C797C7D7E7D80807E7B7B7C7D7F818074
:10467000807E7D7C7C808182818083858485878823
:104680008A8783858A8B8C8C8B8988837F807F7FC8
:104690008485878A898989868789848089868686B0
:1046A00086898B8A8583858485868784868A8886A1
:1046B0008583808280808281817E7E7F7F7E7C7DFB
:1046C0007D7E7E7D7F7F7E7F7F7D7C7C7B7B7B7C18
:1046D0007D7E7E8185838284848487878B8985859E
:1046E00085878886858485858380807F7D7B7979B1
:1046F0007C7A797A7A7A7B7D7E7B7A7B7B7A797910
:104700007B7C7C7D7E807E7D828585837F7F8080B3
:104710007E7C7E7D7C7C7B7A7C7D7B7B7C7D7E7CD5
:104720007C7B797B7E7F7E7E7D7F7E7E7F7E7E81B1
:10473000807D7D7F7F7E7D7D7E7C7F807F7D7E7E98
:104740007F7F7F807E81848380828483808081825A
:104750007F81818283848585888888888788888707
:10476000868481838689898886868687898C8988DC
:10477000878A8C8C89888A8A8A8C8B8888878687A6
:104780008785888C8B8989888A8B898788878583A8
:1047900081807F7C7879797B7D7F80817F7F7E7F40
:1047A0007F7D7D7F7E7D7E7F7F7D7C7D7F7F7E8325
:1047B0008485828082807F7E81868989898C8C8EA7
:1047C0008C8A898683828080818180807F7E7D7AC9
:1047D00079797A7A7B7A7879797C7B7D807F7E7D26
:1047E0007A7A7B7C7E7F84858482858682807F7FC7
:1047F00080807F7F7D7B7D7F7E7E7F7C7A797778EE
:104800007C7D7C7B7776797B7D7E7E7D7C7A7A7AF7
:104810007C7B7A7B7C7C7E7E8082818182828180AF
:104820007F7E7F807E80827F7D7E7D828483848286
:104830008185898987878584858182838486858629
:10484000888A8C8D8E87858582807E7F8083868313
:1048500085878587888686878989898582838584F7
:1048600084828286888687868484868484858482FE
:104870008281817F7D7D7E7F828181807E7B7D7D47
:104880007F80807F7F807F7E7F7F7F807E80807C37
:104890007E807F86867A7F908F8A8E8D8E8A8887AB
:1048A00085858682807F7E808182817F7F7E7B7707
:1048B0007777787B7C7C7C7D7C7A78777877787961
:1048C0007D7D7C7B7B7A7B7E7E7D7B7B7C7D7B792B
:1048D00077757779797C7A77787B7C7C8082828324
:1048E000878A89868382818487868685848588896C
:1048F0008785858080817F7B7A7A7B7C7C797777DE
:1049000074767877797A7A7676787A7B7A7B7B7D1B
:104910007D808483828485868686888B8C88868742
:104920008A89898B8B8B8C8C898A8C8A8B8F8E8DD4
:104930008C8E8F908E8E8C8C8C8D8C8B89898787BA
:1049400087898B8E8E8A87888885848484858886EB
:10495000858789878482807E81817F7F7F81808136
:1049600082828383827E7D7C7C7D7B7C7E7E818255
:1049700083848588878786878684848485838485E5
:1049800082818183848380807F7E7E817F7D7E7F24
:104990007E7F7F7E7F7D7E7F7F7D7A7B7A7A78794E
:1049A0007B7E80828382807D797879797A79777746
:1049B000777777767778757577787B7B7A79797C76
:1049C0007D7D7E7C7B7D7A7A7D7C7B7B7A7D7E7C27
:1049D0007C7C7B7D7C7B7C7C7B7E7B78797C7E7E1B
:1049E0007F7D7E7E7D7F81838383828280807F7FC7
:1049F0008284838181828383848482818489878283
:104A0000818183837F7F8282828587858485888771
:104A10008484848484828083878987858184868551
:104A2000888B89858483888A88878585858587861C
:104A30008585858787848586888889868481808224
:104A40008382828081807E7E7C7C7E808081828366
:104A5000838383848585888A8A8988858685817F02
:104A60007D7A7B7E7F7F807E7C7F7E7C7F7E7B7A73
:104A70007A78787879797B7C7A7C7D7F7C7D7F8081
:104A80007F7F8082807D7B797B7E7E7D7D7D7F8048
:104A90007F797B7F8080818182858482807E7E7C1D
:104AA0007C7B7B7A7B7C7D7F81807C797C80828132
:104AB000807F7E7E7B7B7B7A7D807D7D7F807E7D1F
:104AC0007B797A7A7C8185858383828181818184E7
:104AD000858588898583838583838382807E7D7DA8
:104AE0007A7B7D7D80807E808082838482818484C5
:104AF00082838384888887888A8986868686868654
:104B0000838386898A8B8B8A8C8D88868483838431
:104B1000817E80858685878C8985888C7E807F7D57
:104B2000818683858D8884898A868687868180832D
:104B3000827D80847D7D817E7B7C7B7977747274BD
:104B40007774717072707176777477797776787818
:104B500074747876777B7E7C7B7B7B7C7D7D7C7EB2
:104B6000818180807E7E807F7F7E80838586848633
:104B700086898B8885827F818380818686878886E7
:104B800085878687858889837B7B7C7D8084858BF0
:104B9000898689868384837F7E7B7A7E7C7D808400
:104BA00085878A8785898C8A89898684807E7D7DB0
:104BB0007F8286878B8E8F8F8E8783827D7D7D7DA2
:104BC0007E80858786878A8B868586878788898683
:104BD00084837E7E81817F7E7E7E7C797B7F7E82E8
:104BE000868281818080847E7A7D7E7F8382807EC2
:104BF00078767A82888B81746E66606065696E787B
:104C000081878E96928F90857A797163656C7380B7
:104C10008D96A2A39E99948B7F7976726D6A615E60
:104C200062666F797D7F7E7B746D68636061666E9E
:104C300075797B8185898E909196938E8D8F8D8CE1
:104C40008E909394969BA1A39D9A96918B8581813A
:104C50007D7C7C7F8486898F9395978D81858D8AD5
:104C60007765584E464145546E818B959F9F978C32
:104C70007A6A6254423C414B5B738CA4B9C2C1BE98
:104C8000B09B87776864696E76818B968D7D8796F9
:104C900095969587827B6A605F5E626D828B8F8E50
:104CA0008C8C8987898B8C91989CA1A8AFB4B3AC6C
:104CB000AFB4B2ABA19B9D9A918B8A8D928D858367
:104CC00086837C76777C7972716E6D76858E887B33
:104CD0006C5F503D2F2C354556688199A6AAA68F4A
:104CE000735C452C20273E5C809FB6CBD4CCBCA9FE
:104CF00094857C7371706C69696C73808B969FA2CC
:104D0000957F68503E383B4052708896A2A8A39980
:104D10008F857C77717787929CAAB2B7B9B1B0B60C
:104D2000B6ABA09A9991857B7B8183817E7D8080C3
:104D3000808081817F838C9598876A4D311C151402
:104D400021426B88A4BDC8C6B3916A4122120E13DA
:104D500024456D90AECDE0DDCEBBA07D5E463C3FF0
:104D60004854657B919CA0A09F9A92816C5B4E43B6
:104D70003F4652677A8DA0ACACA69E8F847E7D7F25
:104D8000879AABBAC9D4D5CEC4C0C1C2BAACA2A7A7
:104D9000ADA49797A0A4A59F989895896E696C7308
:104DA000706B7D9EB3AE98826B4D2707010E1D2F51
:104DB0005483A8BCC3BDAD9573441D0D0C0F1F409B
:104DC0006D9FC9E0E2D7C7AF906E5B575654535AF8
:104DD000646A7382919EA7ACABA18F735946372D3D
:104DE0003145607F9EB2BBB7AB9889817B7880925A
:104DF000A2ACB7BEBEB5AEB1BBBCB0A8AAA79884E2
:104E0000756E7177777D878D8C8B8A7F70625A592A
:104E10005A5755688594918A7F6C553814171E2D02
:104E20004A7096B4C2BFAF967552321D181D2A45FE
:104E3000678DAFC4CAC9C6BCAB9886796E58443E6C
:104E40003D404C5D738FA8B6BBB8AC977C625043B5
:104E50003C43546E889EAFBBC0BFB8AEA39C98992C
:104E60009CA0B0BDC1BEBCC5D1CBB7AEAFA794802E
:104E700078787E807D85969B8F857F787870615865
:104E80005F6C6963738FACBCA58A959D7E532810B7
:104E900013131121487FB0C8D9E3D9BF6847312027
:104EA0001C273E6389A3B7C9D3D6D0C4C1BCA48490
:104EB0006A50331D15182A46698EADC0CCCBBBA4F1
:104EC0008B6F503A2F2D39506D869CB0BDC1C2BD3D
:104ED000B4AFA89F9C9893939EAEB2ACAAB2AD9982
:104EE000877A726E69686D7981818083857F776D3D
:104EF000605C53453D414754647A97ABAEADA69391
:104F00007B5F3F251C1A161B2E4E6D839BB2BBBDCB
:104F1000B6A38C796F675D5E6B7F8F9BA5A8A59B01
:104F200095928B85848789878181807F7A736D6C68
:104F30006D6D6A6C727D878E97A3AAAAA5A19D95B7
:104F40008A837F7D7A7C8898A7B5C0C9CED1D0C42A
:104F5000B3A79A8A725E565454576068757D7C7AFE
:104F6000797570696061696C6A67666866666D7795
:104F70007D7D746D6B61544B4A4E565F636A727CE3
:104F8000858785888C9191908B87817976747881DB
:104F90008D99A3A8A7A39C918885888C989B9B9C9E
:104FA0009D9A948F8D89888D908D8784807E787569
:104FB000787A7D817F7A7A7773717073797D7F7D5E
:104FC0007F83827E7A78766F6967686A6B6F757E99
:104FD0008687868889888684827F80807C767778B9
:104FE0007A7C8287878683807B71675E5A5B59599A
:104FF0005A5C5E60656B737A828B919796928C8314
:105000007C79787B7F88929A9D9E9E9FA4A4A0A085
:10501000A0A0A09F9D9FA2A7ACB1B6B9B3ADA2932B
:10502000877D756E6E73767B8385868989898A8A8A
:105030008A8987827C777574787C7F7F7F8183847F
:10504000807E7E7F7F7E8084898B8A898A89827C2C
:105050007A7574716D6B6B6B6B6D7376797A78772B
:1050600075736F6B6B6C6D707681888B9096989A68
:105070009B9B9897948F8B88868889898D9196972A
:10508000908C8A827C78726F6E6D6D6D6C717575A7
:10509000787A7A7A7A777574737174777E7E7F8185
:1050A00084858585858383848182878A898A8E8F9A
:1050B000908E8B857F79736F6D6F767F89919597D1
:1050C00095948F88827C77736F6D696565686C7065
:1050D00075797B7A7A797871696564666B71777CAA
:1050E0007F7F808182817E7D7C7E7E807D7B7C7DDA
:1050F00080878B8B8B8A8A898483827F8183888C4B
:105100008D8F908F8E8C898987888A8A8C8C8989EB
:105110008A8B8E8D8F8F8C8B8C8A898B8485898CE2
:1051200092969A9B99938D8A8684828080838486C6
:105130008B90919595938E8B87817E7B7A7A797906
:105140007776797B7C7E7F7E7F7F7B7673706C6BDE
:105150006C6F72787A7C7D7E7D7C7A777776787BCF
:105160007C7B7B7A7B7C7B7C7B7C7D7C7C7C7C7988
:10517000797C818483848887868584837F7F7F8010
:1051800081838180807F7D7F81828282848481810E
:105190007F7F818484888B8987878787827D7D7FD5
:1051A000838788898B8C8F919291908D8885827F5F
:1051B0007E7D7D8084878888888583827E7B7C79DC
:1051C0007978797C7A78797C7E7E7F7E7C7E7B782C
:1051D000767674747274797C7E7F8182817E7A792E
:1051E000787877787B7D80828184828283838282D3
:1051F0008282828283888C8F918F8D8C8B87878629
:105200008688898B8E8E8C8C8C8B8887868486830F
:105210008280828081878B8D8D8F8F8E8A8684801D
:105220007E7E7B7A7A7B7C7F7F8184827E7C7B7AA8
:105230007977757676777A7C7E807F7F82828484A8
:1052400082817F7B7C7C7E7E7C7A7B7A79787878A1
:105250007B79797B7A797B7B7976767878767C7FB7
:1052600082837A75848B807B807F85877F7D7E8437
:105270008D8B7D7673747F8381838484868483871A
:105280008481848379717375737376797A7B7B7D7E
:105290007F7F7E7C76767A7B7675777B868482804C
:1052A000868A8D8E8B8788888A8E929392918E9231
:1052B0009595928F8986858791948B858B93979905
:1052C00095908F8F8D857F848D8B89857F81878A4F
:1052D0008E908B8D8F8882807B7D7E7979797879AD
:1052E00077797A7A7D7C7B77777F817C76767B7D18
:1052F00080807A7A7D818689878483878E8E8B876A
:10530000878C908E89837F7F8181807F7D7F7E7C6B
:10531000797575797B7B7773777C7E7E7A77787DFC
:1053200085878582796B6A778A9BA094837674845B
:105330009697896D4E4759748586786A69717E881B
:10534000898783807E8083868B8E897D77787B8238
:10535000847B695B5C5F6261605D5D616667696EED
:10536000757672706F71767B838B8E8D88827F816C
:105370008182858384888988858994A1A49E948A62
:1053800084878C929DABBAB79D898695ACB09263A9
:105390003E37527B87755A4B546F90A0826F6D7E5B
:1053A000929A9A8E7C6D676F8395978A6F5A5F7613
:1053B000837C63483A435B6F75634F556F8EA0964D
:1053C0008174798DA3A79A90919EAEAEA2A0A6AA51
:1053D000A9A29C9FA3A4A7B0BFC5BBA7A1AEBDC9EE
:1053E000BD956D6B93CEE9CB8E636C9FCABD844D2A
:1053F000354A78938155384265858C7A6354505B81
:105400006D797768554A4B576774756C5E565C6B5F
:1054100079786A5F5D5F6268727A776F6B707678B1
:105420007471757F868B8C8D90979EA3A49D9DA291
:10543000AAB2B6B5ABA3A4AFC1CEC4A592A2BDCF4C
:10544000C09673738DB7D5CC99675E87B3B6895113
:1054500041556665574C48443F404C575F5E49365E
:10546000313F5768604B444C575D63738586736862
:10547000707E8984736665686B6D6A676C6E6E6E2C
:105480006E6E6F757E84878C949BA09F9A999AA16B
:10549000A6A6A6A1979294999EA3A8B1BDAEA3B0CB
:1054A000CEDEC5978EB7E1E0B89393ACB5A49284F5
:1054B000684938455B5D422D303D434E63705D3C2D
:1054C00033567F87715C606F726F7886866E555E2B
:1054D0007B84725C4D4A525C6465615F626F7F865B
:1054E00084807F7D7E7F878F948F837D879596894B
:1054F0007D818D969A8F858795B2C8BFA191A2C0F4
:10550000C8C1D2F9F1BA9DB8DCD5AF929088716864
:105510007D8A765A5574A0A9876062847767706C1B
:105520004C3541534E382F42585B54596468656975
:105530007785826C606B7D7865616B71716D71765A
:105540008094AAB4A8938A9BABA28A746F7D909230
:1055500087777691ADC1D5D5B493A2D2DEB59FC37E
:10556000D9B293ACC6AA7D76888D7A666583A3ADE1
:10557000AEBECDBE9F949D9462281D3D45230E1066
:10558000111127567B7C666585AABBAD875E5A7470
:105590007F6A4D2D1D2F5B77715D5E73B3BEAC903E
:1055A0008798ACA078574F67878D7C727888A4C4A1
:1055B000D3D1D8E1CA9A96C0C39690B1A6808AAFDB
:1055C000A2715A6981897965719BBAC1C2BDB09ACD
:1055D0008B8A87663019293A321F110B112F5B6EA7
:1055E0005E495886AEB1916D5963818E714326290B
:1055F00054857F554D6D90ADBCB0998F98A8AE9EE7
:10560000795E6B868A776C71808D8E91A3C1DAC9C1
:10561000937CA5D4D3BFA57E76A7C8B0646086A2CC
:10562000916F687EA8D0D2AA8FA0BCC4B7986344FB
:105630005A776D4F372B2E4F7C8869434C83A8A037
:105640007B52486A8C8970573C2F4B787D573E546B
:10565000839A9589828C96918F9993786572929BA3
:10566000836F7581858186A5C3B6877BA3D6D9A8AC
:105670007F92C9DABA9989837D798298997A5E672F
:1056800091B9B78C6F84ADB49680735B556A7A62BA
:105690003831506E716957485066747C52445E745C
:1056A000685D6B776C58556C7D70646E77757E8F16
:1056B00092867A809AAD99786B7CA0AC907373894E
:1056C000989AA6B49D788AC4D5A98298C8DAC79A50
:1056D00070687D90958A6E57618AAB986D648098EA
:1056E0008D7D868567516C8C8257404E70816D50E0
:1056F0004C585A5F63554C5864605B5956586773F1
:105700006C57516888937E718199A3A1937E7A909A
:10571000A8A5917C809DB5AA948A97B3AD8485B5E0
:10572000D6C29F939EB4C8C8AE8767719DB3976D6C
:105730006581A6B6AB9D948C909AA19067485268FB
:105740006854402F23315864432D3958747C6B5A68
:10575000647E8784817767667585816758678083F3
:10576000766F74808482848C8E8989959A918F95C6
:105770009790898995A6A68F7989BCD6B8979AB54E
:10578000CBC9B39F9A948F9DAA977676878B8D907D
:105790008273767D8080785F464B62693C34384006
:1057A00047473E2E28395A6F6D6A6C768FA4A59BA9
:1057B000948D8C90928A7A717476747478787475FA
:1057C0007F8E9791858594A7B0ACA4A1A1A09F9D41
:1057D0009890817888A09B898793A2A9A7A0A2A965
:1057E000AAAAB0B6B2A29AA1A4A0968A80787A7F1B
:1057F0007762585E666961524D535C5A4C43444728
:105800004C56606966677A9293878C9EABA2908EA5
:10581000999B9187827D80827E756D698284787381
:105820007F919C9D948E929C9E948D8A84828C8F75
:105830008B8985838A908A848A95A1A4A0A1A7AA2E
:10584000ABA69C948D8781838474646472756C6349
:1058500060666F71695E5E6363635D5D5F646970FE
:10586000787A77757F8C8E877D7B7E807F7B787A58
:1058700078777B7C7875726A6A757E7973737A83C0
:10588000868B908F87828C989A918C93969293991D
:10589000948888949FA19F9D9DA3A6A8AA9F918D5F
:1058A0008A87837A706D6B6D717474706E71788293
:1058B000837D7C82837D7B7E7E7D7A746B696B6465
:1058C0005B58585B5F5F5D5B5B616767696D7277B3
:1058D0007B7A74757D868A8882848F999C9B9A993D
:1058E0009A9FA3A4A09D9EA6B2B7B0A7A9B3B3AB3D
:1058F000A7A39F9D9E9D9E9B9289898C8B837D787B
:1059000074727275797C7D7A7C899BA09D9694993E
:10591000998C7E7770645851483C2E2B312E2A2961
:10592000313B41484D525D6A767E878A87868B92ED
:105930009BA19B93939EABB1B4B5B4B5BAC2C2BBA5
:10594000B2ACAEAFABA0949294948F8780808588E0
:10595000837B787A80858886838386909D9D948DCD
:105960008C8A89868683776964665D4D413D3F38C0
:105970002A1E1A1F201D1D22292D374758616778BE
:105980008893979DA5B1C0C8C8C5C9D4D8D3CBC288
:10599000C1C1C1BFB7A9A3A4A6A39B968F8F8A89B3
:1059A0008C877C798084817C7D828A89878E979799
:1059B000908D8E8E867C77756E6052484843342B6E
:1059C0002D2F271F242B2E32383C3F434C5968691A
:1059D00068717C868A8D949EADBAC4CBD0D7D9DE4F
:1059E000E4E2DCD8D5CBBDB3AEA89F938D8F918B6D
:1059F00084838789837E848C8C888A8E9496939006
:105A00008F8F87807F7E786D615D58524C473C3721
:105A100035312F2B241E1B1E242829293942515E83
:105A2000656F7884939CA2A5ABB6BEC4C6C9CACA2A
:105A3000CED5D8D3CDCECAC4C5C6C3BEBAB8B9B404
:105A4000ADA6A1A2A1998F8985827E7F7F7E7B7A78
:105A50007C7E7F7E7B7574726E645A534A423C37FB
:105A6000312B231B171B1D1C1C1F212933384349B5
:105A70004C5D6E6A6D777A7E848C98A5ACB5B8B6AD
:105A8000BBC6C9C9CACDD0D3D1CFCBC8C6C4C6BF87
:105A9000B3B2B3B2B0AAA5A4A4A4A4A3928C8889DB
:105AA00089837870706D6563625F5D5D60625B5372
:105AB0004E4E4E4C463F3E3D3B393936363C3D3FDF
:105AC00042474A5059606469717B858B8F929AA5D1
:105AD000ABACB1BBC1C4CACECECDCECDCECBC9C48A
:105AE000C2C2BFBCB9B8B4AEA8A6A49F9C999495F5
:105AF0009088817F807B76726B666665625B504CB6
:105B00005054534F4D494C4E4C4C4C4C4C4B4A4BC3
:105B10004E4E4B4C4F53575A5F62686D73787D827F
:105B2000898D929AA0A2A6A8ACAEB2B2B3B3B5B713
:105B3000B8B9B9B7B5B1B1B2B1ABA9A6A29C9692AA
:105B40008E8B89858582807E7A797C7C7A7676795F
:105B500077736F6E6E6B6866656563605F5F5F61CC
:105B60006160615F5E5F5F5E5F5C5C5F6465666B2A
:105B70007074767B7D82898F959BA0A09FA3A8AA35
:105B8000AAABADAAA8AAACACA5A1A0A1A4A4A2A1AD
:105B90009F9C999897928D868585827B716C6867AA
:105BA00067656163686B6F716D7176747376767219
:105BB000707174726F6C6C6C6C6E70706E6F7070F4
:105BC00073727275787B797C7F7E7F7F7F8284871A
:105BD0008A8B89888C91959291909191918E8A8BE4
:105BE0008B89888685807E8184848382828687886B
:105BF000878785858482817E79767473706F6F6EF6
:105C00006F737577787A7D7E7E7F80807F7D8184DB
:105C100081838889898A8A8C8D8D8B8A8A8A8784F8
:105C20008484838488868483888989898681808224
:105C3000848483817B7C8287837F8082817D7D7F5A
:105C40007D7A7B7C7D7F7C7A7C80817F7F7F7F8279
:105C500081807C7E7D787A7C7C7E80838382828456
:105C600086888A86888B888C8C8B908D7C81949298
:105C70008B8B8B898A888A8988898C8986838282A2
:105C8000827F7E7F8283807F7F7C7A787576757154
:105C90007073757474727174727373767E7C7B7CAE
:105CA000807F8181818181828486858283858683CC
:105CB000818283848484827F7D8083878885807EBF
:105CC000808185858280818586837F828484827EAF
:105CD00081848684838282828281807D7E7E7E7FB3
:105CE0007F7E7E7B7C7C7B7B797777797877767615
:105CF000797B7776797978797A7C7D7D7C808482EE
:105D00007E7E7E81838585827F8183838282838478
:105D10008586848386868786838283878A89888925
:105D20008B8A8988888888888888868283888988F9
:105D30008A8C8A8583868684858683817F7F7E8020
:105D40007E7B7E807F7D7D7C7E82848787878A893B
:105D50008882828280808486858584848383828110
:105D60008080828384818080818282818184858415
:105D700080807F81838282838383838385848283FF
:105D800084827F7F7E7D7E80807F7F7D7A7D7E7F27
:105D90007F7D7E7E7D7C7C7E7D7C7C7B7A7B7D7D39
:105DA0007D7E7F817F7D7B7C7D7F7F7E7F7F7E7F11
:105DB0007F7D7C7C7B7D7E7C797A7C7B7B7C7D7E21
:105DC0007E7D7D7F81807D7C7B7C7D7F7D7A787A06
:105DD0007A7B7C7A7875777B7C7A7C7D7E7E7D7C15
:105DE0007C7C7F7E7E7D80818181838180818282B7
:105DF0008386878683848886858784818080818264
:105E00008383848587878686868889878586898C2B
:105E10008B8B8D8F8E8C8B8B8A8A8A8986828184EC
:105E20008586878887868686888687888785828113
:105E300080828584807F807E7F7F7C7B7B7D80806D
:105E40008080808080838384817F80828382807D44
:105E500080828281808285828183817F7C7C7B7B42
:105E60007E7E7C7D7F8183807A7D8383828587852A
:105E7000838284838282807F81807D7E7F7F7E801B
:105E8000808286838080807E7B7D7D7C7B7B7C7C2A
:105E90007C7D7B7C7D7E7F8181807F7F7E7E7F811C
:105EA00080808182817E7D7D7F7F7E7C7E7F8382FC
:105EB0007F7C7D7F808181808280808080838280E2
:105EC00083858280808485858281808284848383A7
:105ED0008483818082817E7D7E7F7D7E81808081C2
:105EE000828183848585817E7D7B7A7B79787A7DCA
:105EF0007F81828587878686878785818285878857
:105F0000888A8B8A8988868686868786858586851F
:105F100085868785817E80807F7E7C7E8384848762
:105F20008986817F807E7C767476787B7E7D7B7EA1
:105F30007F7E7F868B867A7B827F7B7E7F7E848856
:105F4000817F838485888A85807D7C7F7F7B79774C
:105F50007A8081848484838282828383817D7B7C36
:105F60007B7B80818283848383878B867A7A7C7C27
:105F70007A7573737B807E7F808083878786827F3C
:105F80008181807E7A7A7F8586848188908D8380E6
:105F900086898484837D7C81848486838587867FCB
:105FA0007775787B7D7D77777A7D80848380838128
:105FB0007D7E817D77787D7F7F7F818487858081ED
:105FC000847D7271809395878292A19C9088847C55
:105FD0007065626C6D656878869099A1A49E9697AD
:105FE0009D9B8F847F7B78797D8287898B9298981F
:105FF00096948D827D7B766F67625E5A5B5D5E6094
:1060000061646C716F656883A7B8AF9A8989958F51
:10601000735437242533445E7C8F96A7E5F2DAB2B9
:10602000A1A3A39B90878178666381959292A0AE8D
:10603000B4BCC5CABEA795897B62473D372F2F3CAC
:10604000484E5358616A6D6E726A595161819383EB
:106050006255647374624D372631547A919193B7C7
:10606000DBF0FFD394A4BC9E8C918070696683A6FC
:10607000A9A0A1BADAE7E5DDCBBCB6B7B7A9845EC3
:106080004F4E4D412E22273950636C696D737878DD
:10609000756B543D3039536C654B466087775B496F
:1060A0004F667A7D747698BBC6BEB2ACADAFA6958E
:1060B0008A888A95A3B5BCB0A5B9E1F8F4D9B8AF80
:1060C000C0D0D0B7917370828C7144333C4F6B7ADF
:1060D0006A504B566773644936323C556F6F5A4964
:1060E0005370837A60423946576973696174A1C6F7
:1060F000C9AC918F9FA7937B6E6A748C9F9D8E8F86
:10610000A8CBE8EBD7C1C0CAD2CCB5917067737782
:106110005A3B2C3650686E63544C566C6B4A39406F
:10612000556C786E5E59627582785D4339445D7353
:1061300075655A6D98B8B79B8687979E9986746ED9
:10614000768DA2A19391A5C8DED7BFB0B4C0C9C057
:10615000A27E6B71786B52444C5B616A706C615FBC
:10616000666F7269584D4F5F7781725F5B718B8A82
:1061700067484B5B666B6C6D6D7490AFB4A28C8A94
:106180009DA89B8580888F989DA1A2A3B3CDDAD1CD
:10619000C1BCBDBEBBB2A595847F7F7B5E5E6D7CBE
:1061A0007C797B7A716569797B6853536A858B7BCF
:1061B0006A748C958678706C6D6F7683897F78872A
:1061C000A1B1AA8E7A8291928E8C86848F9EA29B98
:1061D000949DB0BDB8A9A2A09B9088867B675A5CAD
:1061E00060594C4B57656F766F605B5C656C5C4DBE
:1061F000566974786E6A7886877E7B7F7D726F7948
:10620000818487817E8795958A827F80858A8A8A24
:106210008E9496939196A1A5A39EA0A69D92878504
:106220008883725D55575A57585D666F716F6F71ED
:106230006F655B6575746C7172707C89857B7D851B
:10624000898782889296938C8E9DA390807E859676
:106250009986797B86969A8A828B96A8AFA9A79908
:10626000889AA99788857A6D625856585451545B1C
:1062700060606571757173716D737C7A6F70757123
:10628000737C7F7F8184828496A6A59B9CA4AAAA06
:10629000A6A29889818B958F837D8393A09997A1DE
:1062A000A6ADB5B4ABA49B97998A7367666459533E
:1062B00055575452575D666968676A625E6B7369C9
:1062C0005C64767E726772848B837C82939C9697E3
:1062D000A5B0AAA0A3A9A3938F94948A807C838B52
:1062E0008C8D949B9C999BA8AFA391919A9A8B7249
:1062F000666B67554D4F4E4F4E4F596165646562F1
:106300006163696A625D5F6D7A79726B6F8392898E
:10631000818C9EA09DA0A7A7A1A3B0B490909C99AA
:106320008C88888D9296979B9D9A999D9D96939423
:10633000928A80797672685D56514E4A4E52524F1B
:106340005562675F5F686E706D66687176767B7F99
:106350007A7785989C918A97A8ACA8A6A7A8A29EB0
:10636000A5A79D8E8E969C968B8C979C9693989CB9
:106370009996918F93938E8882796E6B6D675A4F41
:106380004B4E50514C4B555E5E5F616264696A676B
:106390006466686971797373818A8D8F949A9A990A
:1063A0009B9D9A98928F9192918E898686868C90E9
:1063B0008E8D8F8D8B909B9D948D8D918F857A7313
:1063C000787973685E595D6464605F646B706F6B4D
:1063D000696B6F716F6E6D6C6C71726F737C868A96
:1063E00088858C9AA09C928F98A5A3978E9398935A
:1063F00088858381838A8E8A878A949B97929290DC
:106400008F8F8A847E7C7C7D776D6B6F7476716FE5
:10641000747979797878787D7C78797B7D7C7E81D8
:106420007E818A8F9191969B9F9F9D9FA5A59F9E00
:106430009F9E9E9B94929292929294969895989AEF
:106440009D9B9692928F8B8A89837B7370747168FF
:10645000676C706F6D727779787978777878747007
:1064600070716F6B69686B6B6C707375787B80890A
:106470008D8A8A8F948F89898D8D8683878C8B8472
:1064800080858A8F8F909192929696928E8D8C8530
:106490007E7A777A7567616C746F686A75787677DB
:1064A00076797C7B7979746F6F6F6A666663676AE9
:1064B00069686F767B7C7D8286827E7D7F807D763B
:1064C0007578787B7B787B8081858686868B8E90BD
:1064D000908E8A8B8E8C848082807C78797C7F7F82
:1064E0007E81888E8F8F908F9395938E8B898584F4
:1064F000827B787A79797C7E818787898B8B8A8D7C
:106500008B8988888783807D7E7E7C7A7B7E828370
:106510008587898A8E9190908C8A8989807D7F7DFC
:10652000787576787A7C7F878C898A8A8B8E8E8B39
:106530008A8A8785817C7777757577797B7E80807D
:10654000807D7B7D7F7E8183817E7B797776797C80
:10655000787271727475777370747A7C7B79797DD7
:106560007D7A797772727477797A797B7B7E82888B
:106570008A8C8D8D91929292959695938F8887852E
:10658000838080878C8D8C8C8D8D8E8D8D8C8A8B6D
:106590008B8A8987878583807E7B7C7B78777675FD
:1065A00074797C7977787976747070737374747693
:1065B0007A7D7D7F80838382848789858385898CAA
:1065C0008A858286888A8885848789888583848766
:1065D00086838487898986858687898987817E8164
:1065E000848582818082858482807F7F7F7E7E7D9C
:1065F0007F7E7E7D7F818384848282838585848182
:106600007F808180808080807F7F7F7E7F7D7B7B9D
:106610007E7D7C7E82878682807F7F81868787865B
:106620008A8F8B86858587878687898A86807E7F05
:106630007F7E7F7F7E81807F7E7B7A7C807C777A85
:106640007D7F7E7C7D7F7E7E7E7F7E7C7C7E7C7B74
:106650007C7C7C7F7F7E807F7E7C7E7F7F7F818055
:106660007F808181828586868686868181828180FF
:10667000828282807F7D7B7B7C7A7676767574766B
:1066800076787C7B797978777776777678787B7B84
:106690007B7B7A79787C7F82828484848483838202
:1066A000818181858682838687898B8A8B8D8D8C7B
:1066B0008B898B8B89878687868482808081838380
:1066C0008588888A8B8C8C8A898B8B898786858440
:1066D0008687888786858684807E7E818382808087
:1066E000808281827F7E7B7B7F807C7D7D7E8081BE
:1066F0007F7F81827F7F7F7F807E7D7D7F7F8182A4
:10670000807D7C7F8083837D7A7E7F81807E7F8198
:106710008384828082827E7F7F8083828082807F6A
:106720007D7F818382828382818384848486868341
:1067300080828484838385837F7E7D7D7E7A7A795F
:1067400078777777787777777779787778787A7ACC
:106750007C80807F7E80807B777879787A7B7B7E77
:106760007D7E7E7E7F808082838483838485868510
:1067700084838386858384858484868889868586C8
:1067800087878685868987848484848381807F7EC9
:106790007E7D7E7E7F828382828180827E818182F5
:1067A0008588878989888B8A878A8D8E908F8B8848
:1067B00085878D8B8885827F7E818283838282809C
:1067C0007F7E7D7E807F7E7C7878787876767A7919
:1067D0007879767575757676797C7C7B7C8082831A
:1067E00083838383848588898683848585868A8B51
:1067F0008A8989898A88888B87828385817E7D7E44
:106800007F7F81848583808080807E7E7A77777A9F
:106810007D7C7B79787675767778777575777979F9
:106820007978767B7B7A7A7A7A7A7A78777A7B7BD0
:106830007A797A7D7E818180828384848283848454
:1068400086847E7C7C7D808180828386868584832D
:106850008383827F7C7D7E7F7F7F817F7F7E7D7F44
:1068600082858586868788878888878584838586CC
:1068700085838283848484848485888B8B8E9293A1
:1068800092929492919191908F8F8D8B8A8B8C891B
:106890008685828080817F7E7E7F818181807F7EF0
:1068A0007D7B7D7E7C7D7C7C7C7E7D7D7D7E7E7C1B
:1068B0007B7C7E807F7E7E818485848386858481C7
:1068C000808080838488898A8888858282807F7F8F
:1068D0007F7D7C7C7C7D7D7E7E7E7D7D7E7F7F7EE0
:1068E000807F7C7C7D7D7E808080828282828180B0
:1068F0007E7F7F7E7E7B7B79787A79767676777AF3
:1069000079787977767676787A7977787E7F7E80EF
:106910007F7B7978797A7C7D7D7C7D7A7D7E7F80B6
:1069200080818281807F7F7D7D7D7F7E7D7D7F7F79
:106930008084868686858281817E8082828183832F
:10694000878A898A8B8C8E8F8D8A8A898A888688A5
:1069500087868C908C89898A8684858586878687B8
:1069600088878786838384848481848583838583E1
:106970008587848382807E7C7F7F7E7E7C7B7C7D1E
:106980007C7D7D7F828382807F7F828283827E7D09
:106990007B7A7D7C7C7D7F81828181828281818204
:1069A000828181807F7F7F7E7F7F7D7F7F818382E9
:1069B0008080828080818484828380807D7D7D7ED2
:1069C0007F7F7E7F81807E818586868483817E80B5
:1069D0008182807E807F7C797A7D7E7F7C7C8282D2
:1069E00081807E7E7C7E7E7F7E7D7E7C7C7B7B7BD1
:1069F0007D7F7E7E8286817F7E7E82817D7D7D7AA7
:106A00007979777877787A7A7A7C7F7E7F818182CC
:106A1000807F7E7C7E7E7D7B7C7C7D7E7F8085868C
:106A2000848587868585858689888785848384850E
:106A3000838184888A8B8D8B8A8D8B8786868586D9
:106A4000858383838383838586858282828386840C
:106A5000807F8485828484817F80808082817F8022
:106A600082838484817F8082817E7D7D8185848212
:106A7000817E7E7E7E7F7F7E80838686827F80840D
:106A800085858585848484848586847F7F7F8180D5
:106A90007D7B7C7D7E7F7D7E7D7B79797979787742
:106AA0007B7B7A7978787B7E8080807F8082808013
:106AB0007F7E7F81817E7C7B7B7A7A7A7A7C7D7E09
:106AC000807F7E7F7F7E80808283828283878581B4
:106AD0008284868684828184868684858583838673
:106AE000868683817F7F8183848380838282807F87
:106AF0007F807F818082827F818282818382828285
:106B00008080818080818183848385888B8B8A8843
:106B100086868587898986848384898C8B8A898AFD
:106B20008A89898887888886848484838282817F11
:106B3000818487888584828183848080848585841C
:106B4000807D7C7C7F807F7D7E7F807F7F81828255
:106B50008284828384818183818080848586858507
:106B60008281828181828382828283827E7C7B7920
:106B7000797B7A767879777476777878777577779E
:106B80007A7F7E7F827F7D7D7C7D7E7D7E7F81831F
:106B900081828281818180807E80838483808080E5
:106BA0007F807F7D7F807C7D7D7B78787B7E7E7E15
:106BB0007D7C7C7A76777978797A7C7E7E7D7D7E25
:106BC0007E7C7A7D7D7A7D807F7F807F7E807F7FE7
:106BD0008183828384848382827F8182818080809A
:106BE000808386868585848383838381817F808477
:106BF000838587898E8E8F8F928F8C8D8B8A8B8ADF
:106C0000878788888887858687888989888788890B
:106C1000898A8887878582838380807D7E7F7E8145
:106C2000818285858383817E7E7F7E7E8080828255
:106C3000818584818181807F7D8081818283808242
:106C40008282807E78797976787D7B7B7B797B7D8B
:106C50007D7F8282807E7E7F807F7E7E7C7E7F7F46
:106C6000828584848581807F8284828182858786F3
:106C7000807F807E7B7A797A797777797B7A7C7B63
:106C80007C7E7C7C7A787776757879787977767877
:106C90007A7B7C7E7C7976797D7F807E7E807F7F2B
:106CA000818283868484878A8A8A8A88898C8C8A6E
:106CB00088868687888A898A8D8988868180818569
:106CC0008685838283828080818181838283807EA6
:106CD000818483838382808082818485838181868D
:106CE000878784868889868685838386848485854C
:106CF000878786878C8D898886848586888A898A15
:106D0000888583847F7D7F8183817F7F808082816E
:106D10007E7F81807E7F8080828383838484838260
:106D200082817F7F7E7C797C7D7E7C78797B78799F
:106D30007B7C7D7F7D7C7D7A7B787878797C7F7E9B
:106D40007E7F7D7B7B7B8083817F7D7E7C7B7B7B6D
:106D50007C79787A7C7E7D7D7F7E7F7E7D7D7D7F68
:106D60007F7D7D81817E7D7F7E8081828283818027
:106D70007F8181838483818486878482807F7D7AFA
:106D80007A7B7C7C7A78787675777978797B7C8168
:106D9000838280807E8081828181838385848180DB
:106DA0008182838484858585848382868788898798
:106DB000878A8C8C8B8D8C8A8A8A8B8986888C8931
:106DC000898C8B8989868788868281807F7F7E8473
:106DD000868788888887858585868786838281815E
:106DE0007F80807F7F7F7F7E7F818282828484819B
:106DF000828383817F80808180828481827E7B7E8A
:106E00007F807E7D7E8081827D7B7B7C7E7E7E7DA1
:106E10007B7B7E7C7E7F7E80838282837F7F7E7E83
:106E20007F7E7D7F807F7E807F7E7D7D7E7C7A778A
:106E3000777B7E7C7D7D7C7C7D7E7A7A7B7B787A9D
:106E40007C7C7F7F7B7F7E7A7B8081828585878645
:106E500084848685848282848281838180807F7F0E
:106E6000818282838180807D7A7A7C7E7D7C7C7B3E
:106E70007C7C7B7C7C7D7F807E7F7F828788878512
:106E8000848482817F8184868682848888878888BA
:106E90008686888A8E8C8B8B88898885878686886B
:106EA00087868686868786827F7E80828382807EB2
:106EB0007C7B7B7B7E7F80807F7D7E7E7F7F7E81F3
:106EC000807C7D7F808080807E7E818382828181C4
:106ED000838483808080828483807F818584837F94
:106EE0007D7D7B7B7E7E7E7D7A7B7E7C7C7C7F7FD6
:106EF000808083827E7C7B7D7E817E7F807F7F80A1
:106F00007F80828180828281868786848484848255
:106F100082817F7F7E7F7F7E7F8081827F8184836D
:106F20008180808083817F7D7B7B7D7C7B7C7E7D7F
:106F30007C7C7B7E7F7D7D7C7A78787778767574B3
:106F400075777877787A7E7E7E7D7C7C7B7C7A7C98
:106F50007D7F8081808082858889898A8B8B898BDF
:106F60008C8A8A8B8B878687888B8C8C8E8D8D8D77
:106F70008A8A8B8E8B87888A8A84828281818282A8
:106F80008386878A8B87868784827F7C7C7D7B7BD8
:106F90007C7B7D7E7C7B7B7C7A7B7C80807D7C7C2B
:106FA0007E8080808082807E7D7C7B7D80848484E6
:106FB0008788888A8C8B8B8A898986838382828062
:106FC0008080818181807F7E81808080807F8082BF
:106FD000827F7E7E7E7F7F7D7D8082818081827EBA
:106FE0007F8281817E7E7E828482838684817F7F90
:106FF000807E7B7A7A7D7F7E7C797C7D7C7C7C7ECA
:107000007E7D7E7E7F7F7F7E7F8180807E80838687
:10701000888A88817B7B7B7A7B7B7B7C7E7E7F7D85
:107020007D7B79797B7B7A7C7E7D7F80807F7E8093
:1070300082858383818080808281828485868C8E14
:1070400089908E7D808F8D8A8C8B8B8B8C8B8784A7
:10705000858687898887878782817F7F81818281F2
:107060007F807E7B7A7A7E7E7C7C7E7C7A7C7D7F54
:107070007C7A7C7C7C7B7A7B79787A797A7A7B796A
:107080007B7F807D7D807D7E818181818180828208
:1070900084838589878988868A898885868581828F
:1070A000858280818080828383817D7D7D7F7E7EDD
:1070B0007B797B7E7F82807F807F7E7C7B7C7F81F3
:1070C00081818080817F7C7C807E7F7F81807F7FCB
:1070D0007C7D7D7F7B797A78787A7C7C7B7A787905
:1070E0007C7D7D7877797A7877797A7B7D7E7E7CF6
:1070F0007B7A78777879797576757574767678791C
:107100007A7B7D7F81828486838382818485858862
:107110008A878686868584848686878988898B8AFD
:107120008A898686898B8B8A86858585898A8788E0
:107130008A8A888785858686848180818181807F0F
:107140007F807F8181817F828486827C7A7D7B794A
:107150007A7D7B7A7A7D7F7F7D7B7B79787C7F816E
:107160008384858583868887888A8B8888888689B2
:107170008B8B8C8B8B8C8A89878585898A88878481
:107180008586888684807F82828080807E7E7E7CE9
:107190007A79797C7E7E7D7E7F7F7E7E8084828010
:1071A0007F7C7A7A7B7B7C7D7B7D7E7B78787A7A2C
:1071B0007C7E7E7D7E7D7B7B7D7E7F7D7E7E7F80F7
:1071C0007F7F8285868482848581807F7D7B7C7EB3
:1071D0007F7D7C7B7C7C7A7877787A7A797A7B7809
:1071E000797C7E7D7E7E7D7E7F7E7E7F7E808080C0
:1071F000807F7F8184888B8D8D8C8D8F8D8C8F90FF
:107200008F8F8E8D8F8D8E8E8D8E8F8E8F92908F95
:107210008C8C8D8E8C8A8C8D8E8D8785898A8B8CBB
:10722000898783818483818181808382828586822C
:10723000807F7F80807F7E7F817F807F7F827F7B5A
:1072400080878684848282848081838285898987FD
:1072500089888888888988838282828281848383DE
:107260008686848584818182808082848383807DF8
:107270007E7C7B7E7F7D7F7F7E7D7B7B7F80858824
:107280008788878282827F7F7F7C7C7E7D7C7C7BFF
:107290007B797A7D807F7F7E7D7C7C7D79787A7B2F
:1072A0007E807F7F7E8283838482818384848481C5
:1072B0007E80807E7B7C7C7D7E7C7E7F7E7F7E7DF3
:1072C0007F818080818282818181838380828384A7
:1072D0008686868688888A8A898A8A88888888892C
:1072E00086858685838485878989868684807E8352
:1072F00086847F7D7E7E7E7F81807F7F808382808B
:107300007D7B797A797879797B7A7A7B7C7A7C7DD6
:107310007C7C7C7D7D7C7A77787B7C7F807E7C7EAC
:1073200081828181858582818384827F7E80818143
:10733000808181807E7E7E808184827E7F82807E4D
:107340007F8082817F81828181848481807E7D7C37
:107350007D807E7E7C797C7E7D7C7B7A7977787A75
:1073600079787A787374737372706D7072706F70ED
:1073700070707477797A787A7A78767A7A7B7D7E8B
:107380007D7D7E7C7D7F7E7E7F80807E7D7D7E7E1E
:107390007F82807D7C7B7C7E7E8081838282807FF9
:1073A0008081807F817F7E7E8082858585848485C3
:1073B000878985838381828788858686888A878571
:1073C000878687858481808385868585848381837C
:1073D00083818586868788858282828282827F7E7B
:1073E00082858483868582807F7D7B7B7B7C7F8199
:1073F00083817F807F7D7E807F7F81818287898975
:10740000898987888B8B8A888889898A8B8B8C8EDF
:107410008E8D8C89888787878787898A87858583EA
:10742000818183858383848180807E7E7F7D7A785D
:107430007A7978787A7A797C7D7A79797876767AB9
:107440007C79797C7B797A7976777777797E7F7AA0
:107450007A7C7D7A7A7A7B7B7A7A7A7C7F7F818468
:107460008785828180828382828283858482807FF5
:107470007E7F7E7B7B7C7C7E7D7E80818282807F26
:1074800081828586828284848485878784858888B2
:1074900088888A8988898989898687898684858672
:1074A000868685868785868888868685868586857C
:1074B000858283828183848688888482828384848F
:1074C000848281848685858281838687858585837C
:1074D000828485838082808083807E7E7E7F81809F
:1074E0007F7F838585868685817F82848585868565
:1074F000827F7E7F80807F7D7E7D7D7C7D7F83829D
:1075000081848584848485868581807F7E80828055
:107510008084858988878989888889888180807E18
:107520007D7B7D7E7F80807C7E7D7C7A7B7C7F7F87
:1075300080807D7D7E7E7C7D7D7D808082837F7F5F
:1075400082817E8183817F81807C7C7C797B7B7A58
:107550007B7E7F7E807F7F7F7E7C7E7F7E7E7C7A4F
:107560007C7C7D7C7C797C80807F7D808181828435
:10757000858384878785858483827E7D7F7F8486DB
:107580008482848A8A8785858383858586848181B0
:10759000817F8181828584818281808482838280CF
:1075A0007E7F80807F7C7D7D7E7E7C7B7C7D7D7E02
:1075B0007C7E7E7D7E7F7E7F807F818385878A86BD
:1075C00088898A8A8B8B8886848485858685878747
:1075D00088898886858684817E7E7E7F7C7D7F7D8E
:1075E0007B7C7B797B7D7D7C777777767879787704
:1075F000767474757877797A7B7C7C7A7977787A07
:107600007A7874737475777877787A7B7C7C7D7EF2
:10761000808182828381807F808081818082838358
:10762000817F7E7E7F818180807E7C7A7B7B7C7A7D
:107630007B7E7F7D7D79777A7C7E80828382807E6F
:107640007F7D7E7E7D7D7F7E7E7D7E7E7F83868448
:10765000818387898A8D8D8B89888B89878B8B8E97
:107660008C898C8C89898A898A8A89878787878986
:107670008A88888888898A8B8982808080808080B7
:107680007E7F80827F7F827E808586888A868484D2
:107690008383848080837F7F83878A8C8A8A89889A
:1076A0008889898B8B8C8C8A888C8B8A878483844D
:1076B0008280818383827E7F827F7B7E7F7D7C7CD4
:1076C0007B7B78767472737474797C807D7B7C7C30
:1076D0007D7D7C7D80828283817E7B7C7C7D7D7CC8
:1076E0007E7F7F7F80807F7E7F7F7D7F80807E7BAF
:1076F0007C7E7C79787879787877787A7D7C7D7DE6
:1077000079787B7C7C7A7C7D7C7B77777877797ADB
:107710007A7B7D7E7E7D7E7F7F8185888686898956
:107720008886888C8B888888858281808382828500
:10773000858382807E7E7F7E7C7D7D7C7C7D7E7C61
:107740007A7D7F7B78797B7C80828282808084874F
:1077500087878684827D7F818183838383807F8105
:10776000838383827E7C7E80838787838080807E04
:107770007F8183817E8182838484858584838485DF
:1077800085858584828284848683818182838486C0
:107790008484858684818080808383847F7F7F7ECC
:1077A0007D7E7B77797B7C7D7B7D7F7E7F8080810A
:1077B000818185847F7F7E7E7C7E81848282817DC3
:1077C000787A7B7C7E7D79787A7B7E7F7E7F7F7FF7
:1077D00080807F807E7C7F7F7E7F8183817E7F7BB8
:1077E000787A7C7E807E7C7B7A76777A7A79787AF2
:1077F0007A7A79787A7C7877797B7C8080828484C5
:107800008385848387858486858282848585899023
:1078100091908F8C8B8D8E8D8A8B8C8B8A88878CA8
:107820008F8D8A878A8B8B8B8A88888886858585C9
:10783000858A868081868989898988878687898AD9
:107840008B8B88868483807F838685838383817FF7
:107850008082807F817F7F80838485827F81817E1B
:107860007D7E7C797A7C7C7F808384848380807F2A
:107870007E7D7D80807D7B79797C80807F7D7C7D35
:107880007F807F808181818383808284817F7E7FEE
:1078900081828382807D8082807D7E7E7D7E7B7AF8
:1078A0007A7C7F827F7D7D7C7F80818283817F7DEA
:1078B0007D7B7A7C7B7B7C78787B7A787C7F7E7C16
:1078C0007A7C7C7B7C7C7977797A7B7A7A7B7C7C0E
:1078D0007B7C7A79797A7E818183838285878483B0
:1078E000848788898B8A88878686888C8B8A8A8C0D
:1078F0008C8C898A8B8C8C8B878385878889898AF5
:107900008986858A8C8C8B8B8C8B868486888885EF
:107910008486898787878583848181848184838223
:1079200081807E7F81828180828383828180808248
:107930008280807F7F7D7E7F838484838282828237
:10794000828282828180828181838381807E7D7C2C
:107950007D7D7A777A7D7D7C7A797B7D7E7C7E7E6B
:107960007F7F7F7E7D7D7C797A7D7D7E7E80838337
:10797000807F818282828282807E7E7E7B77787920
:107980007A7A7C7E7C7E7E7D81838181827F7F800E
:107990007E7C7B7C79787A7A7A7B7B77777678764F
:1079A000757778777A7979787778787A7C7A797D4B
:1079B0007F7D7D807E7E7E7D7E7E7F7D7B7C8184E3
:1079C000828283828284868688898888888886865F
:1079D000868787888887878789898986838285883B
:1079E0008887848586868384888B8987878888862C
:1079F00086868788888885817F828486868382833D
:107A000086898A89888A8B89888787898A898784F1
:107A10008683818082878885848789897F7F7E812C
:107A2000838381817F80808181818081807D7B7A59
:107A30007C7D7E7F828482818080807F8182817F45
:107A4000817F7F7E7D7E807F7F8284878A89888810
:107A500087888886858584817F7F7E7D797A787620
:107A60007675787C7C78777B7A7B7C7A79797A7D7D
:107A70007D7A797879787A797A7A7B7A7B7D7E7E5D
:107A80008284827E7E7C797877747276777B7F823F
:107A90008482838382828384858481818485898AA8
:107AA0008988898C8B8885868A8D8D8B8B8B8C8C35
:107AB0008F8E8E8D8C8C8887878685858281858741
:107AC0008986878887858383878889878888888748
:107AD000848483817E7E7F7F7E8080807E7C7D7EAD
:107AE0007C7B7C7F7E7C7C797B7E7D8084827F7DBD
:107AF0007F8283848382817F7F8080808083838371
:107B00008484848788847E7F817F81858683848244
:107B10008081807F7F7C7C7C7D7E807F7C7B7A798E
:107B200077797B7A797D7E7E7F817F7D7E7E808482
:107B300085817F7C7B7C7D7D7A7C7F7F7E7D7B7C6D
:107B40007D7E7F7D7E7C7A7B797B7C7D7C7A79777C
:107B500075737375787B7B79787A7C7B7A767375AD
:107B600077777B7B77767879797E7D7D7C7E807E6A
:107B70007D7D808080828180807F7C7D7D8082830E
:107B8000838385898D8E8C8A8889888985858C8D6B
:107B90008C8C8986868888888686898A878B908F50
:107BA0008E8C8C8C8A8B8A8A8C8D8E8C8885888B27
:107BB0008D8C8B8A8C8D8A858286878582807D805C
:107BC000818180808082838382807F7F7F808487A1
:107BD0008C8885848383868783848989898A8A8A35
:107BE0008886868483808081848583807D7D7E7C79
:107BF0007B7C7C7E7D7A7C7C7D7D7C7E7F7F7F7EB6
:107C00007C7D7E7F80807D7B7C7C7D7D7E80807F97
:107C10007F7B7A7A7B7D7E7C7E807E7C7A79787AA7
:107C20007C7F7F80807D8081817E7D7B7B7A7B797C
:107C300079787976727275787878767577797A79D5
:107C4000797777757678797C7E7F7F828281828171
:107C50008385878B8C888586888585898B898989AA
:107C60008A87878A8B8B8B89868585858586878899
:107C700088888582807E7D80828384888A8B8B8CB5
:107C80008B888787858382818485868482817E7DB7
:107C90007D80807C7D7F7F7E80807E797A7A7A7C11
:107CA0007E7F80807F828382807F7E7E7F7E8081D8
:107CB00082838281838484868A8B88898B8B898561
:107CC00083807F8083827F7F808283828185878497
:107CD00081828384838080807E7E7D7D7F83868297
:107CE000828282817F7F81807E7F7E7E7D7E7F7E9D
:107CF0007D7C79777576787878787A7773777C7AFF
:107D00007D7F7E7D7B7B7E7E7D7C7D7E7D7D7D7AA5
:107D10007A7C7D7C7D7E7E7F7F7D7A7A7D7D7E7F95
:107D2000807C75747776757777797C7D7C7C7D7EB9
:107D30007D83878483848384898B898685878989E9
:107D400088878688888482838587838183848484E6
:107D5000848381807F7D7D7E818282818182838513
:107D600087878A8888898988898B8783858686869C
:107D7000838487888684848889898B8C8B888B8E82
:107D80008C87888986818586848282828689837DA4
:107D90007D7D7C7D7F7F7F807F7F7E7D7E7F807FFE
:107DA0007F8382807E7B7B7C7E818482807D7E7EE1
:107DB0007F81807E7F7F7E7F7F7E818585828283BB
:107DC000817F7F8085838183838082838080807FA1
:107DD0007F7D7D7E7C78767576787B7E7C797A7DFA
:107DE0007D7D7E7F7F7D7B7C80807B7B7A79787ACE
:107DF0007A7A7876777A7E817D78767878787674F4
:107E000074737374736F7274716D71777773797F34
:107E10007F838A89898C8C8B8C8C8C8B898C8D8DC3
:107E20008E8C8A8B8988868282878886888B8683D7
:107E300082807E7D808383878D8D8D919093968FB8
:107E40008B9494888A8F888186867F81847D7A79D5
:107E5000777A7774767771757A7779797E85807598
:107E600077888C7F77818B857C7B7C807B75757533
:107E7000726F7075776F6F7576767A79787C80839C
:107E80008A90959A9C9FA0A3A6ABADA6A2A9AFAAE3
:107E9000A2A0A4ABA59D9A9799A1958696897E816B
:107EA0007C75797B685F67665F59565A6366605C6C
:107EB0005D646D6A5C5D6F746868757875767574FD
:107EC0007B7D7878736D73777168686D6C635E5CC9
:107ED0005D5D5B57565E65635E5F6D736D70777752
:107EE0007A87939A9E9FA1A6B1B9B3B0B7C0C3BA1F
:107EF000B7C2CAC8BCB6B6B6B4BCB1959DC3BD9A2C
:107F000098A3978F8A6A576D75533F484F504935EC
:107F10003549554F484649565C4F4552675F617039
:107F20008287807E858789867C79878D7F74757945
:107F30007A78726C6E76746A6B798587898D969B78
:107F40009A9BA5AFB1B0B2BEC2BFCACDC5CFDED27B
:107F5000CEE2ECE1D8D8D9D2D0DACEA8A0C7CE9E56
:107F60008A9D947F7863494F573D1E1B2724171322
:107F70001114202115161F2329272534464942456F
:107F80005A6B6C6D77818C928A8085908C7A77831E
:107F900081777476767A7A726B74807C76818B9432
:107FA000908994A6ABA5A4B1B9B1B4C3C5C4C9C9DD
:107FB000CFDBDED1C5C5C4C1D3D3A196C6D1AFA294
:107FC000ACADA89C8A6F67735F38343C342A1C12AE
:107FD000202E24191A1F262D2B252E4952433F519E
:107FE00068726B6E84918C8D8E8C98A08B7E97A519
:107FF0008F839293817C7F777682867A758FA18A30
:108000008093897D9EAA939DC1C9C0BCC1CCD3CDAC
:10801000BBB8D1D0BAC8D9C8D0E0BA99E3BC9CB03B
:10802000B8A9A5967A78817D6C4C384246362418DA
:108030001B2E2E1D14232E2A2523212E43392C449A
:108040005D6362606C818681878E959D9A908B942A
:108050009D8D778393877C7E77768B8B767F9791C8
:108060007E858D8FA0A38E99B1A6A1B7B0A5C1C3FF
:10807000AEC1D3CCD0C6B4BEC9C7C3B5B2D1DABBCA
:10808000AAB8C2AC90898C817C704C4055512F1D90
:10809000232A291F181A2328201C232B3A2B2F5060
:1080A0005F565B71818888898D959C9E94909B9E7C
:1080B0008E84909A8B7D80827E7F7C767885837B90
:1080C00085867B8D9F969B9B94B2BA99AACBB9B9B2
:1080D000CAC0C8D2B7B7D2C5B3C4CCB7A1ABC1B3BD
:1080E0009BACAD88859175636E6E54464C4A3122C7
:1080F0002E2D1E1E251F1A1E272C2E313439404BC3
:108100005B5E5B73867E7D8B92919699969A9A9927
:108110009C958D999C8B858884847A6E866C6E8FF5
:1081200082627FAD9A799AC3A37AA1C9AA97C5D56D
:10813000B1B5DFEDD1BDCCE5DAB7B3BEBBC2BC8E05
:108140008CC3C08A89A093847A5B46525A44252204
:108150002E27181815172722142339332B323945A7
:10816000545549567E8672728A9D9E908FA6AFA600
:10817000A0A7A79FA5A99184959B7D667C97816305
:108180007B9995928F839398839BBC9B8ABDD1A149
:108190008BC1E6C6A7B3CEDBC39EA6C6BAAF9DA071
:1081A000BFB47A669AB8896B8DA18B7A6F57505994
:1081B00055381A1E3E4221162F443B2C313E45486D
:1081C00045434D6271665D7088868491958E908D71
:1081D0008793978C8C898693917D848C7C8795740A
:1081E0006694A9887183ACAE7B72A8B9998E8F937F
:1081F000A9AC9390AAB9B7AE9FA2C5D8B18DA8CDAE
:10820000B89EB0B39191B1A07784A5A07E646D842F
:108210007A4E3A4B55442E242735372A1D45725E37
:108220003037505051544C587273616E828286813F
:108230006974A29A6772ACB07C729FAC908DA5A154
:1082400092A09C7D798178899F825F6A8D9C71481C
:108250007FB5886CA0C5B29F9EA5ABAEA89C99AE19
:10826000C5B1959DB7C4B3939FBEA6859DA38791C5
:10827000986C5E8B8E533D6B85603C4D63594949CC
:108280004A454B574F3A4160684E43647D70606683
:1082900077837C727A87838692897F8BA08A82A477
:1082A000C7B78989C1D9A489B5CAB1ADC0B487801F
:1082B000B5CB9E7B91BCB36A5693996876ABAC897B
:1082C0007CA1CBB18098C6B9928C9AADB69F8583BC
:1082D000949F8B74838F735D5D57544F484E3B154D
:1082E00028503A183F81783D477B73526C8E7E64EC
:1082F0006681958463627C7B5F596F7D7255496CA2
:108300008C7F6451598AB39C5D4282D5BF7D99E1CF
:10831000E2C0B0ADA5A4B9C696709FC45577BCBDE8
:108320006C4989946384AE867EBFDDBA8C94B9A60D
:10833000797F9EAE9D5D4588B484404289B88B4567
:1083400053907E374188956138597D543F7B8857DB
:1083500049597485614C76774A507D9170415E939E
:10836000743B5095B3844251949A717195A9986C5D
:108370005E818F7B7A81848F817B978563869879F4
:1083800081A3A9A68D80A3BDB397645AACDEAE7954
:1083900085B6D1AE87959D787BACAD8185AAA97451
:1083A000486299955E4C82A775364E928F4F417107
:1083B0007E554C6D6F53638A6E2D3380AA712E4C9F
:1083C000A4C58D454D97A35C3D79B29F573670ADDE
:1083D0008D52588FB3995C568CAFAA8146448AA9B6
:1083E00072476DB0BF885A79B2A56769B2D5A560EA
:1083F0005699C2885E9BCAA27881ACC9B089828234
:108400008FA9957074838A97804D517C938D674DA9
:1084100080B08A576499A05C428CB08D725D9DC615
:108420008553576F959171717C8DB09D68627EA068
:10843000B88C4963B3B3664E93BD84474E7C9F9519
:1084400070739179567DA676395FB9C77E364183C0
:108450008F47174C9A97625D8395A09D61346D9EFE
:10846000775681B19E7D99B484639AC7AA91A9B8C1
:108470009073A2CDA36470B3C181597EA996615750
:10848000879C654E8DA3673E5EA9C8854D7BACA2D7
:108490007A464D94A67A6D5C354484A2455BA7AEBE
:1084A000736AA1C6A25D4F8AC5B4655190B3814479
:1084B0002D4986986B5C9CD6C37D4A5EA3B78455D4
:1084C0005E87AC9E614A79A8904D4E847748618F53
:1084D00083605A779A875D6D8E918F7A5261929000
:1084E0006D6588B8C1966E739ECBBE7A6AADD19A1F
:1084F00062679DC69E443478A9834A67A29E8367BB
:108500004A6DB2B47F4C4D8FAE7635428CB98A4BF2
:108510005EAAC99B708CB9C3A76A62A897737A9543
:10852000AB977468523D647D4E3D6E8E865E3C5BBB
:108530007C5F6B89553267805A374588A6766C9880
:10854000A2ACAC8190CEB17E97ADA5935C4492C6AF
:108550008E6495DBD28366A0CDC0895768999B89CC
:10856000888185979E9E8E67527AA792646E888EC8
:108570009F946768817D8A90605CA3CEB6733E5BF2
:10858000A6AF7A6893AF7D4E7A9D7B738A888BA461
:10859000B2965E568B9957244189A7764183965CA3
:1085A000315CA29F613E6488623D60A0BB9A5542E7
:1085B00076979079432A69AAA367335099A2703CB1
:1085C0002E66B2C3B1886492C99559647BA6E6D57C
:1085D0008E98D9EDCD9A6A77BDD09A6C769CAF878C
:1085E00053688C68455F809B9A65518295776C8B48
:1085F000905C497B8C7877614A6077929861609E45
:1086000088586D82787F9EB294687DA59E826B7338
:108610008D8687916F6A9A947C8B7E75A29A8D6EF7
:1086200071AFCD9E5D5994AF7D5E92CBAD6F7AB543
:10863000C38A4E66ABA1625681A9AE896266778D08
:10864000AFA5644A7F9F6C5088BEA661457CA97C1B
:108650004C65929B7F544256819677566E7E61663A
:108660008463335AABBE8D72A6E9D8826694AFB0EC
:10867000AD7C485D7A757D6A3C5BA79F686A9BA567
:108680006C4C7DB19C635F9DCDB06B3F5391AC7FD3
:108690003E214184916660675875A0767EA881432B
:1086A000346FAD965D72A69E7D756A6790995F572F
:1086B00098BBB5B8B18C7F98B9C6A87A81B9CFA25A
:1086C000686CA2BFBDAD8270A8C38A5463A4B8749D
:1086D000375B917D371F66B2A587A1B6A27C6C93EC
:1086E000BD97658CAC8382AC988EB8A6748FB78D1D
:1086F0005264A5AE6D5388B9BC98654967938153A0
:10870000658F77382348663B18518678737E634CB3
:10871000729C7E42588D7A5E6F90AA93ABD9986115
:10872000738DADBC844E4E5E80935D315886755519
:1087300065A2BD8C5A7FCDD5966A95D4BE72689BD2
:10874000A17F91C8C582577EB0904B5EB3CC8C465A
:10875000579FA1583750533E42708B5A3A79B08890
:108760005164A8B87956849F888AB0C1A583848D46
:1087700093B6BD76467CB39B737C9CA78C7184A515
:10878000803E50A0C49C5A344880B1BF934E2640CE
:1087900089B9974E4996BE83526C7F6CB2B3692CEF
:1087A00048909658417BB39E5C5595AF6A3D637582
:1087B00045428DB683495D907C465DA2A37A8FD1F8
:1087C000DFA47AA2CCA36D84B7C39A564789C6B5F5
:1087D00075415CA6A76764A7CDA2584B89C0A45F6A
:1087E0005A909664638E905B345198A36034579E80
:1087F000CEBA7C80CAEDCA998198CFD39E7E9AC0AA
:10880000B3704E78A9976C78AA9D5B508BC5B868F9
:108810005198B5978961305B977B3C30886B48688D
:108820009A915F5786915A3F6472555691AF774D32
:10883000647B919A6B5E919A79767E8D9B7C506574
:108840009EBF9E54478EB790615A6F96BAA46D6AC8
:108850008D8F847C7A9BA86E5AA0B684697086AC92
:10886000BB91595D8D968095A97E576E8D988B78BA
:10887000716A6C7E7357544F40577D775040629BAE
:10888000BCA35C3058A7B06A2C3D86B095718DBAF8
:10889000AD7C77A6C6B07D6481ACA58679677595F9
:1088A0008C6F5D5D799A987C6E7D827993B6945ECB
:1088B00069909EA1935D3B5EA3C39D5F64ADCF9D18
:1088C00087BEDBA6737FB7DAB175798B95B6BC909E
:1088D000767684A3A1796269829986523C5E95A4DA
:1088E0007C4B3C619BAF885C5E839C8871726E6739
:1088F000696D76827255648D8B79868C797A9396C0
:108900007E6B6E84887270867C657092A0937466AC
:10891000737D8990704758838F7D717471708A98C8
:108920007B433866836C556D8E86676D94ADA98EDA
:108930008497947A849689828D8C89897A809B9396
:108940007F8177637B9B896A574947597291AAA7B0
:10895000918086937D6368592B110F173E5F5B658D
:108960007E8BA8DAF8F2E4E0E2D2B8BBC09C655096
:1089700069A1CBC0B5CBD9C9C0D3E0D2A45B406953
:1089800085673F3242553E1822434C353988D6D34D
:10899000BDB9AD9A7153501B015C700E61717EAD13
:1089A000CEEDFCF4F9FBE1B8846A768578553F4852
:1089B0006285BCE8F4EEE5E5E8E6DDCEB48B502850
:1089C0002E3E342F3B434852545E72725F6791B91A
:1089D000C0AB9681572A27372C16121928476A8B65
:1089E000BFECE6C0B3CDDFC4967D6B52434A5E7CDC
:1089F000919294AAD3EEEBE1D8C4AB8F6D5A574C49
:108A0000311C1B293E54677E969888898B796D644A
:108A1000535F8A957E756F533029496B56494F666F
:108A200083A5C8E1F0E9C2ADB8AF8B746B5F535159
:108A30005D738FA2A6B0D1EBE6D1C1B59E7E5F4536
:108A400039353236496176828D9FAEAEA5968574F2
:108A500054313A667B6E67655030203150696C5DE9
:108A60005560738FB4D6E9E5CBADA09071555670C3
:108A70007C716F86A4B6C3D0E1E4D3AE90857B5AF7
:108A800038323B474D536F97ACADAFB6B7AC997F1B
:108A9000654A301F305C79706F7964403941628774
:108AA00089736F8193ACD6F6FDEED0B2977864628D
:108AB0007394A39297B7B7A3A7BECCC7AB846A56EB
:108AC0003E2E32476B83848AA4B3ABABAEA69277BB
:108AD0005430201E1A2B5D888E8C917F5B41323082
:108AE00048656D73818382A0D0F2FBF2DFC9A7785D
:108AF000554D5E88ADB5B9C2B0836E85ABC6BDA21B
:108B00008C6A402A2D3C5C89A5AFB6B2A08F8E89B5
:108B10007466563A2726273F6572778B8874502BE8
:108B20001E25334A6E98AC9E9BBBE0EFDFC9BEA604
:108B300071463E4A6D99BBD8DDC296747FABC4B90D
:108B4000AE9F7444252339628DAAB5B7AA90868C4E
:108B50008D81623D2C3244699198908B79615844A3
:108B600025222F30355380A7BDC4D3E2E3C7A49795
:108B70008D623E435B7DB2D9E8F5F2D4B09CA0AEE5
:108B8000AE9C88807247242844678EABBDC2AC91EE
:108B9000837B746B4B26274A708A928A60432C1A17
:108BA000151D242B426586A6BCC4CED3BF977D7607
:108BB00062433D4F6992C4E3E7E2D5BFAC9D979D08
:108BC000A1937D706248312D47769EB1C2CAB38EA3
:108BD0007B72655B56596F909F968C7C6A4F2D1700
:108BE000161C1E2C4B6685A2B2B8C5CFC19E7E68EE
:108BF00057483D3E5A8DB2C7DCE6D0B1AEB9B8B5E4
:108C0000B2A7927B67564B424A637C8EA4B3B9C32A
:108C1000BC99795E403A5D8DA7AEA99A5A35191371
:108C2000181D2C4D70868E98A5AFB2B09D785D5101
:108C30004B464B6385A2B3C6D2CCBFB6B1AEACA790
:108C4000A9ADA2866B5C50474C678AABC5CDC0AE60
:108C50009F846151618199A8ADA9977E5F3F2317D9
:108C6000161A2C4F708FA8ACA09792897962566221
:108C7000736D67758D9FA39DA6B5AE9A9AADBDC461
:108C8000BCB0A998744E3C3B4151709ABCC3B19D95
:108C90008A68505A738393A4A39173461A1A1C29A5
:108CA0004567889FA3988A745B5457514F67839494
:108CB000A2B0B3A7937C6F76879FB9C7C7C5C0B171
:108CC0009E928D857461514F5A697C8DA3B3A68E97
:108CD0008A938979797F86897C604B3B25192F613E
:108CE0008BADCBD3C1A1744F484134497DACCFE0AB
:108CF000DACCC2A78069656D819BB0C7DACEAB8E36
:108D0000786663696F7A837C695D574F566B829290
:108D100099908486897A6657483F3D394A6786A28A
:108D2000B9C3C5BA9E80624133496F8DB1D6EBECB1
:108D3000D4AD8A82838392ACBCC7C9BBA08A725D62
:108D40005A67738293978F8574563B3237475D74A9
:108D50008A978A6E594B392F2F394F6B8695999E7A
:108D60009F988B8179695B60728698A7B4BBB7A71F
:108D70009695968E92A8B9BFBEB6A18469565159F0
:108D8000616E8295A3A5927A6D6450393644596715
:108D90006F74776C54423D3E4A6C8EA5BFAE9B8B80
:108DA000786659586E95ADB7C4CDC1A4938E909591
:108DB0009BA6B5C2C4B09888786B655F636A6A6821
:108DC0006F7775717884846F5850494240464C499A
:108DD0004343484D596E8AA2AEB8BDB9B1A58E7A4B
:108DE0007A8A9BA0A3B5C9CEC6BEC2C4B09EA4AEAB
:108DF000ACA7A59D8F7F6E605A5F6D777B7B797482
:108E0000695F564D4A505D696B68645E4B2F1C1854
:108E10001F304A6E91A9B1ADA196959BA0ACBDBF84
:108E2000AC9D979A9F9FA4B5C3C7C4C1BAB6B0A55D
:108E30009384786A5A52555E6565666B7279776875
:108E4000554C47423B3945504A3F383435384056F7
:108E50007A9BAFB5B0A89D8D7E809FC6E1E9E5D92C
:108E6000C9B39E91929FB4C7D5D9D4C9B1957E722A
:108E70006E6B6A6E6E685F5A57555651494A4A473B
:108E80003C322A251E1919202638547087949A9846
:108E9000918E89888D9DB4CFDDDEDFDBCECACAC955
:108EA000C3BEC1C5C3BEBAB4A8988D847F78767995
:108EB0007F807A736F6656494239302C2C2A2622DD
:108EC0001C1F242D42617E98A6A5A3988779747AE9
:108ED0008DAECFE8F4F6EAD3C4C1BBB6C2DBE9E796
:108EE000D7C8B9A185706B747A7B7C81847A6E6AED
:108EF000665D5850463E342416120F0B0E131F3475
:108F0000506E88949591897F76706B73859BAEBA0D
:108F1000C3C2B6ADAFB5B4BAC1C7CCC7B4AF9F8FEB
:108F2000868480787172787A797A7E7C716556460B
:108F30003C32261C181512161C29425F7C94A8AFDF
:108F4000A89E8D7B71758192A6B8C2C2BBB3BBC20D
:108F5000BEBEC4C7C3BCAEA39F9D968F8D8B8276C9
:108F6000777D7973767B766F6758463830261E1D7D
:108F70001C1B181B232F43607E95A2A6A394867EFC
:108F80007B838D98A7B0B3B7B6BBC8D0D2D2CFC7BA
:108F9000BFB7A99EA3ABAAA29B90817D8386878D34
:108FA00091887B706452413C3E3E3A31241A181F2E
:108FB0002B456B8FA2A7A5A095877A7A8590989E5E
:108FC000A4A7A6A5AAB3B4B5BABFBEBCBDB9B1AC7F
:108FD000A99F8E847E726C77878D89847A6B5A4FB5
:108FE0004B47464847434241332B2D333E5165762C
:108FF000878E8E8B8C8C84808993999EA6ACADAC29
:10900000AAA9A59995A2AAA6AEB8B4AEA9A7A199F6
:10901000908E8B8585898A84786D645D56565A5DFD
:109020005855524C4845424551626F78858A858033
:109030007D797575787B82919999999B9D9A97977F
:10904000989CA1A2A2A4A7A8A39C9897929093965B
:10905000989691857B746A65666C706F7174726D99
:10906000646568696E75787C7F7D787575747171DB
:109070006D707880808285898D8C8C8E8E8B898DA9
:109080008E8D8D8F909193939090989E9F9D9793A6
:109090008A847E7B7B7D7B7A7B7A7C7A7F878C91CE
:1090A00093928C837B797874706F6D6B6C727A821B
:1090B000888A89878988858180808383838281806B
:1090C0007D7C7E7F7E81818587837C76726B676BFA
:1090D0007274767778757374747880888C909493B2
:1090E0008C86817C7877797A7C838B8E919494922C
:1090F00091929392908E8C8B888684818280807EE0
:109100007D7C7C7A7774706E6D6C6E737471717126
:109110006D6C6C6B7075787E7F81807B7E7E7C7CD5
:109120008184878785848484868A8E908C8C8F8FB7
:109130008E88858787838184898E908D8884827DBF
:10914000787775777D7E80807E7C7A7A7A7B808462
:109150008B8F8F8E8A85807E7D7B7D8085898C8AB2
:109160008B8B8D8A8B8D8D8D8D8C8C8D89847F7E64
:10917000807E7E7F82838382807A7473727173753E
:1091800078797A7975757678797D7E81878A88880D
:1091900088898886858785868A8D8D8E8A8B8D893C
:1091A0008685868687868582807E7D7C78797C7FB1
:1091B00080807C7975746E6C6F7274757472727164
:1091C0006F7071707275787C7E7E7C7D7B7D808413
:1091D0008584838487847F828586888A8B8D8C8B27
:1091E0008C8D8D8C86878A88858283868584818212
:1091F000807D7A797A797C7B7A79777678777576DB
:10920000767574767A7A7B7D80838384888A89896F
:109210008A88888C8887888A8B8A86858A8E8E89B8
:1092200088888582828488898D8D8B87807A7978F9
:109230007B7F848687858381808082848784828304
:10924000827F7E82838388898582838283848484EB
:1092500083817C7A797A7A7B7D80838281817F7F2A
:109260008081807E818385888984808284848382D2
:109270007F808285828282817E7C7E7D7D7C7C82F5
:1092800084868686847F7E7D818484838383817EB9
:109290007B7B7C7E7B7A7B7F7D7D818281818384E9
:1092A000827E7C7B7C7C7B77787B7977767777781E
:1092B00077797A7878787776797A7D8180808587F2
:1092C0008685858382817E7B7A7A7D878F89828776
:1092D0008D898282817C7F88847E8083807B7A8175
:1092E0007C73797E7D7B7C84888685857D777773AA
:1092F0007D8A88837F787981888576717D817F7D7D
:109300007E7F8A918C80797B82868586878A8E96FD
:10931000988C7D7F898D89888C8C8B8C827F848FC3
:10932000969389878E8F8681807F878F897E7B82C7
:1093300088878287857B7F8A877C787F86847C7F0D
:10934000848380808A8C838186858382807D767207
:10935000818F887E8081848885827F7E848E8C81C7
:109360007B7B838686888881818A877F80878684C5
:1093700085878178777D80807D7B7E807E7B767916
:10938000868C857C808D8C807878736B645F5D576C
:109390005762676569767E7D7B7B83868991949130
:1093A000878792968B848080807E7D807D7B7C7F8A
:1093B0007C797672737473706A6C75726B676767A9
:1093C0006A68696D6C6B7276787B7D7F7F73636D85
:1093D000A0BD9F92B8D3C5ADA3A9B09D8F917D6E5E
:1093E0007F8B7D6D64718D8B767782909E9A909144
:1093F0008F8F9DA396827D878D887F6E666B634F6E
:10940000474B5055555458595E6766605E67737593
:1094100070747F8888899092939494949A9E9C9B70
:109420009FA4A09EB0BEA78D9FBDB3A8C4CEAA9E88
:10943000B8C0A68F8B9597806268726466797061F8
:10944000697E8E8B757388928E8678797E78737537
:10945000685960686354474E564D4243494E504FD9
:109460004C55666D696E777775787B797B808685DC
:1094700083858E8E85848D929392969EA3A5A8A7B0
:10948000B0C3C6AB96ABC9BF9D97B0C5BB9C89980E
:10949000B6B8947B8EA093858077777D65655C52A6
:1094A000687D68505C7078725A464D6470644F49AC
:1094B000525E6C6C5C4E5C7B887C66677E8A837ACD
:1094C0006E6A778179726D6E77827965606A787F6E
:1094D0007B747A8B9797959693949FAAA99C97A54E
:1094E000B6B4A49CAEC9BFA0A3C3CBAF989EB4BC76
:1094F000AA9391999C958B827B727176705D59616C
:10950000645D5052646D5F55606F6D5E5D6B726A35
:109510006765625E5D6169675F585E6B66676D7007
:109520007279848788929B9F9B9AA1AAA89C949702
:109530009E9D9387868E938D7F777D82807A7470CF
:10954000737B838C8E8C8D9EB1B7AEA9B0BCBFBA35
:10955000B4ADA6A2A5A2948A8987817B6D6363615D
:109560005B5553555659616767656974776F676ACC
:10957000757E75625C65727068656E7A7D73747FE6
:10958000817E84847E838A8B8A8986878884838986
:109590008C8886898B8B92948C878E9A91858897FC
:1095A0009A8E837E818E948E827D85979B8B808917
:1095B00098A1A49889848C97948070788786766A1D
:1095C000676B73736C65646D7B7A6B6D808F8F874F
:1095D0007C828E8F88827A757F8985776E7481818F
:1095E000776E6E79817D736868747C7C736F778029
:1095F00083817B747779787E83766B747E7D776DDB
:109600006D767B787677797B7F818183838386898A
:109610008C9294909194969E9F939199988F87881D
:109620008B8A8686827D828A8D8882838D948F87BD
:10963000888B8D8A7F7C828483827E78787F82810A
:10964000797378807B737475787D7B7573717079AD
:109650007A6D6A71777A79737375787B776F6E77C5
:109660007B7B746D717A7B7A7A78777C7E7E7B7B6C
:109670007C7E807E818686868C919295969391934E
:1096800091929291909395979693979D9D9A989584
:10969000929292928D898B8D8C8783838F8C83811C
:1096A00084898A857E7F84838787827D818487827F
:1096B0007A74767A766F6E6F72727271717271737C
:1096C00074706E6D747A7B79777C8284817E7E8102
:1096D00081807F7B79777979797776787675787EEE
:1096E0007D76757A7D7D7A797E8484858380838A90
:1096F0008C8987898988858381828889837E7E8217
:1097000087827A777C7F7E7A76787C7E81807B7A8E
:109710007F84827E7F83898B878182868684818213
:1097200084848383827E7D81838382828486848312
:1097300084828281838487838186888683818587EA
:109740008481807F7C7C7B7C7A76787B7B7B7C7E53
:109750008082817E80817E7E7F807E7E8384817D0B
:109760007D808183828081858C8C878B9192909380
:10977000918E8F8E8E8F8F8D8A8A87827E7D7D805F
:10978000827E7C81827D7A7F827D79797E7D7A7A04
:109790007C7E7F7F7E80817F7E81817D797B7B79EE
:1097A0007B7F838080828183848485848282828699
:1097B00086837E7E7F7E7F8283817F7E7F7F7D7DAD
:1097C0007D7E7E7B7B7D7F7E7D7D7C7B7E7E8081C2
:1097D0007E7D81838284888584868988848384874A
:1097E00086807E7F7C7D7E7D79777B7D7E7C7D7EA5
:1097F000817E7A7C817F828B888281878D908B8627
:1098000088898987858A928971697E918C7B736C3E
:109810006A73797B7D7B7981857B7F8F7F7C787292
:10982000787F786F6F767879797C8285838181857E
:10983000837E838477768C9689868E969C91828BA4
:109840009C93828B9C9790949290958D80878F8625
:1098500086938D77758D97837A868D877968738ED9
:1098600083657083787D8E847178878E8B837C7C12
:109870007D868B7B6C777F757275706E716C717A7B
:109880006863858B707995938A878490A094848A85
:109890009493919197938E948D87949777909784D2
:1098A0007A7F8A8A7E7A81847879878776768179C9
:1098B0006A70807D6D6574847D7272797D75757E48
:1098C0007B7173787C8383797A84858488877D7FB4
:1098D00087847F796D71807C74746E748369567926
:1098E000846670887F7A888782827A7A888776769B
:1098F0007F7B858F6F6592A58E8A969BA19A8B88B8
:10990000817B88897577817C77756E707A756B6CD1
:10991000717A7D6B5F7282736F7E7A7B857D7F89C2
:109920008B807278827A726E6B6F726F69676C70FF
:1099300072756E6E7E7D778A91868B91909A9A99D8
:10994000A6A8A3ACAB9EA7B3A79EA5A39DA8AA91CA
:109950008EABAF9F9EA09FA098897C7374766A5B44
:1099600060645E5B5E605E5A5B60616774726667CE
:10997000757D7971727B84827D7A7B80867D6C7146
:1099800081745E626E6D665F5F696E68676C727E21
:109990007D7079888685898C99A69C91A4A8A6A0BB
:1099A0009EA7B5B3AAA9B8BCA6A1B9C3ABA5B9BFB8
:1099B000B7B7B4A59EA4A08C7C80837463626663F1
:1099C0005D5F584C505C564344585B48455359536F
:1099D0005862615F676E6A676E797A706A747B73CA
:1099E0006B6E6B6F7C7B6F6F79766F7581867C7524
:1099F0007E8A898C9492959A959EA4999DB4B1A7DC
:109A0000B4BFBDBAB9C0C6B7ADB8BFB6A7ACC1BECA
:109A1000AAACADA1A2A4928180817866615F575300
:109A20004C4745494B413F484B41415052474857AD
:109A30005F5B6264606C7568667C827C77757B8135
:109A40007B7578737B877A6B7880797D8482808060
:109A5000797A83898C8C8D9199A19D939AA0A1A4E8
:109A60009D95A7B5A498A4B8B9A59CAFB7B1ADAB67
:109A7000A5ABB0A1878591887574736A67655D59D8
:109A80005C605B514B4A4A48494A4A4E504B505FD2
:109A90005E58657577737882827B7A7E7D7E787575
:109AA0007C7E7B787C81847D7981858080858787B9
:109AB000878A8A8489948D87939C9B9B9997959F8D
:109AC000ADA69A9FAAA9A8A3A2ACB0A8ABACABAF15
:109AD000AC9A949690857F7E7F7D777475736B6367
:109AE0005D5F63625C585B615B555A666964667270
:109AF000737276797C848172758683767B807D7DB6
:109B00007F756E828D77768D8E84837F808888873F
:109B10008379848F85899D978998A099A0A3A6A30E
:109B20009DA0A1999CA29A9CABA69496A5A0989A58
:109B30009793958A7A72797B6F656A6A605F584AF3
:109B4000555F4E485450474D4E4C545A54546067DC
:109B5000656F7972737D7A7781807A8288837F815D
:109B6000848987878C87858A88848585808283829B
:109B700082868688878A8D898C979792979FA09FE7
:109B80009E9DA2A5A1A0A2A5A9A49D9FA29B979ED0
:109B9000A19D988F8C92948B837F7B746D635F60A3
:109BA0005B565A5E59555455585C5E60605F6167FC
:109BB0006C6B6E747A7C7E83878D9295999B989955
:109BC0009B9A989798928C898B8B888481808388C4
:109BD000858285858283807D82827C7E8785818562
:109BE0008A8D908D8A9298989A8F8493A09A97954F
:109BF000939694908F8D8887837D7D7E7772706F2A
:109C00006B66615D60635B5858555B5F5858616176
:109C100062696A68707572777E7F82858688898EB0
:109C20009089898B8B8D8E8B8987878581818789A8
:109C300084858886818384838384807D80828182F9
:109C400086848386888A8A8787898A8B8B898B8E8C
:109C50008D88868C8D8A898A8D8F8A828184838182
:109C6000807E7B7C7E77777B7A767675747375726F
:109C700070747876757578777A7D7A7B7D7E808052
:109C80008383808082838281807E7F7D7D818181CC
:109C9000858B8E918E8D908C898E8E8B8E8A888B03
:109CA0008C8D8F8F908E8B8989898989888C8E8AFB
:109CB00087888C8B8885848282848281808282825C
:109CC000817E7C80807E7C7A7B7D7C7D807D787BC4
:109CD0007C7A797976777B7F7D7D7F7C7D7D7B7CCF
:109CE0007C7B7F837F7B7E7F80807E7A7C7F7C7B9A
:109CF0007B7D82837F7D7F7E7D7E7E7D7F7C7A7B88
:109D00007C80807C7D7E7F807F7E7E7C7D7E80846B
:109D1000837F8283838385838282817D7B80818030
:109D20008283828080807F7F7E7F8080807D797843
:109D3000797976797B7D7A77777A7A797879777895
:109D40007D7D797A7B797B7D7F807F8081807E813C
:109D500085898A87888A89888887878988868A8E7C
:109D6000908F8D8B8A86878A8A898C8E8C8D8D8C3C
:109D70008D8F8F8D8D90908C8B8B8D908F8E8E8E06
:109D80008784888D8985848787868380808586827D
:109D90007D7C8388847F8184827F7B787A787575E7
:109DA000736F6E70727373777976797C7C7D807E49
:109DB0007E8284817F7E7F8181838586868686827E
:109DC0007E7E7D8081807E8182818180808084858D
:109DD000817F7F8081818082838280838582848568
:109DE000848589867F7A7B818685827F8188847E4F
:109DF0007D7F7C7C7D7D7A7A7978767572757C7AC8
:109E000078797B7876797B7D7B76777E7E7A797BB5
:109E10007C7E7C7C7F7A797F817E82817F81807E5F
:109E20007F7E7C7B7B7B7A7A797A7B7B7D7E7C7F75
:109E3000868D8B888A8B8A89888990918C8B908F6C
:109E40008A898B8D89898C8E8C888583848584838F
:109E50008687888582827F7F838282817F828381D9
:109E60007A798490836C738F97897879858E8874DA
:109E7000748C856177AFA1645682BAC79D66629281
:109E8000C1B77E546192A57A505F91A7875B69A69E
:109E9000B0867691998085ABA9786F946A464F7A9F
:109EA0008A6749678F8B73697382878B8A796A7136
:109EB0007664586983938F786065839286787C99FD
:109EC000B6B29B8282A0AB9090B1A87C7AABBD99D0
:109ED0007880A1BEC6A1695A80A79B695378A093D8
:109EE0006859799F9670708B91847A6B4E3E5A7741
:109EF000633C33547E764F598897806B6A706A5FF3
:109F000066726A6572776860728B9176586697AEF2
:109F10008D65688BA29E90847C75819F826D8396EF
:109F20009298957D7581858A8E79738F9B938D80AC
:109F30007C8587878E8876797F7A85969791989B9E
:109F40009696A5A083777D838367495A756E645C76
:109F50005B768E8B817980999B745A7399977E83F7
:109F6000998C7786978A756F778379666C766A5E47
:109F70006D7E725D565D6864584A3439729C80719A
:109F80009FC4C1BAAB8E6E4B31353C39393A4A85E4
:109F9000BDB7A2C1F0EFC7A8B0CFCAA28A786A7FC6
:109FA000A1A58C849CB9CBD3C6A9978D827C6A511C
:109FB0004F55483941648B8E6F4F3F40526F837CC1
:109FC0005F45382D32598A97836C6162697697C7ED
:109FD000DFC49B97B9CDCDCDBD98818E9F91717116
:109FE0008C96898796A1A0969BAAAC938082837653
:109FF00077847A574C6B8B826B5E585143353E5059
:10A000005958524F57636C736C59618A997F6A70C3
:10A010008EB1BAA3877B84A6AD88788C8A8E86861B
:10A020008D8189A7A5ADCBC1977E6C616A72808C4A
:10A0300080717B8FAAC7D6CEAC75515B727F898F3A
:10A04000887B727995B5B39D978F7D7A7A6B5848E6
:10A050003C3B4956616E7B7B7572717276818F9342
:10A06000867A736C7D9BAAA99F8F878C7C6874838A
:10A070007C7986877768728CA3AEAC9A81747D8C6C
:10A0800090868593A3AAA5937E6E5E596058453647
:10A090003141566381A8AFADB8B8A694747C76718F
:10A0A0007F8C8984797691A2938682796551454B1C
:10A0B0005D656A76776567899B947E675C554D5CC4
:10A0C000777B79756A66717E867F645675B5E9F02F
:10A0D000DBCBB8936955595B5350576E94BBDAF498
:10A0E000FBEDD3B99F774F3C404D617DA7CED4C3E4
:10A0F000B0A59C826A6058463C393F536C7F87828A
:10A1000082837769605D66777C6A523C313F72AAD0
:10A11000C1BBAA9272492D36515A5863A7D1EDFCA2
:10A12000FEF4DBBA93684D4E5A739EBAC3D5E4DC95
:10A13000C8AE8E6E4E2A1E3350656665728A9DA526
:10A14000ABB4BDA4725A5A544E504729151B3867F8
:10A1500096AAA1907B552A171F2D3D516891C1E405
:10A16000F2F7F2DFC19766413B486290C6E2DDCC70
:10A17000BCA57C4E3C474F484A6F97957C798F9F92
:10A180009999B1CAC3A1837F7B6654482E181F3E9C
:10A1900073A4B4A89A8963331C2337477198C5E91F
:10A1A000F7F8F0D9B3865432313D5381B6D5E1DDAD
:10A1B000CCB0855533315885887773776A585E7C83
:10A1C000959CA4BAC9B89D908E7D5B402A1C284CF2
:10A1D00080B0C5BDB0946543353F63776F7082989A
:10A1E000C5F2FAF3ECD0A475472D384D5C7DAFD4A1
:10A1F000D8C8B9A1703E283158879C93866F4D3BD3
:10A200003D4F7295ACC1CFB28380A4B8AE885C3AA2
:10A21000345891B9C4B2957652342D4373696E990E
:10A22000CCE9EDDBC0A38055322538567192B5C319
:10A23000B6A48B63371D1C2D598697968C704D3FA5
:10A24000434E6182AED7D9AC8A9EC0BC956D59632E
:10A2500088BAD7D6C4A67B5039363F48566D92C3CC
:10A26000E7EDE1CDAE8E6E4B353140658BA2AEB7DA
:10A27000B59D7D5F3B20243E69969A84807D5A3A45
:10A280003C566A697199C7C2947F939B7E6A89C064
:10A29000D8C1A6A49B7751536B66473E82A9C9D803
:10A2A000D2B382616F84724D4F7C9C959AB9B68708
:10A2B00056425B7E7A7292B7AF827394A2784B4C0F
:10A2C00062645C70A3C8C295635372A0B7A79185FE
:10A2D0006D585353462F1E274D7BA1BAC2B99F78A4
:10A2E00049344E6452425584BFE2E3CBA57B5340D0
:10A2F0004C6F848998BBD4D1BAA8A29D8C6C4F496D
:10A300004A485E828B8DACCED4B17B607397B3B874
:10A31000965A3534486998B7BDB0936A3E3F434278
:10A320003A405C8CBFD6CFBA936445465F6B5B46C0
:10A330004A6A9DC8D6CDAD7951507B9B86655E58E3
:10A340005882B3BB957589AEAF907F6E47272B4A75
:10A3500079A7CAD9D8C9AD91704422171C273C6A85
:10A36000A9DBD3AFAEBFB69F95815534325385A4D8
:10A37000ABAEAB8D798DA8A27F6861596595BFBFE3
:10A3800095635F8BB0AA937850282341607DA6CB5C
:10A39000D8CAAB825C4E564B281E3C6AA0896E6BB5
:10A3A00083A5BFB2804E3C4E79A6C3BEA275566D42
:10A3B000A3B89A737CA6AD88819C93675B83ABA29C
:10A3C000754838465567879692A9DAF5F0D9B48D65
:10A3D00083907F503D5684A9A17059605C6B9FC0EB
:10A3E000B285606A98B8A879606B859DA992635020
:10A3F0006C9CBFB4826680ADBDAC896959576A7BDD
:10A400006330141F395C7A8D9BB2C1B093846F4363
:10A41000304B80A497664A546EA1CCB9778DB7DAD9
:10A42000D0A79BA7AEAD9C754B3A4F7F9F906755C9
:10A430006D90977F6866624F516B755D49526A6D8A
:10A440006051433D4D7183755541567C867D8CAE80
:10A45000BAAA9A9DA49269535F85AEB8A193A9D177
:10A46000E5DBC0A99891979C8E6341466C8F9480E0
:10A470006A6C786C52526F7F79706D798B8F8D8D8D
:10A480007D5D463B3640678D9CA1B1BAB6B2AFA1A7
:10A490008A6E647A949A948B8A96ADC3C8A3857E9B
:10A4A000828D9DA190674A567C9BA59682808D8E59
:10A4B00076595365767D8590907C707475695034BB
:10A4C000374D4E3F4B6F96B1B8AF9D7F5D45435BB7
:10A4D00089B5BF9C7B87AECED3B28B7B79819192BD
:10A4E0007D584359829A91755B627E8779614D4AA6
:10A4F000566F909E8E8794A29A7F615660686661BF
:10A500006C849BB0B69F81726A665B4848607175C7
:10A510007F93ACBAB19B8D858177675855647782FC
:10A52000817B73798DA09A7F66646566758E938C46
:10A530008C9092989DA0A29C89756D6C7492BCD9E8
:10A54000D4B39DA2A8947B7685929193A1A79FA74F
:10A55000BED1CCAC8268656865666F7E8075707BA5
:10A56000887F6E615C554B464A54595B67716A65DA
:10A570006E818F89726D859DA2998C8690A5B4B7E6
:10A58000AE9D8C8A939D957E778FA2A2AAC3D1C8D7
:10A59000B19A918977696A79837D68606D76888FD1
:10A5A000867367635C4D4B607576665C5D6059567B
:10A5B0006A817C6A657285919C9B8F7C6F7690A185
:10A5C00098846F6B7683828187909791867E7C7A60
:10A5D0007D82888E897971736F737F7E756F7585C3
:10A5E0008E81675656678BABAE9B7E605B74919C89
:10A5F000917D71788995938E90938E8783796C6520
:10A60000707C807E828C959185776A686C79848471
:10A610007B76726D74859089705A61828A725E59F8
:10A620006A8BA9B3A28A7D82909D9C907E737A8E5C
:10A63000A5B1AFA193929B9FA099887873737883FB
:10A640008C92938C7D74778084827A757267606B4C
:10A650007A7F77686A809392806F6153576B828CA0
:10A6600086756D788590938A7A6B6D7E91938D8DCA
:10A670008F9A9F938687898E95938C8A8D8F8982F6
:10A680007D7A7C86969A8F807977777E8479665BEF
:10A690005D75959F91857F7A7775746F68778485EE
:10A6A0007C757172747A858C8C837D7F85827874D9
:10A6B0007A84847E7975787E8589847B7C8797A16E
:10A6C00098857E868C8D8C8E86756769788690934A
:10A6D0008D847D7C848984786F707474757A7C76BF
:10A6E0007578767176818D938C7E7168646A7685D3
:10A6F0008E8D8D8C85776B676F7E909A9B948F8FF4
:10A700008E8E8B837A72747B828A91989A9C9994AC
:10A710008E867F8B906F618FB49578867C7D8981E2
:10A7200089A6A893908B664B667B5444789A89835C
:10A730008C88705F635E4F606452647E7165697C73
:10A740008D79667E8776737694B598778A9891919D
:10A75000868DA8997C878F8682847D645F84917DB5
:10A760008EA27F6E8D95858078789495665079A1BC
:10A770008B6E8291818A9B837686878DB6C9996913
:10A780007FA088779EBDAB97A5A98C756D575E7924
:10A790006D5D72908E6653829E785E6C855E4775A5
:10A7A0009078758A92866259717269746F69788738
:10A7B0009B99716F8F7F6E8C907061718E978A9468
:10A7C000A49D9B9C9499A093929374657C7F7786BB
:10A7D0009181778092A1A496847C7A77717687960E
:10A7E00089798DA7987A6E6F716A6876807F818289
:10A7F00087918B7F775C4F616A626D8187878E97C7
:10A800008C73718584797C78666169706854566D43
:10A8100079838A776F8892837F878573757C7A9036
:10A82000A28E807C6F6B798A8D82808B8A8A8F7DE5
:10A830006870765C465781A1AAACA9928999906507
:10A84000381C17314C566678869FB6B8A183706A5B
:10A850006B706A595E7583837D80919FA0A6AA98CC
:10A860008B8B8C7D675B61656172887D67647085A9
:10A8700086706263666B727B7F78717C827C787590
:10A880006F62536188B6E5FCE5CBD0CDB29E856C96
:10A890005F47313B5C8CCDF8F6DDC7C2AE8D6949B0
:10A8A000465B7CA1B5B0A6A4ADBDC4B19A88715D6C
:10A8B000584D302031464D514E494F5D66614E3DF9
:10A8C00032364C605E56575A6D929A837E8E9395BF
:10A8D000A3A48E83909DAAC1D2D2C6B9BCC4BBA783
:10A8E0009DA3B5C3D3E2D4AE9DA8B3B1A492888C86
:10A8F00098A6B2B8B0A49D8E7A7577736F72746D96
:10A9000060575A60625B4E433D3D40444847423A7F
:10A91000363943463F312F3F4E555D5F6A736E6A4D
:10A920006B6B65667783868B8F90949F9D9B9B9BBB
:10A930009FAFB9B9C6D9DDD1C9CDD3C9C2C3BFB3E1
:10A94000ACADB1A797939082869CAFBABFB4ABA5CC
:10A95000906D4F414442383D494B4F575A5544330F
:10A96000261F1B1811121A212A43544E52616E8061
:10A970008D9292897E81837266717F8F96999C9C5D
:10A98000A1A5A0999CA0A3A89B8E939899A7B0ACD1
:10A99000A9A59B908D8F9AA7B0ABA0A5C2C1BFB649
:10A9A000AEAEACA29A9289847E7C8597A49F948F48
:10A9B000928D7C5F4237393526212C3C516163638F
:10A9C000696C6E6959494457707A7C82827C7B79C4
:10A9D0007C8B9BA4ADADA096877366656A75818AF2
:10A9E0008E939491908E8C8885808185898D9596A3
:10A9F0009189817D7D7E7D7F8891989FA8AEB3B53A
:10AA0000B6B8B4ACA9AFB2A89387898B847C7C8993
:10AA10009FACA894847D6F5D4F463F3B3A35394EDD
:10AA2000657073726A5F56514C4E5357606D757BFB
:10AA30007C7A777B828F9EA29E9B91806E656369F4
:10AA40006E6C727B8084817D7C7D77716F6E6762B6
:10AA500060666E76838E8F8E8579767F868D959BE8
:10AA60009FAAB8C7D0D2CECFD8D7C9B8ABA29B9532
:10AA700095A9C9D6D3CECECDBD9F81654A342115C7
:10AA80001721334D6A83989D9489745233201B2378
:10AA9000324660737C8084858685817C6B686865BE
:10AAA000625D5C605E5D615D595B616E7F8A8E9503
:10AAB0009B9A96918F8F8E8F9498999C9A9CA4AB19
:10AAC000B3BBC1CAD6E0E9E7DAD6DAD1C4BCB5B4C3
:10AAD000B3AA9E999DA9AEA8A19B94887565625959
:10AAE0004A3C35373933323C4343413F403F3C3A9F
:10AAF0003A454C4742474C4E50586A7981807C7C9D
:10AB00007E7D7B7B788188878B92948D8882807F05
:10AB10007A75716E6F767D838888868685878C8F3F
:10AB20009094989FA9ACB1BAC0C4C9CACDD6D3CBB2
:10AB3000C5C6C3C1BCB4AFACA39B95908F87786CDE
:10AB4000645A5249403E3D3A3C424644403D4245AB
:10AB50004344454C53565A62696C6D6F71787B81E2
:10AB600086878281807F7D7F81828586898B8E8E9C
:10AB70008C8E9294928F8E8F8F8984858689898816
:10AB800089898B8F949A9A979293979CA8B1B9BF11
:10AB9000C4C4C1C0C0BAB9BBB8B3B1AC9E98979891
:10ABA000948B83796E675C534B433D39363436352D
:10ABB000323236363437393D4144484E5150535A7B
:10ABC0005F6A74777A7C7F7E7B797C7D80878D92CB
:10ABD0009497999CA0A1A3A6A7A39F9C98959290B7
:10ABE0008D8E8F8F939A9FA09FA1A09D9A979695E7
:10ABF000969599A2ABB2B4B4B0ADACB0B2B4B5B4A2
:10AC0000AEA7A2A0A09F9D9992867E766A5F5652BB
:10AC10004D464444433F3D40424446454440424BF8
:10AC2000515760697173757674767A777273717142
:10AC300073767A7E7F81888C8D8C8B8989898987D0
:10AC400085878D8F929AA1A2A3A6A5A4A5A7A5A248
:10AC5000A1A4A9AFB5B7B4B1AEACAEB3B5B7BCBFE4
:10AC6000BDB8B7B4AFA89F948B857F7C786E6C69B4
:10AC7000625D5E5B565049443F3C3F42413F40422B
:10AC8000454A4F51555E6364646B6F6E7073716FAC
:10AC900070717374737170747674797C7E7E808544
:10ACA00088888889898B8B898B929B9FA4AAAFB057
:10ACB000AEB0B0ACADACAAACB0B0B2B4B5B4B3B099
:10ACC000B7BAB3AAA198928E88827D7874716C64A9
:10ACD000625F59544942403D393A3A393B3D3E3F23
:10ACE000424446494B48494E535A606A73798288B8
:10ACF0008A8C8B8D91918F8D8B8D8F90919497975E
:10AD000096979390909294929196999C9EA2A3A7C5
:10AD1000AEB4B8BBBEBEBFBEBAB6BABEC1C6C8C767
:10AD2000C3C0BBB1A79E90857D7978777373736C30
:10AD3000655F5A514C46403F3B393B3E3E3F43489E
:10AD40004B51575C5E5F5F61646869696C70757ACE
:10AD50007F858B8B85818183878885848383858BA1
:10AD60008F8E8F979C9FA2A4A19E9A999694969C51
:10AD70009F9FA2A3A3A4A3A4A3A4A3A4A6A9ADAE8A
:10AD8000AEAAA8A49C969088817D7A76726D69653A
:10AD900058473D3B38363B43495259576162615DE4
:10ADA000544C4949505E65676360606160657073CB
:10ADB0007479787A818B8E8B898784848993989A29
:10ADC000A5A9A8A697848D999C9EA1A2A1988E88DA
:10ADD0007F8396A2AEC4D6DCDED7C7B4A08D7966D9
:10ADE0005E5C575861646A767B79787468605F69E5
:10ADF0007586959FA6A59F9B9895918E8E8A837B3D
:10AE00006E5B412B1A110E111621354F646D6E7059
:10AE10007A7F81858D9BACB8BDBCB8B294858386A2
:10AE20008D97A2A4A3AAB1BDD2E4F2FBFFFBF1DE91
:10AE3000C7AE8F6D564841434D58636C767D7E7E1C
:10AE40007873767E8894A7B3BDC1BDB6ADA8A19B2B
:10AE500093877962483114023A968622011F2D3A6F
:10AE60004E56565755586067788FA3AFB4B2A7981F
:10AE700086766B6B6D757D879BB2C5D7E3E3E1DDAD
:10AE8000D4BFA9958272645953565E67717F909EB4
:10AE9000A2A5A7A39F9EA0A7AFB9BFC0BCB7B1ABE7
:10AEA000A49B8F7B634A2E190C06040A11192632C3
:10AEB0003C43444443414046526577899CA8A9AA33
:10AEC000A4988B7F7A8293ACC3D2D9DACEB8A0880B
:10AED000776C5F5656596169738194A4B0BBC8CE34
:10AEE000D0D4D4D5D4CDC4C4C2B9B4B2B1B1ABA25C
:10AEF0009788755C42302622252D3A464E4C463FB7
:10AF0000362A201B1A21303D495C686B70757981A7
:10AF100091A7BECEDBE0D7C8B8A38B74534F525471
:10AF2000565B62686E76808F9DA9B3BBC5C5C3C5ED
:10AF3000C4C2BFBEBEBEB9B0A69F92806E6056505E
:10AF40004D51545B605E5A5448393029252A333BB1
:10AF5000455360676C6B67656469778BA0B4C2C941
:10AF6000C3B6A68F7D6E5D50515C6372879096A1CB
:10AF7000A39FA8AFACACB4B7B2AEA89E9C98989F64
:10AF8000AFBDC6C9C9C3BBB09F8F84786E66635C12
:10AF90004F4537281D181517212E435E8A9CA8A0FF
:10AFA00091847A727178848F948F887D6F635B55FA
:10AFB00056626D788B9CA2A6AAAAA8A49F98969484
:10AFC0008A81868E8D8B8E919FAFBECFD9DAD6CFF8
:10AFD000C5BDB3A39385776960574F49423B3A3E5D
:10AFE000404855606F828D959A99948879695D5231
:10AFF0004541434D58667687949CA2A4A29C9183B8
:10B0000076695D5252555A64727B858E908F90920C
:10B010009196A0AAB1B4B7B5B4B0ACA9A9A5A299AC
:10B020008D7F6E5D51484342464E5A6671797D80F0
:10B030008283807D797876777676736F6C625C5ADE
:10B04000565456575B6D818E9EAFB6B9BAB19E8F7E
:10B050007D695B4D42404248566C8AA2B6C8D4D73F
:10B06000D3C9B9ADA0958D8C9093939192969492FB
:10B070008E8784817B706A645C575C626D7B81899A
:10B08000918D867B6C5D554E4952606A747F8485D4
:10B09000827E7C7E81888F92908D87888F8C8C8F2A
:10B0A0008F8A83776A666157555E6C8198B4D3E85E
:10B0B000F0EFE5D8C7AD917E6F6464697079868ED4
:10B0C00098A2A6A4A6A49E9387766150453A363AE4
:10B0D000414855656F767A7A78746E6E72787C83A3
:10B0E0008C90908D84786E665F5D5D5C62676A733C
:10B0F0007A7D8494A7B7C5CDCECCC7B6A18C78672E
:10B100005C565C6D8195ADBFCBCEC7B9A8938172FB
:10B110006461646B73787A77736D67615E63656C85
:10B120007172726C665F59555156595B5F656B71F0
:10B13000777A7D7C7A76736B645F5C5A5E666C7836
:10B1400087959FA8A8A8AEAFA9A6A3A3ABAFACAEA6
:10B15000B1AEAFACA39B948D837B75777E838B98C8
:10B16000A3ABACA49C9183756D696A72787C828272
:10B170007B706B635D5855545452514F4E5051542F
:10B18000585E5F5E60626973787B848D8D8D8A8482
:10B1900083838382848A939BA2A8AEB3B7B3B1B0F2
:10B1A000AAA7A49990919594989B9C9EA29F9892EF
:10B1B0008B837E7C797E8485898B90938D83817F40
:10B1C0007B7167615D5957555253575A5E6363648B
:10B1D00064605A565351535459636C79868F99A2BF
:10B1E000A7A9AAA59F9D948C898683838484878937
:10B1F0008E91959496999C9C9998958B8585858A36
:10B200008F929493928E888A8A837F8182818588A7
:10B210008E94989796938E8880776E6357565B5E70
:10B2200064686C707473706C6A6764636164676A85
:10B23000727E848B919496928E8A827C76737275DC
:10B2400078818A8F959A9B9B9B9C9A9694949697CB
:10B250009B9E9F9FA2A1A0A2A09A96928C88868472
:10B260007F80807D7D7B7775777A7D808386848201
:10B270007E7A76757676787979797673737271736A
:10B2800076797B7C7F7F7E807F7E7D808281817FDF
:10B290007B74706F6B6D707375797C7E7E7E83823C
:10B2A00082858585878786878684807F7F7C7E7D73
:10B2B0007B7A7A7D7F82878A8E908E8C86817E7C57
:10B2C0007B78797D818487898D8D8C8B8C8A898729
:10B2D000837D79797A78787A7C7F818483827F7C98
:10B2E0007B808385888B8D8C8984807E7D7B7A7939
:10B2F000797C7F80808383838381807F7E7B7A7863
:10B3000074747270727170717474767C7F7F8286CF
:10B310008889898785868583817F7E7D7978777C1A
:10B32000808085888A8C89858281838385878A8BC2
:10B330008B88868583828184878A9195989D9B9945
:10B340009994908C8784807D7B78777A7A7A7B7EDB
:10B3500081818180808381848483838181817F7FD7
:10B36000808282828282807E7E7F80808282807DD7
:10B370007A7874717276777B7D8184858785868300
:10B3800083858587898A8B8E8E8D8A8B8986858633
:10B39000868484827E7E7E7E7F7F7F828384838399
:10B3A00084868887898B8B8A86848482807F7D7E51
:10B3B0007F828384827D7E7F7D7C797976747371D0
:10B3C0006E6C6B6B6D6F71767B7D7F82868A8F91E1
:10B3D00092918C8A86807E79757575767778787B80
:10B3E0007B7D7E7E7F808384868685848381838344
:10B3F0008686858586868484858686898A898A89E3
:10B400008784817E7D7C7A7A797878787978797A80
:10B410007D7F7F838685868989898A8A86878885D4
:10B4200082838686868683817E7D7A777879777730
:10B4300079797B7B7A7B7A7B7C7D7F818283838435
:10B44000848484828282828282817F7D7B7A7A79FF
:10B450007A7B7C7D7E7C7C7C7D80818486888A8BE7
:10B460008B888887858280807E7E7E7D7D7D7E7FC5
:10B47000818080818382828585827F80807F7F7CBE
:10B480007B7B7A79797B78777C7E7D7F82838789E5
:10B4900087868586888684817E7C7B7B7C7B797AA7
:10B4A0007A7A7B7C7D8084878B8B8A8A858684826E
:10B4B000807F807F81818182818183838385878A68
:10B4C0008C8D8F8E8D8A898887848381808082830A
:10B4D0008486878A8E8D8C8D8D8C898C8C8B8784CD
:10B4E000817F8080807F7F7E81817F7F7E7D7B7E6C
:10B4F0007F8182828584878A8A8583838688847E09
:10B500007F878985828185898780818B8C7E778101
:10B510008D897E79848F847B84857F857773777A24
:10B520007D7D7B787A828887827E797B807F7B773E
:10B53000777772727982868585898E8F8B84838EE8
:10B54000908274727E86857F7E7B7A87928F8A89CD
:10B550008E938F86838B8D867F7F81827E7D848D87
:10B560008C807C88928B7A798A8D7F7578807C74C8
:10B5700074767677787C786D68717E82796A687384
:10B580007D7D78716D6E747B7B777672777D7A784E
:10B5900078797E888B837C7C8594978C888E908D3F
:10B5A0008989857F818589898280827F7E85857C66
:10B5B00073737A7E7C78746C6D7879747474747C2F
:10B5C000837D797E8188877F7D848784838080895D
:10B5D000928F807A83939C8E7774868D8783817A0D
:10B5E000777C81858076777F8281796F727D7C77A9
:10B5F0007A7C7B7E8081827F7E85847D7F898C873B
:10B600008180868D8E887F7677808D8D7B67739322
:10B610009A8572708190896E5D6C7D7557596571E0
:10B62000736F6F6E768B95887B89A2A6928999B08D
:10B63000B4A69899A4A6A194898A8F8C82797078EF
:10B640008785756C76877F6E6F766F61585656501A
:10B650004649504743556059576371747783949CAA
:10B66000999CACC2C4B6B3C1D2D5C8BFBFC3C7BE14
:10B67000ADA3A19D959497978B869499887B828999
:10B680007F6C5F635E5046433E3D3E3C38322C3219
:10B69000404747465168766E738EA4A6ACC6D1CE9D
:10B6A000D1D7DEE3DDD0CFC6BCBBB1A6A0999398BD
:10B6B0009C8E84888C877C757366585450453A3AC2
:10B6C0003A37353534383E3D404548556562647DEE
:10B6D000949496A6B9C1C3CCD8DADAD9D6CECCC761
:10B6E000BDAEA2A09C908D90867D84887B746F6592
:10B6F0005E574F4636323933262C34312D363D3E97
:10B700003D40444D56606D78777890A7ABAEB9C395
:10B71000CCD2D0C9C1C7CEBEABAAA99EA5998689F5
:10B72000918C7D74726F655B585448474A433F4221
:10B73000424244444345494C4F51555E666A6F78D6
:10B740008590969DA9B6B9BCC4C5C2C2C6C0B7B9DA
:10B75000B7ACA2A7AD9C909693857E7C746961621C
:10B7600062554F5550495359505256595E6368655A
:10B77000606A78776E7689919396A3B0B5BABDBDAD
:10B78000C1C6C3C1BEB8BCB9A9A2AFB3A69A9898A6
:10B7900091867E7F776662645C56554C4F55515159
:10B7A000585A565A645E576474706C778A969196AC
:10B7B000A39893AABBB4B4BABCBCB5ACAAADB0AAAA
:10B7C0009697ABA4898996978A7B7575695E615A4D
:10B7D0004B4C4D48484541464543474E5654515CB5
:10B7E0006E6E6A76848C8B8A97A4ABAFADA8B1B924
:10B7F000B1A6AAACABACA89899ADAB928D999C922E
:10B80000857D7B756F6A5C4F545F5647455455493B
:10B8100048535A5D5B5B67726C6B7580898A939D38
:10B82000A09F9C9BA2A8A396979D9790938F858E8F
:10B830009A8D7F86908C7E737377726A5D5558619E
:10B840005B4C4E5D66605A5B6773736A6C7A848486
:10B850007F8498A39C9CA9B3B1B1AEB2BAB3A5A49E
:10B86000ACA99E9596998B8391907F828C887F78E6
:10B87000767D7865656D6C64605F63625F645F5C54
:10B8800069736966768685797F98A59F9CA5B3BB09
:10B89000B6B2B6BABDB9ABA1A7ACA08F9695807869
:10B8A00085847B7C7B7777726F6E5E5765614F54C2
:10B8B000615D5756595E5B5763696567777E777B35
:10B8C0008F9A9595A0ABAEA4A4B1B2B1B5ADA1A32A
:10B8D000A69B8E8587867772797B736D70746D6693
:10B8E0006F73675F5F605D5856585453585A595D7F
:10B8F000666A6867747D7B7A86959A979BA9B2ABD6
:10B90000ADB8BBB7B6B1A8A9A8A19B918C8C88761D
:10B910006D727A77665C6A7A76675F6C6A564A55AA
:10B92000605A4D4E565B5C5359686B6A757B7A88DA
:10B93000979B9A9CAAB8B5B0BAC1BFB8B3B7B7A81D
:10B94000A19F9794928A83817C79786C686F7370D9
:10B95000675F67726B61636A6F6A5F5D616564618F
:10B960005F6165686B6F7A7F7D82919E9F9BA0B0BF
:10B97000B9B1A9ACB9BBB0A5A4A7A29B928E8E8B7E
:10B98000857F78777D7B6F6E707072726A64676E88
:10B990006D6764666869656061646767696B6D702F
:10B9A0007178848484898E9EA3959D9E8083A29ABB
:10B9B00093A5A097998E8895908282848A86756FC8
:10B9C0007A838379767D8078767676726D70716B06
:10B9D0006361666764615D5B606A6A6265757D78F4
:10B9E0007179868C8D8A858993948F89878F9390BE
:10B9F0008E8D85828A9390858390949192938E9078
:10BA00009798948D89878889857C7B7B7C7B7772EE
:10BA1000757571717474797972727A81837D7C80A5
:10BA200081828484868685868D918F8785929A9679
:10BA300090959CA2A4A09D9CA1A39C9C9C93909259
:10BA40008E8789837875787B77716E707273726F69
:10BA5000767A7370747375787778777578756D7298
:10BA600077797A7773797B7D84827F888D837E88EE
:10BA7000948A7C82908F8B8B82828E93928D878723
:10BA80008078848D7B6B6F7A817B71737E7F7A7710
:10BA900079787881867D7B8386847D7B8A837E79B5
:10BAA0007881867D797C82868080898B8985838474
:10BAB00085797784847D7B7978767577746B727BF2
:10BAC00079766F6F7B7774828882807A78828A8AAF
:10BAD0008174778183878780808790958F8A8E8A0B
:10BAE000848B9291908B87888E918E898080898DAE
:10BAF000847873797E817E76747D83817A767E8880
:10BB0000857E7A787C83848688837C858880858E10
:10BB1000897E828A8A898989898482848A847D7BD4
:10BB20007F807E7E80827F7A79797D7F796E727761
:10BB3000757376737675727171737A7C77797D75AA
:10BB400073848D8782858784878F8A868A88898D8A
:10BB5000908D888587848184837C8081838C887F95
:10BB6000808488887F797E7C7B7C7B7D7E797C7EEF
:10BB7000746F757773717374797C7A777A81858342
:10BB80007E7B7F878B888684868886828181858379
:10BB90007D7D8284827E7C83847B7B867E797A81B4
:10BBA0008077787E7B767372757977737170777929
:10BBB00071797F777E857C7E8783848D8B8B8B8666
:10BBC000878E8E8A88878889868487888A908F85E1
:10BBD00082878C8E88838B8F857D818587857D7D0F
:10BBE0007C7B8488807B7C8186827D7D7E807D7C61
:10BBF00080817D83898585888886868789848186FA
:10BC00008581828A8C89868A8B898C8984878A87B8
:10BC10008285878480848988817E838784827E81EF
:10BC2000807D80817D7B81898B877D7C82807A7716
:10BC3000797D79777E7F7C7D7A7A82868585807D25
:10BC400080858685807D7B7D8182827B777C7D7D02
:10BC5000827F7A7C7F7F7D7D7A787A7E7D78757829
:10BC600077797D7B7676787A7B7D7E7A797A7B7E32
:10BC7000817E7976797D8286827D81838687817DCA
:10BC8000848685848080807E7C807B7B82828388A2
:10BC9000878084868483827F8484807F807E7C7D8D
:10BCA0007E7B797B7A787A7C7D8185827F818484B2
:10BCB00086847A7A7D7F8085817F7F81807F7F8087
:10BCC00080828385837C7D858683817F7F7D7D7F68
:10BCD00085837C7D7F808185898785868783828631
:10BCE0008684838889817B8185858585827C7C812A
:10BCF0007F8081827D7B7C7D81848787838385842F
:10BD00008381878A858082868381848887848383F0
:10BD10007D808B8988837C7C838383847C7D7E7D0E
:10BD20007F7E7D7E7B7671737A817E797677777E72
:10BD3000807B797C7F7F7E7E80807E7E7E7D7E7F25
:10BD4000808587817E8189878582828183878A88B1
:10BD5000828183858484807F8387877E767B8181CF
:10BD60007F80807D7A7E8182817E7D817F808583D8
:10BD70007D7D848785838383848A8E8C8583858972
:10BD80008A8988888583878886888E8C8784848240
:10BD90007F8184838485817F7B79818B80797679AB
:10BDA0007F8285847C777B7C7F86878786837E798C
:10BDB0007B828583817F7976797F8588847F7E7D8C
:10BDC0007D8385807D7A7D81827F80858887838160
:10BDD000807E7E818485817E7E80848787857F7C4E
:10BDE000818181817C80847F7E86837C7C7D818350
:10BDF0007E7978797E807E7D7E7F7C7A7E84827B70
:10BE0000797678807C7371717281817371757881B4
:10BE1000857D7D7D777B827F7D82827C727E837C47
:10BE20007574787D7F7A7C7F85847E75797F7F7F4E
:10BE30007D7B7F85837E7B7B7C80827C7C8078732E
:10BE4000838C847D7A7B807F7C84908C83828083CA
:10BE5000919C9A91867E879393877F869595857E20
:10BE600086909490857D7E83898886838185867D72
:10BE70007B868C827B75768289837B767D8B8377CC
:10BE8000797D878D8781817C8289817A7F878B8488
:10BE9000848985859190857F7F858B857F8A8C7944
:10BEA0006E788281837D7372737983867E75767CEA
:10BEB000827F79757B87897C7D8383878C87828766
:10BEC00088858788888D8F8986878B8B8683858DEB
:10BED000909092867F8B8D8182837778817A71773B
:10BEE0007C7E7D736B707A7A7372737273757376FE
:10BEF0007B79787B7872787C7576797A7D7C7E7FA9
:10BF00007976808382838385837E8591877D83870D
:10BF100082858C8B8683868C8D8A827F85837F7CCD
:10BF200079767980847D757A786E7581827F7D7C63
:10BF30007F7B798187837B757984858183838893EF
:10BF40009085828280828686827D7F878684898EA4
:10BF500089827F7F8387888A837A798286878684AD
:10BF6000817D7D828582808788827F7F7B7D8786B9
:10BF70007E7E7C7E85817C838683838584837B7FB4
:10BF80008E94877B7B8388848288897D77828B856A
:10BF9000848B898686838181838A8C7F7E7F84835C
:10BFA0007F878979787E7A7C85857D7471787B79C5
:10BFB0007B7E7F7E79788084827F81837F7C7F8493
:10BFC000817D7A7A7E7F7D7F85857F797B868E8B6A
:10BFD000827C80838383847F787A8082828282805D
:10BFE0007B7B8082817F7D7F7E7D7D7D7B7F858663
:10BFF000888C8881818384818283837F7C8285820F
:10C000007F80858684827F7D808285857F7D828812
:10C010008987827F7F818788878480858281898BD9
:10C020008B8D8B858485868B8780808080868B88AE
:10C030008282848383817F7E7D7C7E7F7F7F8184FB
:10C04000838482827F7E7E7D7F7E7C7B7B7E7D7E05
:10C050007E7B7C7E7F82808082807F8082807D7DEF
:10C060008183817F7F7B7A7D8386847F7F818183CB
:10C0700084817D7C7D7E7C7B7C7F808285847F7DCE
:10C080007F8083817D7C7B7D8284837D7A797D7FC7
:10C090007E7A78787E827C787C7C7E817D7B7A7AE1
:10C0A0007B7D7E7D7B7979787B7C7C7C7D7E807FCF
:10C0B0007F7D7B7A7A7C7E7D7C7A787C84868482A4
:10C0C000838182858788878686888885828385851F
:10C0D000858482817E80828383848482818281813F
:10C0E00081818584827F7F80808283817F7F83843A
:10C0F0008684828281817F7E7D7D7E807F7F7F803E
:10C1000080818584838282838383858382838687FB
:10C1100087868584848686848484848488868384D0
:10C1200088878582848585898B89878485838387B1
:10C1300085807E7F8282828182838383827F8081E9
:10C1400083858581808284868484848788878380B0
:10C150008386828183807E7F8181828181807F7FCF
:10C16000838584817F807F7E7D7E7E7C7A797C7DE5
:10C170007F7E7D7B7A78797A78777777787778772A
:10C18000787C7E7E7D7C7E7F808082807E7C7C7BD6
:10C190007C7A787B7D7E7D7A7A797B7E7A7A7E7FE7
:10C1A0007D7B7D7D7E7E7D7E808183858786878782
:10C1B0008889878786848382838585828282828339
:10C1C0008280838483838385888888878486868425
:10C1D0008584848687858587868585868584838111
:10C1E0008182848384878886868685858685848403
:10C1F0008585858383828386878485898B898989E0
:10C20000868686858586848283848280807E7F7F01
:10C210007F8080808182817F7F7F7E7F7E7D7D7C2D
:10C220007D7B7D81807E7F818382807F7F8085860C
:10C23000838283848182827F7F808080817E7F7FF2
:10C240007E7C7D81827F7F7E7E807E7C7C7B7B7B13
:10C250007B787676787B7A7A7A79797A7877787754
:10C2600078787577787A7A797A7A78787A7C7D7B3B
:10C270007B7E7E7D7E7F7F808280808180808081CA
:10C28000827F80818484838487888684848685866F
:10C29000858584858382828384827D7D7D7E7F7F88
:10C2A0007E7F7F7E7E7D7F7F7E808182838383838E
:10C2B0008282828282818183828386898B8C8C8731
:10C2C00086848486898A88878888868789898888F9
:10C2D00088868789878586888989868686858585F3
:10C2E0008584848586858481818085878582828214
:10C2F00081817E7F7E7E80807E7A7978797B7A7973
:10C3000079797B7A7C7D7A777B7D7D7A777A7A7989
:10C3100077797B7E7F8183808082848283817F8224
:10C3200082817F82818082817F7E807F8081828204
:10C3300082828382818080828582807F7F808280EA
:10C340007D7A7B80817F7B7A7B7E7D7C7C7B7C7928
:10C35000797A7A7C7D7E7E7D7E7F817E7D7F807F07
:10C360007E7E8184827F82868483848381818383AD
:10C37000838485817F7F8386868484848182828092
:10C38000807F7F7E7F8082808286848486898A897E
:10C3900087878583868A8987837E81848483828256
:10C3A000848381818486868284848486878883814D
:10C3B00082838689878281878986828387837F8338
:10C3C0008784807F8285858382828486837E7D7D4B
:10C3D0007D7A78797A7B7D81807E7D7D7E7E82818B
:10C3E0007E7D80807E7D7F7F7C787B7F81807F7D6E
:10C3F0008083817E7F7F8080808486817D7F807D39
:10C400007C7E807F7D797A7C7D7E7B7E7F7D7D7D5D
:10C410007E7C7D7A7D7E7B7D7C7B7C7E838581823C
:10C42000817D828785807E7F8182807F7E7D7E8008
:10C43000807F808281818484828485837F7C8086E2
:10C4400088857E7D818482807D7D7F807F81807DE7
:10C450007C8084827D79797D7D7B77777C7E7C7E14
:10C460007F7D818382807F7D7C7D81817F7C8284D2
:10C4700083817D7E808080808186827F8389898898
:10C4800086868A88848987858A8A88878888888832
:10C490008584888C8F8A8585878787888384838233
:10C4A00080808082848485838080817F7C77797C92
:10C4B0007B76767D7C78787C7D7B7D8084818080B6
:10C4C000838481817E828787848181828486878537
:10C4D00083838888858283878A8A837F8084878410
:10C4E000827E7E7F7F82827C7A7E7D7E7F7E7B7D68
:10C4F0007F7B7C86847D7C7F7E7F8387827F828238
:10C50000808283808080807E7F7E7E7F807F7E7C35
:10C510007C7F7D7C7F7E7E7F7E7F7F7E7F8183812F
:10C520007E7D7F808284837E7A7B8185837E7A7B19
:10C53000828483817E7D8183818487817F828684DA
:10C5400082827F80838485878281868981808380BF
:10C55000818689837A7B83868080837F7F808285C2
:10C5600084818281818285817E81838280808385AE
:10C570008383878A868586878684837E7E82847F7E
:10C580007F817E7A7C80817F7976777B7B797C7FE7
:10C590007B74797E7C767777797C7F7C7B807E7AF2
:10C5A0007D7A767A808080807D7B808889807C829D
:10C5B000898D898585878482838281807F81848437
:10C5C0008282848587888380828686848280807F39
:10C5D00082827C7D83838285878484868686817E31
:10C5E0007E7C79797A7D7C797A7A77788185848086
:10C5F0007B7A7F807B777C7F7E7D7F80807D828859
:10C6000086807D7B8389877C77797B7E7C7A7B7A49
:10C61000787B83837E7C7B7E8588817E7B7C818129
:10C620007F817D7B818A89817F83868281888B85DA
:10C6300083878A8988888888888A8988898A898678
:10C64000858886817F8286837C80858683818281BE
:10C650007E81858686827A7B8488837B7E848681C0
:10C660007F7F7E808282817E7D7C808886817E7EC7
:10C670007E7F7C7D84837F7E7E838D8C827B81899F
:10C680008B858385837C7A828B897B78838B908E64
:10C69000857E858B85818387827C7A7E797C7D7E91
:10C6A0007D79797F7E7E7E7C787C807C7A7C807FC1
:10C6B0007E8083818082828184848181818486835B
:10C6C0007F807E7C82827D7C7F7D7C808282848272
:10C6D0007E7D7F7F7D7C7C7F7F7D7F827F7E7F7F75
:10C6E000838586837D7B808587827E80808082872C
:10C6F0008882818381808485817F7D7E828482801F
:10C700008083868786827D80858381827F7C848901
:10C7100086818184878887878582828280858883D5
:10C72000807F8183828384827F7E8082817D7D8001
:10C730008182807D7F8485848382838885828080D6
:10C740008281817F807B7B7F817C777E837E7B7D06
:10C750007F807E7C7E838481807E7F8282828383D1
:10C760008280807E81817C7B7F81818285858482BD
:10C770007E8188847F7E7D8185807A7A7A7E7F82C1
:10C780008485817D7D7D7C7F7E78797E807A797CD1
:10C790007F807D76757B818380797B827B7E7F7FC6
:10C7A00080817D7C7E7D7B7F83817B76797D7E7CB5
:10C7B0007A797E7F7879827E777F87848486828388
:10C7C00088888B8B8484868585827F7E807E82812B
:10C7D0007B7C8387888281817C7D8386847D7C7F4E
:10C7E000838080827E8184818387898A878483860F
:10C7F0008787868284858582807F8183888B8781F5
:10C800007F808789888885868D8C878584868B8FB5
:10C810008A878484888A8A8A8883828787868783AE
:10C8200081828180828082858583828080817F7FF2
:10C830007E7B7A7C7E7F817F7F807F80807D7B791D
:10C840007C81838382807F81848284837F7F7E78E2
:10C8500075767B80807A787C808485818184837EF4
:10C860007C77747673706F6E6E777B777778757779
:10C87000787470757776777C7E79777B79777B7F34
:10C8800081888F888284827D7D81807F7F7E7B7A94
:10C890007C80828382848887898D8E8E8A86858239
:10C8A0007F8185837F7D80828182878D8D8D888247
:10C8B000838684848788858587888B8B8A87878A07
:10C8C0008E908985878584878E908E898C8E8E90B8
:10C8D000918D91978E8685807F8789837D78736E11
:10C8E000737B7D7B7F817B787876787B79797E7EA0
:10C8F0007A7C7F7D81868481817E7D7A787D7E7F52
:10C900008187858079777A7C7F7F7E7D7878818743
:10C9100083868C857D7F86878583888D8A8E8D86AC
:10C92000898C8B8E9288818587818386848484819B
:10C930007E7E7F807F817F7A77726F70706C6D7979
:10C94000828485847F7C76747A7A777B7E78787629
:10C95000706F717273716E767D7A75757B7D797685
:10C9600078797E8382828283827F7D797D888F8DB4
:10C970008A8F948F837D7D7D7F7F8086878583826C
:10C980007E7E7F80868E8F8D8E8B81797A7C797981
:10C9900078797F8085898B8D8A837D777D7975779E
:10C9A0007A76747B828181837C7673777F84878EAD
:10C9B0008B87888583898B8D8E8A85817F7F77732E
:10C9C0007C8081827E7A7C78716F70747376828DC0
:10C9D0008C8A8B8E928E8A837C7B7875737877763F
:10C9E000777C7D7D8085888E908985837C7981891F
:10C9F000898B8F8B8A8F938E8A8D8F908F8A8A8E68
:10CA00008B878990948E8B8C837B7E7F7B7D807DD2
:10CA10007D808180838B8C888885807C7472727025
:10CA20007374767777797D7E7E7C7C82807C7B7B5D
:10CA3000787C7F7F84817D7F7D7D80807C7C7F8012
:10CA40008284888C8C89827E7F7D7F8585858884A1
:10CA5000807E7F8387888384817E80818384868AA9
:10CA60008B878180807D7C818786827D79767572D7
:10CA70007377777A8081838989898C8A87888D9278
:10CA80009394999793969A938B8A8B8A8B89827EBB
:10CA90007874706D6D6D6E707678787B797B7B7C49
:10CAA000818383878C8A85898C8886888C8A898310
:10CAB000828583818080807D7C7D7F818285888A5C
:10CAC0008D908E8D8C8C8B86868B8D8D89838080CE
:10CAD000807C7574726D69635F5C57575855504E12
:10CAE0004C4D4E4C51595A5E656B778D98908B8E9C
:10CAF00096A0A9ADABA8A8AAAAB1BFCAC9C5C3BE12
:10CB0000B3ABAEB4B3A79381746A605F5F5C524409
:10CB10003B3A455056524E4F545B67727C7C7D8148
:10CB20008A969B979796959495908782807C70665D
:10CB30005C55555453524D4C4F565D5E6068737C46
:10CB40008389847F8C9DA8AAA3A1A6AAB1B5B3B3FB
:10CB5000B4B8C0C5BFB8C1D2D8CCB8AEB1B3A79035
:10CB60007C7B7F725845485B655F53576A7C7C725B
:10CB70006E75858E89898E8F908E8A8983817D746A
:10CB80006C625B66624B453F2F47532B1D33332747
:10CB90002B35434B4B556A7B82808392A1A4A4A47E
:10CBA000A7AEB7B9B6B4B5B2B9C9CDB9B3C4D6D0CA
:10CBB000C2C9D9CEBCCBE0CBAAACBFB7937C85961B
:10CBC0008D6D5B6D847C5F586C7872665B6172758D
:10CBD00066595C65645A57524C51564D3E39404433
:10CBE0003420202D2A1D1E2D303138404656676CCA
:10CBF000707A838E9196A4A8A4A9B2B0AAB6C0B642
:10CC0000B1B5B9B7AFAEC3CDB8B3CFDCCACADEDDFC
:10CC1000C3C2DED0ABB9D2BC9D99A3A2706C6B63CA
:10CC2000615C59595451564E48585A4D525A5856AB
:10CC30005D5F5D5E5E5A61645B565759585550485A
:10CC40004346504D464E5E615B64757D7A808F929F
:10CC500090999D9BA3ACB1B1ACB1BAB1AFB7B1AC37
:10CC6000BEC3BCB0AFC2C9BBBEC8C2C1C3BDBEC0DB
:10CC7000B9BBB9A89B9B94816D60645D4340483CFF
:10CC8000363D3C373B3D3E3C3A434736364C574FAA
:10CC90004C566266686A6B6F7474706F6E696C680C
:10CCA0005D5E656665677076767C84848796989706
:10CCB0009F9EA0A5A7ADB9BAB6B3ACB0BAB6B2B78D
:10CCC000BAAFADB9B3A2ACC3B7A2B4C8B7AABFC21A
:10CCD000AB9EA19A897E7F7259545D4C3A454D4373
:10CCE0003A3A3A3E403F403E434F4B4656645F66B9
:10CCF000777E7A7A848A868585808283786C707262
:10CD00006B6C6E6C6B6B6E716F727D7D7985918FC4
:10CD100097A3A9A8A9B4BCB5B5C1C2C1C3BEC1BFC0
:10CD2000BFC1BCB5BEC8C6BAB9C5C6BBB2B0ABA65A
:10CD30009C887C7C79675B5B595654453A40423508
:10CD40002C373F39373D444F5A555868716F7078CA
:10CD5000858B85828F95908F918B84827C7A7C7C69
:10CD60007A746D7174696976716D7C888584858D3E
:10CD70009A9E9CA3A69FA6B4ABA3AFB5B5B4AEB222
:10CD8000B3B5C5B38390C9C7A3A4B9BCADA0A2A6CF
:10CD9000A19683747672645A534E52513739423D8C
:10CDA0002A26393F34343C46555452616B6B696BCB
:10CDB0007585868186867F8184817E82847C737678
:10CDC0007C79747A7D746E787971788280777C87CB
:10CDD0007D7C97A1898092A5B2AC989FBCBEAEB075
:10CDE000B5B0B2B1ABA8ACB7C1B7A9B4B59C969E6B
:10CDF0009B9B957E7A7E756F6855555B4B40494984
:10CE0000403A373A3D3A3837383C3F3E434C5A6215
:10CE100062667783898889979F989BA7ABA9A5A706
:10CE2000A39EA19C93928B807C7C7876716D7D9B78
:10CE30009F75618AA3837D9B937688A9A0899CC1F5
:10CE4000C3B8C5CBB09AAAB29C8C99B0AA97A1B32B
:10CE5000A58F9092897D797A6B5F645F4C403934FD
:10CE60002E272B3B36303B413F4448474B54646BA5
:10CE7000656D7B7D808E939197A4A8A7ACB3B3AF6B
:10CE8000AEAA9F97948C868B8B756E7C82766E7221
:10CE9000737177787272797C7C82878B9CA2A3A64F
:10CEA000AEA8A1A7A9A4ABB2ADA69E9FB0BAB6B1D9
:10CEB000B4B4ADA6A0968B7F767066594E48433EBB
:10CEC00039342922293734292D373C404243424303
:10CED0005165626075888A8C959EA4ABB0ADAAA896
:10CEE000A9AAA5988E8E8A837B7170746F67676913
:10CEF000686A707E8787878E8E8D9FA99A9CAEAD5B
:10CF0000A7ACB4C0C0BCC2BEB8BDB3ACB7BDB8B4AA
:10CF1000ADB4C5C0B6BDB8A4968D846E555B4D3B0F
:10CF2000363A352C2A2923283839353E494E566061
:10CF30006A737B7B7C87949A9A9CA09F9C9A968B21
:10CF40007F7E7B70605E61554B525252595C616CC2
:10CF50007782897D768AA09D97ABC0C1C2BDB0BCE7
:10CF6000C9B79F99A2B1AE9492BADAD6C2C5DAD443
:10CF7000C3C1B39D948B7F6D4B42585340342C41B9
:10CF80006A66433D4A5868686A737077898A868101
:10CF9000808C886F6E7A766F685D534C463B3F4459
:10CFA0003A373E455059585F6974818486939A9EFA
:10CFB000A09EA1A2A5B1B1ABB5B4A7A5A7A5AFB5D9
:10CFC000ACADD6FFE8BAC3E7F0DABDB2BBAE918232
:10CFD0007161646656454B63736F67748FA09A974F
:10CFE000A2AAB1B2A79D958A897E5E535C5E4D333D
:10CFF0002A3430221E1C1D25292323334B4F45552F
:10D00000666D707175858F8D8F959B9B949CADAA75
:10D01000979399A2A398939BAAC6CCB6CBD8D8C90C
:10D02000ACA2A69579645A5A5749434C5762717617
:10D03000798FA9AFB1B7BBC1C8BFAEABA79B8E7983
:10D0400061666F55302C302C261D242D2624292274
:10D050002A3934333B434D4E4B5F7072757D8B9D47
:10D06000A6A5A5AAB6B5A8A1A3A29E999397A5B176
:10D07000B5B7B5BFD1DAD2C3B4ABA799837473790E
:10D080007268676C77838A959FA3ADBABCBFC8C925
:10D09000C2C7C9BCAEA096918C8071684D42342441
:10D0A0001B18161310141B1B1E252D344353616EC1
:10D0B00077889DAAAAAEC0C6B6AAAEB5B1A3989607
:10D0C00097958A7B86AABAA798B5DBE6DBCED1E135
:10D0D000DFC4B5B3ABA299867A75726B5F5D62658A
:10D0E0006466768382889BA5A39E98A0AA967C7E80
:10D0F0008D8A6D56585F4E30212324170F151B1C47
:10D100001A1C2D444C505D7590A0A2A4B0BBB7A7CB
:10D11000A6AFAA9C938D8F9288838E959AA2A29C8B
:10D120009A9EAAB8B9AFB0C3D3CAB5B3CACDA287C5
:10D130009AA1846D6A757E6D555E75786D67707F96
:10D1400084736874837A6A6C777662504A504E3F73
:10D1500033363D3A2F314046414150636867768609
:10D160008585929FA49F979EA8A49A928F98A19933
:10D1700086889A999188879DA294A1A28CA4C2B016
:10D18000AABEC1BDB2A7B4BBAEA7A4A4A5968A8F00
:10D190008E847B7778746760656764585E5D4F48FE
:10D1A0004E5655463C434945413E4450504F5864C5
:10D1B0006D706D76868B87888B929D9F9BA2A6A2B1
:10D1C000A2A5A5A09D9C9D9C9895908B919B958DCB
:10D1D0008F999A96918E89888781787779756E670D
:10D1E000646A6E6C6D7275797F8182888B8C8F8F8B
:10D1F0008D8E9197958F8B86827C726F6E6758515A
:10D20000555048484A4F4F4C54646B6C727A838532
:10D2100086888D959A959493929086848B807E8251
:10D2200081817D75767D7F7C7D7F83858686888DF7
:10D230008E8C8E8F9090918D86807B7D7F7E7D7A87
:10D24000787A7C7A787F838083898A8A8D90908EA1
:10D250008C8D928F86807F7D7E7E7D7B797C8485A0
:10D26000848D969A9B98969C9F9A97979594938C69
:10D27000837D8287837D7B7E7B76787F7D7C8188C2
:10D2800088817B7C7F7F7A7A7F7C7A7B79747674E5
:10D2900071717376777673737475767A82898F8FEE
:10D2A000929392969B999493928F90908A888A8C6D
:10D2B0008E8B8B939C9C999C9EA3A39D969A9997E9
:10D2C000938D8B89847C787774736D6260666968EE
:10D2D000686766696F7375777981828083898883CF
:10D2E0007C797A756E6D6D6C676461646B6E706F5E
:10D2F000717270778288878587888C89868382821D
:10D300007E79787B7C7C7A797A7E7C7A7B7C838759
:10D310008B8A83818B909090949590878786827B6F
:10D32000716B6A6A66676E7679787F868583848694
:10D3300087878786878A857B757477787A7C7D7BFB
:10D3400078777774727373737880807B7D7F84893C
:10D350008A8A8D90918F8B8A89878986827F808047
:10D3600080818384848A8C8C8F908D8C8C8A8C8B2A
:10D370008582828080807B7777716F73736F717322
:10D38000767B7D8183817F818488878482878B8778
:10D39000828084878B918E8782817F7F80807E7F51
:10D3A00083807B7D8589837E838783817E7A7D8070
:10D3B0007E81847E7C7D7E7C7E7F82878989868457
:10D3C000848582858986807D7E88888185867F8127
:10D3D000837F7D7C7B807E7F817D88988C807F743D
:10D3E000708293A7ACA1A0927C858E85857F727197
:10D3F00069677C7D7483857A7B7F7F7B746A5B46FB
:10D4000041506D96B5C9CBB491694331394F6764CA
:10D410004E4E607393B5D1ECF0DDC09768656163E3
:10D420005F50556E7C8C9C9894A9B8C1CBC1AB91D0
:10D430006D54515060748296A3A5AEA695938D7DD0
:10D44000828A8993A0A0988C837E7A7A8082858A4A
:10D450008F8F9298978F8E867E82837E848B898A27
:10D46000898A918F85765C49474B5A7C949BA19E13
:10D470008A735F545D718187867E74706C646162AB
:10D4800062626B79868F928B7C6D68686F7873733C
:10D4900077736F6E707B8B8F9598928B7E7D7D7985
:10D4A0006E6B6F74787C7C87918D87857D7B7A6DC0
:10D4B00068747372858D7F8396948D908976737767
:10D4C0006F6E78766A6459505868788698A6B2B6B6
:10D4D000B0A29486705E57575D6C788597A2A4A21F
:10D4E0009A8B7B6B636263666D79848B8F8D867D8F
:10D4F000726C5F585E5E5C69757F95A09A98949295
:10D5000095918684827B797D88969B9A999B948954
:10D510008A94969BA0988E8C8B8C8F8C847E747151
:10D5200072777D828A8F909298999288877E6C5DBF
:10D530005C5F616771777982887F7C84847A767496
:10D5400070686976807B7A879299A3A5A6AFB0A20E
:10D550009B9994908C8B96A4A8A5A0A0A49F94902E
:10D56000908C8D929696918F8D8E8C877F79767028
:10D5700070736E6E726C686A69636A6F6C6A6762F8
:10D5800059534D48494C5258626A73879393929607
:10D590009A9A93868897968A7F7B7D7E7A8C9FAFB6
:10D5A000BAC2C0B9B1A8A3A2A4A6A49F9184796D60
:10D5B000696C70788181807E7468646563686D6D64
:10D5C0006A63575150494049514F525559687274D6
:10D5D0007E92A2A9A08D8484745B4D4E5865707AAA
:10D5E0008192A2A6A7AFBFD0DEDCD2CBC6B5A08CFD
:10D5F0008991928C898D939796979EA6ADB1B0A88C
:10D600009A8A7458484138312B252F46595F6573E3
:10D61000848882786C63573F231715151C273F5F5A
:10D620007D91A1BBD4D8DBEAF3F2EBD8C5B5A492C7
:10D6300089848891989FA9ADADB1B8BCBCB5B0A69E
:10D64000927A634B392C25273855697077808B8FF8
:10D650008881827D6B4D2F1C141111121B2F46598E
:10D660007496B5CEE2F1F9FEFFFBF1DECEBFA692D5
:10D6700081797A7C7C8695A0A8ACAEAFAFA79C8C54
:10D680007867523B261B182432393F5164707476F8
:10D6900075756E5A443B342A2321222E4A58708FC6
:10D6A000ACBED0E7FCFFFCFFFEFBF3DFCABBADA5C1
:10D6B0009E96918F8F8D8F919296999A93887A6A80
:10D6C0005A45301B141518222D3742515C5E5F619C
:10D6D0006868635C55504B454448525E6C7D91A42C
:10D6E000B4C3D0E3F0F1F2F5F4E8D5C5BBB5AFA90A
:10D6F000ADB5B9BAB3AAA7A29B90837D7563524A10
:10D700004339322D2E2E2E3233303436302F383EE0
:10D7100040454B535F6262666B7173748590999D4F
:10D72000A0A8B4BCBDC4CDD5DCDCD0C5C5C1B6AFE6
:10D73000ADAFABA39B999791888586837E797573EE
:10D740006D625959595755514E4D4C4643454B50B2
:10D7500053595C5F6062686E6F71767E8184868BE0
:10D7600091989C9EA4B2BFC3C6C8CBD0C9C1C1B258
:10D770009EA6B3AFA8A49D989185807F7A78767392
:10D7800075767474777774727073736D65636263A2
:10D790006465676D6F7275757573716D67666567C2
:10D7A00067626264686D747B86939C9FA4A6AAA935
:10D7B000A6A4A2A1A29F98939294929191939496D9
:10D7C0009493928E8A888585827D7571737675773C
:10D7D0007C80878D92949290908F8A8482817B74D2
:10D7E0006D6865656566686A6F727270707577746A
:10D7F0006E6B686766625F636C707071747A818447
:10D8000083878D9091928F8D8C8D8E8F9497969922
:10D81000A0A7ACAEAAAAAEABA4A09C988B837E793D
:10D82000756F6E6E6A6767636263646A6A68676869
:10D8300063625F5C5A5D5D5C606366676E7474779B
:10D840007B8084868686838183838484888C8F9181
:10D85000969C9FA3A6A6A8ACACAAA7A29D98938DC0
:10D860008A88868383848587878C9090908D868232
:10D8700081817D7C7D7D7C7D8080807E7F7F8082BC
:10D8800082817F7E7B7A7D7B79797D7C7F807F80C2
:10D89000858480807F7F7E7E7E7D7C7D7E787877AC
:10D8A0007372717474777A7C7D7B7B7D7F7F8384D8
:10D8B000818285838687888C8D8E8F9192928F8DC1
:10D8C0008D8E8F8E908F8F8F8C8D8A87867E797AC2
:10D8D0007978767472716F6E706D6E6D6B6C6C6B47
:10D8E0006C69676869696A6C6D6D6C6F7272767B62
:10D8F0007B7B7D7D7B7C7D7E7E8085898D919291F9
:10D90000969797989B9E9F9F9C9A989595918F909C
:10D910008D8A8A888381807F7E7D7A7A7473716F25
:10D920006C6A696A69676664636366696B6E6F7067
:10D93000747A818382818185888E9293928F8B8B7A
:10D940008E8E8F8F9090908F90908F8F93949594D0
:10D9500093918C8C8E8F8F8D8A88888A8B89848016
:10D96000807C7A7C7E7B78726F7277787B808E9BEE
:10D970008978818683878A8783716783998A74749B
:10D98000807F6E71808079726864718595978A7DD9
:10D9900071686B7784888C8B82756B6A888D8780C1
:10D9A0007C808788858A939797938E88898C8E96BA
:10D9B0009D9B91878079757B868F908B85858483ED
:10D9C000888F91908C8A877C73747B828482817E1D
:10D9D0007672777B7F7F7F807A6E70808F98968C4F
:10D9E0008786817C7A7B807C716764697583877E9A
:10D9F00077706A7583837B716E757A7B78777C8BA1
:10DA0000908986828085909A9B958F867B7A858E79
:10DA1000908C827E7E7D7D7C747284A3C4AD7D59A2
:10DA200059768E92723D0F01103C6F836D462A31FC
:10DA3000588AAFB7A1919BB4CAD2C7BABBC0B8A12C
:10DA400083707996ADB0A79380879DABACA99B8777
:10DA500079758299AFAE916B52566F817C58280BC5
:10DA600007132B423F220F152C4B707F7268738E69
:10DA7000B5DCF3F3E1CDD1DEE3DCCAB29B89828869
:10DA800091968F7B6766748D947D656485AEBDAE1F
:10DA90008D71718C988971563F383F3F35312823FD
:10DAA000263755757F756B6C88B1C4B59A909BAE5F
:10DAB000B4A8947F6F6D77868B88817D8190A2AAB0
:10DAC000A59279676F8EACB39D746582A3A99B8381
:10DAD0006A513C36495F54393040647F7E747B84A0
:10DAE0008691A7BDC5B19382858E968C705247539F
:10DAF0006E8B959096AFC9D7D4CBC4B99E7655544A
:10DB0000799C97725A6C95A8957A695D463A4A5005
:10DB10003C3142648B977D6E8BB4C2B092948D7E03
:10DB200065473C4D5E6260687C9FC1D8DCCCB8B470
:10DB3000B7B4AB9065423D455D839B8E72759BB7D4
:10DB4000AF9C8C7D7C765D3C25212E476C89826A5A
:10DB5000729DC1BA917C93AFAB8E6A5464868A6C15
:10DB60005A6C89A3BABEB1A1929CC2CFB691716919
:10DB700074786859638A9D806C85A6ADA18F827C7C
:10DB80006F58371E20313E4F6A787687AAC1AF8A18
:10DB900087A8C0B089707B9DA4886F6FAAA7988C56
:10DBA000858CA7BAB2936E6272867C553E465F84BE
:10DBB0009B81616E91A49B81747A7D72553623227C
:10DBC000334D554E49597D9FA69389A4C9C29C9255
:10DBD000AFC8BC938097B2AE91776F7789A4B7B383
:10DBE000998B9AB5C7BB977377918D706D868B6E45
:10DBF0005C70878577726F6358472F1A1D303934F0
:10DC00003242556E92A19491B1CDCAB3AFC6CAB497
:10DC1000A5AAA68E6E5B5F6D7979767B9AB5C9C72A
:10DC2000B7ABABB2AF916750577081714F486988FD
:10DC3000856B5D68736E5B412D1F273F463B364405
:10DC40005E757C879BA6A29DA7BECDC1A79BABB5E9
:10DC5000A07E6F6E70747A8487838DA3B5B2A0990D
:10DC6000A4B1AA8D7574796F58474B5866665545AF
:10DC70004C636B5C473D435869695D5A697F888393
:10DC80007D8195A8A99D98B0CDCDB6AABDDAD7B2B1
:10DC90009AA1B6C1B8A497979CA3A69C80839094A0
:10DCA0008269616A7879644B423F42494434292948
:10DCB00034464C484B5257585C686F6861616678CF
:10DCC0007F73778E9AA5BCC6BEC0D4DBD5D2C9B24D
:10DCD000A4AFBCB49A8790AAA89192A099857E8798
:10DCE00088746B7064545D696054525A6B777771B5
:10DCF0006D73828374646269675A5860625B65778A
:10DD00007E7E7A8188898A8D8F908E8D99A8A89D34
:10DD10009FADBFC6C2C2C8CFC9BBB4AD81797A714D
:10DD200059433E4958626665707C8288857F82844B
:10DD30007A737478756D6467758992846C6E889354
:10DD40007F6159687977634F566F8184807B8CA897
:10DD5000B4A9958FA0A6937A6C686C65564B485110
:10DD6000626E69666C7682949E968D8E969A8F838B
:10DD7000818183817E88979F9D97969B9FA2A49681
:10DD8000888994968A797378869396948F8D8C8FF0
:10DD900090908F897968666D736851465F6A695C97
:10DDA000576D8B9588777486999A836C6F818E8B6B
:10DDB0007C7172879C9E96949BA2ABAEA69D9DA003
:10DDC0009C938D8E9191908D8D8A817974767F81CF
:10DDD000786D6968666768636066747C7770758261
:10DDE0008D90867A787D80776660666767656770F4
:10DDF00078838A8D95A0A49F99989B9D9A918882FB
:10DE0000828588847A72737D8376696B777A736F83
:10DE1000727B7F7C7C849095928F919396928D8576
:10DE200079747B7E77706E77878C807B8598A099DC
:10DE30008C8991938F8A837D818A8D8578757A7E8E
:10DE40007C756A63676864605F616567697074792F
:10DE50007F817F808486837F7F7C777779797A7BE7
:10DE60007C858F92969CA2A6A8A9AAA9A7A9A59EDF
:10DE70009896989B9A90888B908E857A787C7B7CFC
:10DE80007A706B6E706D696D7275797D7D7D808243
:10DE9000817B736E6D6E6F717070747A8183838114
:10DEA000878C8F909393949594989A97959390904C
:10DEB0009194938D8782868D8D87828283828788D5
:10DEC000827C76777D7E7A757271706F6E6F6F70FF
:10DED000727171767B7D7A7B8184817E7B7A7B7D9A
:10DEE00079777A7D81848482818081878B897F762E
:10DEF0007A868B888079808A8D8A868284898983D4
:10DF00007C7B7F827F7B7A7977787A7A79838B883A
:10DF10007F7E8286867F78767374777673767B7F52
:10DF20008385868586858481807E7D79717175760D
:10DF3000797D7F7E7C7B848E8D837F82898D8986AF
:10DF400084808085858182838382828387868382A1
:10DF50008182888B8B88828487888D8C8082867C66
:10DF60007A817F7B81817A75747A85857D787B83E0
:10DF70008887837A79848C88827F81868F90877E58
:10DF80007E8082817B787D7F7B7B80848A8B878586
:10DF9000898D8D8B8A8683818282807D7F807E8140
:10DFA0008384878D897E7C7D808584817D7D838946
:10DFB0008A8A8A8B89888889837B787B807F7B7734
:10DFC00074767A8085837E7D82868586847D76736D
:10DFD000727271747774706F7983837D7D82888BA0
:10DFE0008A8F908D8B847C7B7B7D79747987888602
:10DFF0008F928577717780786F7073737379828869
:10E000008B909598958A7F797671707273706E6C2B
:10E010006C777E7A767C82868985807E7E76757A3C
:10E020007A7D7E7A7A7E8180878F8C8A8B92999393
:10E03000898284868686848687898C8D918D868365
:10E04000827A787C77716C6967696F757977747A91
:10E05000828485888E8F8D8D8F8F8B83848D8B832B
:10E06000878C9194908F9496928E8E8B8F948E87BE
:10E070008485827E8288898784858A89847E7D7E64
:10E080007C7A7B7F8081827B767B7F8286817E7DAE
:10E090007F7C7A7B79767775716F6D676A6D717049
:10E0A0006B6D7074767C828B9092949BA0A0A0A0E4
:10E0B000A3A6A6A6A8A7A4A0A1A29F958F8B8B8597
:10E0C0007A6F6A6964584C494E52525354534E4CBD
:10E0D0004E52585B5A5B5F605B514E5055585960C9
:10E0E000707A7B7B84939C999BA8B9C3C6C5C8CF23
:10E0F000D2D2D4D8DAD7CEC7C5BEB1A8A29E968652
:10E100007A726D665A4F4B48423D3F4A51493F40F3
:10E11000433C312F364246403E444943414F5A60CA
:10E120006875848F98A3B4C1C7CCCED0D8DADADAB8
:10E13000D9DCE1E4E0DEDBD5CFC9C2B8B1AAA49A4C
:10E140008D7E71665F5A5650463F3D43545A4E4845
:10E150004F4E41322D3945494A4758726C504D5700
:10E160005F6B70737D858D91919EB0BCC1C5C9CF29
:10E17000CECAC9CAD1DAE1E2E2E3E1DACBBDB5AA9F
:10E180009B90887D6D574840393535373C3D302769
:10E190002D456A7C7C8B978E7D644A3B1305040772
:10E1A0000B172B4B78A8CCE5F1F7EAD1BEAE9782DE
:10E1B0007D777987959FB3C8D2D8DEDDD6CDC4B838
:10E1C000A99A89735F5041312724242831404F6335
:10E1D00078848D918B756060645A4B4B50565A5AB7
:10E1E0005E6F7E7D787B7E8084878890A4B6BBB985
:10E1F000BABBB7A891837D79726E768A9AA5B2BAB6
:10E20000C5CFCEC7B9A8967D6351453C3E43464E27
:10E2100060676C747C7F807A6D5E51444D5E62678E
:10E220007685898685888984796E6A6D6D74859412
:10E23000A0B0C0C5BFB1A4978A7D737376787D8383
:10E2400095AAB2B4B8B8B5B0A28F83786B676A717B
:10E25000787F89887E7A796F655E5C6165615C5BD9
:10E260005D6E7D80797A7D786858575C5C5959601D
:10E270006A707A89939CA6AFB5B4ADA7A6A29E9DFD
:10E280009E9F9E9B959598999490919496938F8933
:10E2900084807E7977797B7B777371767D7E7F7DD5
:10E2A00076695E646F6B5F6069675C4F4C53544D79
:10E2B000484448535A61748EA6B6BFC1C1BDB5A5C6
:10E2C0009C958C8A8F94989BA2A9B1B7B9B6AEA23F
:10E2D000968C837B777B7E80878D8E8C827E7C760E
:10E2E0006C66656063798C8F8B8F8C7A624F423A53
:10E2F00032251F253040556A83A0BAC7C2B9B9B2CA
:10E30000A7978B8C969C9EA3ABB4BFC1BFC0C1BE68
:10E31000B8AC9F9C9A90837E787978685A60605BED
:10E3200057595F60595E778F8E8C939387756357CB
:10E330004F41332724252B36486284A9C2C9C7C55B
:10E34000CAC3AD9E9A9A938B868994A4B6C0C9D14C
:10E35000D6D3CAB9A8A193807D77665C574E434651
:10E3600050595B59595D57546B8A8F88878E8670D8
:10E370005243423D2C1D1E21232D3A4E6D91B2CAAF
:10E38000D4CFCDCFC3ADA2A6A89D9396A2ADB1AF79
:10E39000B7C8D6D1C7BDAFA2928274684F443C3A89
:10E3A0003B40474D58656D6B686A768A8B7B757A02
:10E3B000735E4B4347433A34313038434F637FA158
:10E3C000B7B8B8C1C6C1B4A9ABAFA698949CA4A76E
:10E3D000ADB8C4CED2CCC2BCB1A192857767584C3F
:10E3E000433E3C414A51565F66696963687C8C894B
:10E3F00081828277665957584D3F3A3733384656AF
:10E400006A88A6BABFC1C7C8BEADA2A1A39D939595
:10E410009B9FA6AFB8C5CCCCC8BEB4A98F8074678B
:10E4200057493F3B3A3E44484E555D62605C6987C0
:10E4300095918F8F8677675A5751443A33323742D6
:10E44000526682A5C3C9C8D0D0C6B8A8A3A6A29A4E
:10E4500096959AA7B4B8BDCBD1CBC4B8A798887706
:10E460006A5E4E4343404148515D65696C6E67602A
:10E470006C848F8D838182755F4E46423E332726A2
:10E480002A3342546A8DB1C4CCD3D7D9D7CBBAB2D0
:10E49000AFABA49B9AA6B4B6B8C1CDD2C2B5A99A67
:10E4A00088796B6359514A43434C50504F505757EA
:10E4B00054627E8F8A8286897E6754514F3F281C22
:10E4C000181F2E3A496A8FAFC3CAC7CBD2D2C8B27F
:10E4D000A4ACB7AC989EB0B6B1B0B8C8CCC2B6AD1B
:10E4E000A69E93867A70665A534B464B50494345D5
:10E4F0004949454E6C858D89878C8E7D65574E4286
:10E50000312018232E3842536F90ACBBBDC1C8D107
:10E51000CFC4BBBCC0BDB6B1B8C1BDB6C3C8BCA733
:10E520009DA0998B817E7E7A6F65605D56504942D1
:10E53000444747404154707C78777A7D7869544DE0
:10E540004F46342625323C414F6380A4B0AFC1CB47
:10E55000D4DFBF92ADD8D4CCCAC4CBD4CBC2C0BE5A
:10E56000C0BAA8979195948471767D786D65656938
:10E570006961584E4A433932353532394C595E66F5
:10E580007682817B73685A48362828343F4E6D92D4
:10E59000AECFF0FFFDFEFDF5E9D9CABAB7B09F9E38
:10E5A000A8ACA39A9A9A9C988E7F76726D61575701
:10E5B0005653515153545756575B61635A4C495205
:10E5C000555353575E636560616E77716B6D706F05
:10E5D0006B6B77899BA4B2CADFEAEDEDEEE6D6C598
:10E5E000B8AFA49686807E7A747478848C87818094
:10E5F000807C746F6A6762635F5853565C606363C4
:10E600006264635C57534E4A434245474B565E63D0
:10E610006974818A90979FA4A7A9ABAFB0ABAFB83C
:10E62000BDB8AFB6C1B6A39A9B999182746F6F6B58
:10E63000626171807C7789A3A7907F838E938A7BA8
:10E64000706D6A646C7265586170706F6C696B6D27
:10E65000615256615F585C6A6D6A727D89939896C3
:10E6600093979B94939A99969D9D979DA5A19D9B09
:10E670009896938B8891969997908E949B9FA0A142
:10E68000A9ADA6A5AC9C827D7D6B6A7975727F7100
:10E690005458665E6061453748524A426A72616703
:10E6A000776F686F737173757479889495928B84A2
:10E6B000899595919EACA093A2A99DA7BCADA2B748
:10E6C000BDB2AFAFB0B1ADA1908890978F81737597
:10E6D000858779635D64625C5C564F5C574A57601E
:10E6E0005054717767595B6F79686582856D728A5E
:10E6F00084787976787B70768D8A8C9B8C6C728B23
:10E7000090929EA08D8084848DA19C8E949191A0E6
:10E71000937F98AA959EB6AC9FA7A5908C9880658C
:10E7200073857E7A7A6D6A7B7F797B8386817C7440
:10E73000696E6F61666D5C637B77717061636D6933
:10E7400067707169656F796E647076696876827FCB
:10E7500077767C7B777E8B86808A87848F8C8D9F73
:10E760009994A3978FB1B9A8B4AD95A1A99FABAD6A
:10E770009EA3A79A9B9F9897958D908A70667B81A0
:10E780006F64645D555E675B55594F43515C504EF5
:10E79000595B5E615F5F564E657A695F6A747E772A
:10E7A000717B7F7C7F818491958A8A9DA39FA3A69C
:10E7B000A29D9CA6AB9F9CA4A5A09FA4A29DA4A142
:10E7C0009596978E8889837D7C7671757163647167
:10E7D0007066645D5F737564646D767A736E757769
:10E7E000717881786F79827E74748694817687954A
:10E7F000908E90878696A0938C9391929E9A939AEE
:10E8000093848C9C9388969F9086959A8981838027
:10E8100082878378757E847975817E7A8B7577811E
:10E8200076737973717D86867E747582867C737249
:10E83000726D6C6E6971818789867781968D7D8115
:10E840008079868D847E7E7C89989B9E9B8B7F8041
:10E850008384817E81837E787C8D988A83918D8C60
:10E8600099846979867D8685777F86818C89809475
:10E870009983797E7E7A736E6B6F79716B73696140
:10E8800070766F717A82837F7E7D828671687C81EB
:10E8900076706B7C9D937F8C998E7B77918B979A0A
:10E8A00088868A86888E909287747480868A84741B
:10E8B0007B8D806E7783827E7A7986908B8480755B
:10E8C0006C727D7E7A7F817B8897897C817D7B7F5E
:10E8D000777576717D87777A867F828D8781858847
:10E8E0008A8377747A80817D787A85928F84869006
:10E8F000948E797489887883898389877A828C8ACF
:10E900008476747D77757C736A726D68747C7271BD
:10E9100078797376857B6470857E7C7F6F84877D54
:10E920007A7E868C8F8F8A8796988A887F79888F5F
:10E9300092988B879699939DA1968C817679807B0E
:10E94000778288797789887B82938E73738E9A9386
:10E9500090887B786F6A7A80695F6A707578787959
:10E960007A797E7F7C828A83828D897B787A777EB2
:10E970008D88798691808097A39C978F7C778B99DF
:10E9800090888589968A7F999A7675847C87968601
:10E990007C8B8C8187938A7F85807A856E75807267
:10E9A0006B767B838479788F9273637478747E7FBF
:10E9B0007476756D747B6E6878807A787B82908CC3
:10E9C0007D8B967262848D787A7F7D8C917F828830
:10E9D0007A7A81818A8875839E9686818085857DF5
:10E9E000878D899490787A898B878184948F7777C3
:10E9F00090A29A86858885959D847B8E8F8186904E
:10EA0000908A7E7A7D8087877872888B75788B85EF
:10EA10007F83777B94948085998B7986756B6E71F3
:10EA2000807B57597C827E8679768F907A7A858D25
:10EA3000836D6E8D8F65516B85858080889AA690D9
:10EA40006F707A76777875898F70709294858875F3
:10EA5000627C896A526076775F566F7C747A7A69D5
:10EA600069685C6F938F75737E7D8A9C91889B9F8C
:10EA70008F898F908C8C99A293818995949792809D
:10EA80007D8A8982869094866A708E8F705E6C8093
:10EA90007B788687879891736E7A8E9E82785F5690
:10EAA0006C74707F8781786B6A6D6978877B787703
:10EAB0005D649299838183807F7A7B89907E6D717A
:10EAC0007A797A807E7976727E8F7E5D74A3A69441
:10EAD00090807795B0998095AF9F8C9BA89E9A92D5
:10EAE000898F8C7169737671726B636155495A6F46
:10EAF0006760768288918F8C928D91ADBBB6BCCBCE
:10EB0000C9B9B1A98D75684B3B4957637B7F829624
:10EB10008F796D50352F23131621334A6F859EBF91
:10EB2000DAE6ECEFF0E8D1BCB5A68F7C63586A7BDF
:10EB30007B8CA8B5B4B5AB8F70543A271A141A243D
:10EB4000243857667FAFBAA5A7BBCBD2CED0CFBBF8
:10EB5000A8A59A95998F7E848F959D9C8F7B6248FE
:10EB60002F1C171B1C181A2135516983959BA6B7BA
:10EB7000C0B5B6CEDACFC3C9CFCBC8BDADAAA798B2
:10EB800087776650392415101010152636425872B2
:10EB90008597A5ACB3B0ADAFAAA5ADB9C6D3D6D253
:10EBA000D0CBC1B3A290795E49321C141419202B2A
:10EBB00039506D889CADB8BAAF9986776B62606E3C
:10EBC000828FA3BCCAD2D6CCBCAA998771533A29EA
:10EBD00022262C34475C7391A8B4BEBBA88F7A62FE
:10EBE0004D454A54678194A6BDCCCDC9C0AE9A8923
:10EBF0007259422F282B31425B738BA5B7BDB9AB3D
:10EC0000977E5E4D46404555647B99B4C6D3D6C9C0
:10EC1000B8A9947A624B3A35383E50699BB2BFC26C
:10EC2000BBA88D725A473E3F4755657C9AB5C8D4FC
:10EC3000D7CCBEAE987B624F3D373B44546B869D2C
:10EC4000ADB8B6AB9A85705A473E3D465463758D54
:10EC5000A8BECED3D1C6B39F89705E4F44454B53F7
:10EC60006273818F9A9D9389817469605A56585C4A
:10EC700065778B9CB2C7D3DBDED7C7B9A38C7A6A22
:10EC80005A4F4D4C545F697580888D8C87807568AC
:10EC9000615D5A5E68788B9FB4C6D5DDD4C8B9A2D1
:10ECA0008D78624D403A3A414C576677848B8C8E12
:10ECB0008B857D726A646366728597A9BDD0D5D550
:10ECC000CEC1B2A18C7869523E332A2B353F4F65B5
:10ECD0007788969B9C94897E736E6E707889A0B4B9
:10ECE000C5D1D6D1C7B9A99788735A473829262ED6
:10ECF000384860748491959690847A706A6A707BC3
:10ED00008DA0AFC1D1D8D5CBBFAF9F8D7C68543F0C
:10ED1000332C282D3642526377868F9590857F77E6
:10ED2000767B8390A1B5C4CFD6D5CCBFAE9F8D7B6B
:10ED30006958483B322D2B3441474F5D6F808B9093
:10ED4000908E888381888F939AA8B7C5D0D3D1CA73
:10ED5000BDAC9C8D7A6956443A332E2D3641494DCF
:10ED6000535F6E7F899093939393979CA4AEBAC39D
:10ED7000C9CDCCC4B6A799897765524339322C30B6
:10ED8000353C44494B505C6E7C8A99A3A4A4AAAF3D
:10ED9000B1B6BDC4CACECAC3BBAD9C8C6B5E514775
:10EDA0003B332D2B323B4144474A566677899AA420
:10EDB000A9ACAEAFB6BABDC4C9C7C3BBB0A6998A29
:10EDC0007D7265594C3F382F2932393D40454956AF
:10EDD0006B8195A4ACAFB1B4B5B4B6B9BDBEBBBA86
:10EDE000B2AAA4978A7D70645645392C22222C340D
:10EDF0003B3F434E61758A9CAAB3B6B7B8B8B6B468
:10EE0000B5B5B2ACA8A6A39D94897E7365584E464D
:10EE10003E362E2D2D30383E44556776A3B2B9BE0E
:10EE2000BCBBBBB9B4B4B8B9B6B2ADA8A0968E8617
:10EE300080786D635848392D282C32374D697F937F
:10EE4000A8B4C1CCCCC9C9CBC6BAB3B3B2ACA7A025
:10EE50009B978F8986837D736455442C1A161A21DB
:10EE60002A354D6E808F9FB0C1CCCECECAC3B8A616
:10EE70009EA3A7A3A1A0A09D9897948A7D6B5847B5
:10EE8000342215151C212A384C69818F9DB2C3CAC2
:10EE9000C3C1C0BFB8A9A1A5A9A6A5A6A39A8F86DC
:10EEA0007D725E4D443A281A191B242D384A63742A
:10EEB0007F96B1C2CED2D2D6CFBDAFAEB9BEB8B2B8
:10EEC000B2ADA59C938C86755E5045372A1F1715E9
:10EED000171A22324C6474849FBCCDD4DBE1DCD1A0
:10EEE000CAC8C6C5C3BFB7AEA0968A827A69534561
:10EEF0003E332418131819171D212C435B6D829A79
:10EF0000B2C8D4DAE5EDEAE7E2DBD1C4BEB8B0A01E
:10EF10008C83817660514A44392E292724252E3945
:10EF20003E404F697C8894A6ADBAD3D5CED3D0BE2F
:10EF3000BBBDB3B1AA99918A786F62524C463F4EDD
:10EF4000563E30373E3E3C455051586A6E707F9376
:10EF50009EA4AFB2AFBABFB6B7BBB5B8B9ABA4A0A9
:10EF60009287817464584F4542403E4245464E5117
:10EF700056656A6B74797D82868A8F959B97949883
:10EF800099A2A39596988C88857B787878776D6E12
:10EF90007872767F7C7B7B767878797D797E7C83CE
:10EFA0009597918D87837D838F837C868280847BF8
:10EFB000798178757E706E786F73867F79838080B3
:10EFC0008E908E969A9BA5ACA59EA4AAA298959089
:10EFD0008D836E69736B606060676E65687270794F
:10EFE000817C7F7E75797E819095979C999EA5A660
:10EFF000ABAAA7B1AD9D9E978C98937E7F898B8A93
:10F0000080777B7A6F70695656615E636F6967714E
:10F01000726F6D727B817C7576787D848B98968912
:10F020008C847C8D979BA8A2978C828E93828C95E2
:10F03000888E98939894827A6E6C828B8F92817866
:10F040007A6E686A595152494A5B5D5B64696A76B7
:10F05000848B8E8A888C96A2ABB7BBA89EAEB0ABD1
:10F06000B8B6ABB2ACA4A89B8C88786C756F6060A6
:10F07000676F6C656C6F6863585E757778837A74B8
:10F080007A777982888B8E9392868D998A83887F0E
:10F090008180727685807A79787D7C7C77717377D0
:10F0A0007A756A6059616F707E8A72667879798440
:10F0B0007672818181877980938685978B78746554
:10F0C00065717480837D7F7E777C7D839392949736
:10F0D000898E9C8C89988E8C9B9589867A80969750
:10F0E000959E9A908F867E8D968B827C7C8C89747F
:10F0F0007078726F6E707B797274787E847B6E78B4
:10F100008179808B837F8D877E8B958C8E95909176
:10F11000918E908E857B7B8A98A09B94988D8D8D07
:10F12000817C7774878F807D82817B7B8585777FEB
:10F130007E6D6F695C64645F655E5865685F5E6282
:10F140006B71768487899497958D80828476788197
:10F150007F84867E8C94888C8D7E89948C94968610
:10F1600081796F777E7C7C838A7E666A756D768016
:10F170007C838778777A787D7E838F8176858373A9
:10F1800078848D9A8D738096908B877B7C7E707A45
:10F1900090919CAFA9A3ABA9A4A1A1A489837D83CD
:10F1A000867779817A808268677C7E86897A706BBF
:10F1B0006C7A766468736C6C6E63656B6A7C8D8642
:10F1C0008A978A8FA6977F7B6A65757D7F847F7912
:10F1D000787C7A6B6A79777F908787968D81867C39
:10F1E00077888E8A8E939896857F8180847D6460EF
:10F1F0006B6B635A55605E4E5C6B5C57687F8677BD
:10F20000799096A0AB9894AA9C9099857F949997B1
:10F21000A09E8F807577767B867C6B6D7479726F1C
:10F2200073767B7C7A828B8E908EA1B7A49AA69CF3
:10F2300098A8957E8D87717D8B7E76756F777767C1
:10F24000667073706E75828F9596999E9490979064
:10F250008283807471757B7D7B7B7B808A90866ED8
:10F260005C6572695A5A5A5D738388989B817E9750
:10F2700092858F8E8DA2AEAFADA1979997948D8D0B
:10F280009583758B8664666E6770706E7D756F7C16
:10F29000715F676E68696F7E85797780797D7D782B
:10F2A000808185948E7D8C988C939480776E69761E
:10F2B00077676F80807B808A8B8D97918888858027
:10F2C00086929AA09D887D91A2968D887E7A70699B
:10F2D0007575686A6D6E797971757B7C7E88928DA3
:10F2E0008B8D8181928F858682859088818C939089
:10F2F0008E89756C7677675C5D636564707B747A04
:10F3000089867F7A727A7F8093947F828A8B9296A5
:10F310008F90887D838B867D8082746D7F7E766DF5
:10F320006B67657175767F807F81879390817E8C16
:10F330009388797B817A767A7E817977888F8C8FB2
:10F340008E89826E6A6F67748A91A2A8948D8F826B
:10F35000868771665F4E55687899B3B7B5A9A1A441
:10F36000947F7562514E4A53646C7C8E8E95AABA16
:10F37000C7C9BBB4BEC6CBD6D3B9A18A6652544F57
:10F3800049463F3D4D5E7EA1ADB5C0B49F8D776FC0
:10F39000736A5D5C4F48525D656E788CB9C8D5D68E
:10F3A000CABAA898836A58524F4C4C566D8EB3C453
:10F3B000C1B8AC9986776755402F2322283B5573F7
:10F3C0008D9D9FA0A1988A796B676358555E626393
:10F3D00069737D7F8393A1A1A09E948C817C848797
:10F3E00080818484898DA0BDCAC6BDB09E8F765FA2
:10F3F000513F30241C253542597C9BAAA8A29683F4
:10F40000716B655A4B3E42515D6879929EA5B4C3BB
:10F41000C6C3B9A0887563626A737E858C9293A017
:10F42000BACDD0C8BBAB9A836A554838261E273858
:10F43000465D7D9BB1B7B0A59982675F5E5244413E
:10F440004C6171819AB3BDCAD3CEC5B499826B5455
:10F450004C54606F7F8F9B9D9CACC7D6D4CCBFAF04
:10F460009C8977685B4833292E39465C7C9AB1B811
:10F47000B3A79783706B66523E3D47545D6C88A579
:10F48000B9C4CFD2CABEA8907A5E4947515A6A77AA
:10F490008599A9B7CEDDDAD0BFB0A08B66584534C8
:10F4A000292C3844556B86A4B3B4AE9F8B7E7970FB
:10F4B000614B3D3D4856606F89A4B6C4CBC9C0AD11
:10F4C000957F69555059636F79879AAAB6C4D7DE7C
:10F4D000D4C7B9AA9786735C493B2F2D333E4D6143
:10F4E0007E9AACB4AFA1989085786753403A37358F
:10F4F0003B4A5D738BA3BDD1D2C7BBAF99867665FE
:10F5000061615B5C6773839CB2CAD9D9CFC1B3A375
:10F5100092816D56413224212C3848618E9BA1A2E4
:10F52000A4A9ADA79B8A76695C49414246535D6BAD
:10F53000858E7F89A2A9ABAEAAA29B979282756F96
:10F540006B708091A3B9C0BBB4A898897B68594CF3
:10F550003D2B202028364A5E727B818C9EAEB7BD43
:10F56000C0B8A28A776A6262676F7779797B869B77
:10F57000AFB8BCC0C2BCB3A99D90857C7673767DC4
:10F58000888A8A8A877C7468605F5C534A40373710
:10F59000404F5C667179899DA9ADB3B38F786B6676
:10F5A0005D565C6260636D788899A9B5BEC4C2BAC5
:10F5B000B3B6B3A79E9E9B9799A3ABAEA89F978B1C
:10F5C0007C71645B5143312D31333A4249535E655E
:10F5D0006E767C81807A6F5F504B50585C5B5B5CD1
:10F5E00061748CA2B4BDC0BEB9B5B8BFC2BCB1AD68
:10F5F000AAA8A8ACB8C3CCCDC8B5A39589827E72A1
:10F600005D4E474A525E6C777C7E7C7B7C807C734F
:10F61000675443363030343B3C3A3C41586B7E892A
:10F6200089868688909AA1A8ADADAFB2B8C5D0D969
:10F63000E2E3DCCFBEB3AA9E8E81786E6C6F767FDC
:10F64000858A8A888A8782807C6D5947392D231F55
:10F65000252B2C2D343F5263697179777070798333
:10F66000898B8C8B8E919298A7B5BEC2C3C2BBB456
:10F67000AAA49E90827F80807F838C98A4A9ABAB44
:10F68000B0B0A79F9486766559514A45423E3D48A1
:10F690005763717B7C7A746A6869686559514D4B10
:10F6A000525B6877848E989EA2A7A8A9A4A09A937B
:10F6B0008F8E9094999A9FABB5BFC8CBD0D0C9C05C
:10F6C000B39F8E7E6C605851535B656D6E6C6F7628
:10F6D00078787B7B756A5F564E484646494A4F5359
:10F6E000555D6A727E8A8A8683817E7F8082878961
:10F6F0008B949DA5AFB7C4D9E7E7DFD7CFC2B19D43
:10F700008C83796E6A7077797C838D9A9A948F85D1
:10F71000776B5F58514A453E3A3E40465C5E6061B9
:10F7200062605A5857575652535D6164737A7B88AA
:10F730009BA6B3C5D3D7D4D3CDC3B9B5B7BAB7B1E8
:10F74000ADABABA5A5ADB4B1A89B887D71635B588B
:10F75000534E4E5153575B60696E6B655D50423A34
:10F7600036373737373D444B566474818E9BA6A994
:10F77000AAAEAFAFB1B5BABCBDC5CCD5DDDEDBDE60
:10F78000DDD5C9BBAB9E8F81776D635C5B5D5F5FD1
:10F790005F666C6C6B69675E4C3427231F212C34C9
:10F7A00038373C4D5C616C808E908A888D969AA02B
:10F7B000A7B5C5D2D4D1D7DCE1E9E9DDCDBCAFAB8B
:10F7C000ACA69C8D7D6C62738793A4ABA1A0928242
:10F7D0007F654A35010E6F5F04123E4254646D89A5
:10F7E0009AA1A991776C574A4E525F6C6D758CAB9C
:10F7F000CCE3EAE9E0D3C9BEAC9A87746863656E6E
:10F80000767C858D9DB2BEBAB6B1A59988715F4AE6
:10F8100031201B202E3C516C8597A2A8ADA08A7385
:10F820005F4F4542455165798693ACC6D2D5D0C16C
:10F83000B19A827367594E4F5866748598A2ADBECF
:10F84000C6BEB2A596897A6551433730353D495FCA
:10F8500076899BA9AFAA9D8E7B6B5C4A4347515B1F
:10F860006A7E95AFBAB7B8C0BEB4A1897563534A72
:10F87000535C5A606C829CA69E979EACB7B2A297CE
:10F8800087736658493C332F35475B6F81929EA73B
:10F89000AB9F8F7B6457564D4A58647199B0C9D05D
:10F8A000C6BDBEB9AA8D72656466687379767B8BB6
:10F8B000A1B0AB98878B9FAEA49389817C72624D77
:10F8C000392B283850626B6F7A8FA1A093867565AB
:10F8D000615D534E5A66728499B2C3C2C2C8CEC526
:10F8E000AD8F7A716F7681867D7989A4AEA7958D6B
:10F8F0008E8C8EA2AD998683857F6C523A2E2D35E3
:10F90000435861677F9FB7C0B4A0928B83745743FD
:10F910004651647E8C8C9AB2C6D1CDB89089857BD5
:10F9200069585A626E86949BA79B8C9DAA96878E77
:10F930009A9F92807D7A6D5F4833282224354855FE
:10F94000698DACBABFBBAC9D91826A524242536290
:10F950006F7B899BB4D3DEDCD1B9A29FA49E8B7050
:10F960005A5F6F808E8D7F7E93AAB1A58E6D586091
:10F970007580755E546276786A51403E48627C7C40
:10F98000767F95A8AFA897836C5F697063555562C1
:10F99000768B96989EA8B6BFC1B7A4907867574F4C
:10F9A000556775798292A0A2A2A5A497866E4E4152
:10F9B0005774735C5B72888A7A6A66615C5F6B6E8F
:10F9C0006466809EB2BBB7A49A9F9D907D695B5987
:10F9D0006174878F939EB2CCD9D3C6B8A99E938306
:10F9E0006F5B4D4B5061767A777A8795988A726013
:10F9F0005B6A7A79665D6C7E7D715D4C464A5157D3
:10FA00005B5F667790A7B5BCB4A1989C967D615268
:10FA100056616D77818993A5BDCFD1C4AAA7A08A6D
:10FA20006F584E54595A606662698199A096877CD6
:10FA30007C81796A6C7568555F767D6D5A566B81ED
:10FA40007A645B5E697B99B0AF9A8F9FBBC0A388D5
:10FA50008897A19D88726E798EA4A89894A9BBC03E
:10FA6000B9A4928C806E60524344525C646A6F6E9B
:10FA70006A707D847A5F4F5F7F8D7C6672929F9201
:10FA80007D6860696E645D5F6781AAB49B96B0C84B
:10FA9000C6AF9797A49E88787475797B4F56626736
:10FAA000685F505267797A76727B91A3A2968C84B4
:10FAB000817C6B5D564A47505A626D7D9BB6AE9A0B
:10FAC000A3BAB99F8B93A09C8F8A8E97A0A1978F82
:10FAD000939C9E9589807E7C818173676C7E8B87E9
:10FAE0007D767984826E606970685E5D5C5F677543
:10FAF0008587797993A49985818583756B665E5A2C
:10FB0000606D73767E8D989A98A2ADAC94939FA603
:10FB10009B816E7F9F9C8B909080809BAEA79182F3
:10FB20008A9DA5A4988B848181827D6B594F4D530A
:10FB30005D62584E556A75736B666B7A7F818B8DEB
:10FB40007C737D888789856F5D708E8C7064738B04
:10FB50009692837E848886888B847C7C80838B8F3E
:10FB60008F91979EA8B7BDAB9DA6B3AF9B84757AC6
:10FB700080755C4A505F5D4C424E595A5E605958E0
:10FB800066737366616F7B7C82888B90A8A9A6B12F
:10FB9000B19B929C98847A7C756C6E777A767A8425
:10FBA0008784888A888C908F8D8A8E99A09E9D9D4F
:10FBB000A3ABB3AC9B969D9D958C847A7273786B46
:10FBC00050424246483E363945525E686B738491D6
:10FBD0009293979184828A8683868680838887879A
:10FBE0008B8C867F848F8C8386919B9FA09D96991A
:10FBF000A5AB9F908D8F8D857E777681939B9C9D05
:10FC00009FA2A5A29A8B7E7976665C5F56545B6450
:10FC10006D6F6B68717D7B716A6A6D6F6D62616B10
:10FC20006F6F70737674747A8286858890999C9BC6
:10FC3000999794928E8B8985817C787A7C8085894E
:10FC4000898D94959A9E9A9291979B9B9692929366
:10FC500096958D8888867F7C7C7D7B7D7D76767F82
:10FC6000848587847E7E807C70645D5959575555A4
:10FC70005A5E6266696B71716B70787C7A746F75AD
:10FC80007C7B797774737879797A7C7E868B8D8C9E
:10FC90008D90939696968E8B8C8F92939090919850
:10FCA000A1A7A29D9B9E9E988E888282807F808243
:10FCB00083868787888C8C877F7D7F7E7974737439
:10FCC0006E69686B6F6D67626566616163626266CB
:10FCD0006E7273726E7581848480848A9095989711
:10FCE000979A9FA3A4A29E9A9CA19D97979A9C9E47
:10FCF0009D989A979191948E847D797C80807B7772
:10FD0000777C7F858A867E858A84827F7A7A7574FD
:10FD10006F6D726E696D716D7173707074767878D5
:10FD20007476787C7F7F7E80838C92959692939A6E
:10FD30009D9694938F8A8986827F7B7A7C7C7B795F
:10FD4000767675777C7D7F807E7F81827C787878FF
:10FD50007879797471737775716E70727576747065
:10FD600070767E807E808487868484838385868582
:10FD700086888B8A8D939597999C9B9A97918C8571
:10FD80007E7F7E7C7C7B80838383807F807E7A788D
:10FD900079777677767577726F6F6C6B7376757827
:10FDA0007C8084878888888989857F79737274725A
:10FDB0007274797B7D7E8083848484848482828053
:10FDC0007D7C7C7D7E7E7E8080838584838586822B
:10FDD00084898B8A8986858685827F807F7F7E80E5
:10FDE0008183858A8D8B8C8C88878787878585859D
:10FDF0008485848281838482807E7E7F7E81807DF3
:10FE00008082817F7D7D7C7E7F807D7C7D7F7E7B0F
:10FE10007C7C7A7A7E7F80848786828488898686C5
:10FE2000858688857F7F7F80807F8086878687899B
:10FE30008C8887898A878482807F7F7E7E7B797B9E
:10FE40007A78777676787D7F7C7B7C7E7D79777615
:10FE500073727173757A7F7F8085898C8E8C8C909C
:10FE60008E8A8A878888858284858181828284823D
:10FE7000828284828385878988888889888483832D
:10FE8000838485868481818586868686888A89851D
:10FE900084837F7F7F7E7F82848385888786848535
:10FEA000878B8E8E8D8B8D8E8C8B8A8783817F7EC8
:10FEB0007E7D7B7A79787C7D7C7E7D7E81817E7C77
:10FEC0007876747373737879777B7C7D7F82848690
:10FED00088888988878684828486858383858481CF
:10FEE0008181838685817F7D7D7E7F7C7A7778792D
:10FEF0007B7A7A78757575777B7B7877787A7B7C77
:10FF00007A797B7B7C7E7D7A77797C7E797A787949
:10FF10007D7E7F807F7F82828181838486868686C4
:10FF20008686888B8C8A878889868381807F7E7F7E
:10FF30007F7E7E7D7F7E7C7B7B7C7C7D7F7F817FE7
:10FF40007E7F7E7C7B79797C7B797A79787A7C7FFD
:10FF50007F7C7D7D80838482808084858585858586
:10FF60008689898D908E90918E8D8E8A88888889D9
:10FF70008A8B8986858584838282848481807F7D43
:10FF80008084858787878988898F8F86747B847B27
:10FF900079848B857A839188808C89797F83797B3A
:10FFA0007B7473777D7C7273787070746F71767206
:10FFB00074767878747572646B7D716E7F7E757CF3
:10FFC000857D7780867A7F92867C8B8B848F8D85EA
:10FFD0008686878B8B9291889190868A85818C8A80
:10FFE000848A898E9589838F877F868383817A84AB
:10FFF0008D8B969D92939B9995918F927FEF7EF03A
:020000040030CA
:0A0000008CFFEFF79FFFFFFFFFFFEB
:00000001FF
